:020000040800F2
:100000000000011031AA03082559030829730108CB
:1000100035AB030835AB030835AB0308000000001F
:100020000000000000000000000000006D5F0308F9
:10003000695F030800000000655F03081D0A0108EE
:1000400035AB030835AB030835AB030835AB030804
:1000500035AB030835AB0308B98A0008E58B000807
:10006000A98B00086D8B0008318B00088DAB000850
:100070007DAB00086DAB00085DAB00084DAB000820
:1000800039AB000825AB000835AB030835AB0308D6
:1000900035AB030835AB030835AB0308F58A000818
:1000A00035AB030835AB030835AB030835AB0308A4
:1000B00005FF0008F5FE0008E5FE000835AB030863
:1000C00035AB030835AB030835AB030835AB030884
:1000D00035AB0308250C010835AB0308890B010873
:1000E0007F8A000835AB0308895F030835AB030836
:1000F00035AB030835AB030835AB030811AB00087B
:1001000035AB030835AB030835AB030835AB030843
:10011000ED0A010835AB030869A801084DA80108DC
:10012000FDAA0008E9AA0008D5AA0008C1AA00088B
:10013000ADAA000835AB030835AB030835AB03089F
:1001400035AB030835AB030835AB03082959030861
:1001500099AA000885AA000871AA0008510A010896
:1001600035AB030835AB030835AB030835AB0308E3
:1001700035AB030835AB030835AB030835AB0308D3
:0801800035AB030835AB0308A1
:1001880027000400A0280020A82900200000000063
:100198001006000816000800AC290020B429002029
:1001A800000000001406000801010400F02A0020E5
:1001B800DC3D0020000000000000000008020900EB
:1001C800B63D0020E03D002000000000018000084E
:1001D80002000C00C03D0020EC3D002000000000A3
:1001E80000000000F7010600B03D0020F83D0020A7
:1001F800000000001C0600080A020A008C2B0020E0
:10020800003E002000000000220600080312330010
:100218007F3F00204C3F0020000000002C06000813
:1002280025005A00983E0020F23E00200000000001
:1002380000000000F6110C008C3E0020803E0020DB
:100248000000000060060008012008005445002056
:10025800A0450020000000006C0600081A000800F5
:100268003C450020A8450020000000007406000856
:100278002C001000C0490020B049002000000000F8
:100288000DFC01082B002400F4490020D04900206F
:1002980000000000DDFB0108090201007E4B002080
:1002A8005C580020000000007C06000801020500E0
:1002B800945D00201062002000000000A92F0208B1
:1002C80000020500605800201862002000000000AD
:1002D800000000001E000400A05B00202062002037
:1002E800000000007E06000822000C00245B0020AD
:1002F8002462002000000000820600082900500047
:10030800D4620020E0660020000000000000000029
:1003180014000200D06200203067002000000000B6
:100328008E060008100003006C620020346700206D
:10033800000000009006000828000C006062002001
:100348003867002000000000940600082300100011
:10035800506200204467002000000000DDF2010820
:1003680019000500486200205467002000000000C2
:10037800A0060008F8110100446200205C67002014
:1003880000000000A60600080001040040620020EA
:100398006067002000000000A80600081B00F400A9
:1003A8006C670020BC680020000000006D45020852
:1003B8002F001100A0680020B06900200000000094
:1003C800AC06000815007000146C0020886C002032
:1003D800000000000000000003000100106C002075
:1003E800F86C002000000000000000002A006000F7
:1003F800206B0020FC6C0020000000000D97020814
:100408000C002400DE6E0020746F00200000000045
:10041800119E01080E20EA00D66D0020986F00207A
:10042800000000002DB7010813000400286F002009
:100438008470002000000000C006000802010300CC
:10044800C16D00208870002000000000399E01085E
:100458001F000E0058720020787200200000000073
:10046800C4060008050201004072002088720020BE
:1004780000000000D206000803010600D271002027
:100488008C72002000000000D4060008F901040066
:1004980044780020487800200000000045F6000855
:1004A80018102C00147800204C7800200000000060
:1004B80031080208FB010100E47700207878002069
:1004C80000000000E1610108FC010900B07600208D
:1004D8007C78002000000000A56101080A101200C5
:1004E800847600208878002000000000DA060008E2
:1004F80006001600547300209C78002000000000BD
:100508004DB7010805000600887900201C7B0020F3
:1005180000000000EC060008F511620020790020B8
:10052800247B002000000000F178020826000E005D
:10053800987B0020887B002000000000F919030840
:10054800FD011E00D08500202C8600200000000040
:10055800D5F50008FE010800BC8500204C86002067
:1005680000000000296201080B2010009888002074
:10057800D088002000000000F206000834001000B7
:10058800A88F00207C90002000000000359702080A
:100598000D002C007C8F00208C90002000000000B3
:1005A8004505030812100C00608F0020B890002049
:1005B80000000000020700080C0201005C8F002008
:1005C800C4900020000000000E070008020203008B
:1005D800708F0020C890002000000000000000007C
:1005E800FA0102004C890020CC9000200000000095
:1005F800396201080400800060AC0020F0AD0020E2
:080608000000000000000000EA
:1006100020030000C409000019012828240100005B
:10062000000000004A01B400D601270000000000CD
:1006300000000000000000000000000000000000BA
:1006400000000000000000000000000000000000AA
:100650000000000000000000000000000000010099
:10066000000000000000000000000000E80364003B
:10067000040A00017E05EA05B405320020000000EE
:100680000100C800141E010064002C0128000300B2
:100690000001050000000001000000000000000053
:1006A000000028010000040090010000000000008C
:1006B000000000000000000000000000000000003A
:1006C000080000000000000000000100000000051C
:1006D0000000000004010100000000300100005A89
:1006E0000000000090012C01C800640020000300FD
:1006F00001002B21231E64010100000001000A01FA
:0F0700002900000000010005464F52540000017F
:10070F00010000005001000007000000020000007F
:10071F0000000000000000000102030406070809A2
:10072F00010100009C090408903704080000000034
:10073F0000000000AC090408B40904080000000020
:10074F0001200000B8090408C009040800000000D7
:10075F0001400000C40904089C2A0408000000009E
:10076F0001200000D0090408DC0904080000000083
:10077F0004000000E0090408E0460408000000003F
:10078F0004000000EC090408EC1404080000000049
:10079F0001000000020100000000803F0000803FC8
:1007AF00FF00000028E00308050804000000000017
:1007BF00D0FE0308ACFB030814E0030800000000A0
:1007CF0054E0030805080A0000000000D0FE0308EB
:1007DF00ACFB0308ECFD0308000000000000803FA5
:1007EF00010100005DF8010800000000000000009A
:1007FF00FFFFFFFF010101002D202D2D202D2D2D9D
:10080F002D202D2D2D2D00000000000000000000D8
:10081F000000000000000000E00100000000803F29
:10082F0008FFFF00303030302D30312D3031543053
:10083F00303A30303A303000000101010100000041
:10084F00000001010C4604080F00000021AC020853
:10085F000000000000000000C4020020E045040872
:10086F000000000000000000000000000000000079
:10087F00903704080000000000000000580300201B
:10088F0004000000604504080D0000005DB302087D
:10089F00AC1B002000000000FC3E04080D0000000F
:1008AF002DB30208A01B002000000000EC3F04083D
:1008BF000800000000000000941B0020040000004E
:1008CF00683F04080D000000BDB10208881B00201E
:1008DF0000000000FC3F040803000000D98B030850
:1008EF00701B002000000000F0450408030000000A
:1008FF00D98B0308581B002000000000C03C0408DF
:10090F0001000000000000000000000000000000D7
:10091F00000000000E0000000000000000000000BA
:10092F0000000000E0450408000000000000000087
:10093F0000000000000000009037040800000000D5
:10094F0000000000580300200400000010450408B8
:10095F000300000061B10208401B002008000000E6
:10096F00683F04080D000000BDB10208881B00207D
:10097F0000000000FC3F040803000000D98B0308AF
:10098F00701B002000000000F04504080300000069
:10099F00D98B0308581B002000000000C03C04083E
:1009AF000100000000000000000000000000000037
:1009BF00000000000E00000000000000000000001A
:1009CF0000000000F84504080000000000000000CF
:1009DF000000000000000000903704080000000035
:1009EF000000000058030020040000001845040810
:1009FF0003000000D98B0308B81B00200000000083
:100A0F00C03C0408010000000000000000000000CE
:100A1F0000000000000000000E00000000000000B9
:100A2F00000000000000000020700020702D7200F8
:100A3F00D44504080F000000000000000000000073
:100A4F0000000000F0160020FFFFFFFFFA0000007B
:100A5F0001000000010000002D202D2D202D2D2D37
:100A6F002D202D2D2D0000000000000000000000A3
:100A7F000000000000000000A83C0408B03C04087F
:100A8F00B83C040800000000000000000000000057
:100A9F00000000008E3C0408040000002937020803
:100AAF000000000000000000C03C0408010000002E
:100ABF000000000000000000000000000000000027
:100ACF000E00000000000000000000000000000009
:100ADF00A67900200100C40900000000A4790020BD
:100AEF000100C40900000000A27900200100C40920
:100AFF0000000000A07900200100C40900000000E0
:100B0F009C7900200100C409000000009E7900209C
:100B1F000100C409000000009A7900200100C409F7
:100B2F0000000000987900200100C40900000000B7
:100B3F00726D00200100C80001000000706D0020E0
:100B4F0032003075320000006F6D0020055A05002D
:100B5F006A6D002000FF01006E6D00200100000093
:100B6F00780300206C6D002002000000CCFF03080A
:100B7F00696D002000FF01006D6D00200100000075
:100B8F00780300206B6D002002000000CCFF0308EB
:100B9F00E83C04080F000000000000000000000007
:100BAF000000000080030020107200209CFF2C0129
:100BBF0000000000F60000200A000000ECFD030812
:100BCF00344B0020E0150C1700000000F50000204A
:100BDF0008000000ACFB0308F40000200500000033
:100BEF00D0FE0308364B00200200000004FE03086D
:100BFF00166F00200100FF7F01000000146F00201E
:100C0F000200000010FE0308CA6D00200300000060
:100C1F0020FE0308C96D00200300000020FE03081A
:100C2F00C86E00200000F40101000000C66E002015
:100C3F000000F40101000000C46E00200000F40168
:100C4F0001000000C26E00200000F401010000004E
:100C5F00C06E002000FF0100DC6E0020E803D0070B
:100C6F000A000000DA6E0020006401000A00000094
:100C7F00DB6E0020006401000A000000D46E00202B
:100C8F00006401000A000000D96E0020006401001A
:100C9F000A000000D86E0020006401000A00000066
:100CAF00D76E0020006401000A000000D36E002000
:100CBF0000FF01000A000000D26E002000FF0100BB
:100CCF000A000000D26D00200000F40101000000B6
:100CDF00D06D00200000F40101000000CE6D002057
:100CEF000000F40101000000CC6D00200000F401B1
:100CFF0001000000CF6E002000C80100CE6E002062
:100D0F0000C80100CD6E002000C80100CC6E00208D
:100D1F00006401000A000000CB6E002000FF0100FC
:100D2F000A0000000B6F002000C801000A6F0020AE
:100D3F0000C80100096F002000C80100086F0020E3
:100D4F0000C80100076F002000C80100066F0020D7
:100D5F0000C80100056F002000C80100046F0020CB
:100D6F0000C80100036F002000C80100F03C040818
:100D7F000000000000000000000000000000000064
:100D8F00003D0408090000000000000024040020BA
:100D9F0004000000083D04080900000000000000E6
:100DAF001804002004000000BC42040809000000E1
:100DBF00000000000C04002004000000203B040889
:100DCF0009000000000000000004002004000000E3
:100DDF00103D04080900000000000000F40300208B
:100DEF0004000000183D0408090000000000000086
:100DFF00E803002004000000203D04080900000063
:100E0F0000000000DC03002004000000283D04085F
:100E1F000900000000000000D003002004000000C3
:100E2F00C03C0408010000000000000000000000AA
:100E3F0000000000000000000E0000000000000095
:100E4F000000000000000000003E04080000000049
:100E5F0000000000000000000000000060460408D1
:100E6F000700000000000000480400200000000000
:100E7F00103E040808000000000000003C040020A1
:100E8F00000000001C3E04080800000000000000E5
:100E9F003004002000000000C03C040801000000E6
:100EAF000000000000000000000000000000000033
:100EBF000E00000000000000000000000000000015
:100ECF00243E0408000000000000000000000000A5
:100EDF0000000000343E04080D0000000000000078
:100EEF0084040020000000003C3E04080D000000B8
:100EFF00000000007804002000000000443E0408B9
:100F0F000700000000000000700400200000000037
:100F1F004C3E04080D000000000000006404002097
:100F2F0000000000543E04080D0000000000000007
:100F3F0058040020000000005C3E04080700000079
:100F4F00000000005004002000000000C03C040816
:100F5F000100000000000000000000000000000081
:100F6F00000000000E000000000000000000000064
:100F7F0000000000643E04080000000000000000B4
:100F8F000000000000000000604604080C00000094
:100F9F0000000000746D002000000000783E04087F
:100FAF000C00000000000000766D00200000000023
:100FBF00883E04080C00000000000000AC6D00200B
:100FCF0000000000983E04080C0000000000000024
:100FDF00A06D002000000000AC3E04080C000000D3
:100FEF0000000000786D002000000000B83E0408EB
:100FFF000C000000000000007A6D002000000000CF
:10100F00C03E04080C000000000000007C6D0020B2
:10101F0000000000D43E04080C0000000000000097
:10102F007E6D002000000000DC3E04080C00000074
:10103F0000000000806D002000000000E43E040866
:10104F000C00000000000000826D00200000000076
:10105F00F03E04080C00000000000000846D00202A
:10106F0000000000E43B04080C000000000000003A
:10107F00866D002000000000F83E04080C00000000
:10108F0000000000886D002000000000043F0408ED
:10109F000C000000000000008A6D0020000000001E
:1010AF00103F04080C000000000000008C6D0020B1
:1010BF00000000001C3F04080C00000000000000AE
:1010CF008E6D002000000000283F04080C00000077
:1010DF0000000000906D002000000000343F040865
:1010EF000C00000000000000A46D002000000000B4
:1010FF003C3F04080C00000000000000A26D00201F
:10110F0000000000443F04080C0000000000000035
:10111F00B06D002000000000503F04080C000000DC
:10112F0000000000B26D0020000000005C3F0408CA
:10113F000C00000000000000B86D0020000000004F
:10114F00844604080C00000000000000926D00208F
:10115F0000000000683F04080C00000000000000C1
:10116F009A6D002000000000703F04080C00000082
:10117F0000000000946D0020000000007C3F040878
:10118F000C00000000000000966D00200000000021
:10119F00883F04080C00000000000000986D00203C
:1011AF0000000000903F04080C0000000000000049
:1011BF009C6D002000000000343504080C00000076
:1011CF0000000000A66D0020000000009C3F0408F6
:1011DF000C000000000000009E6D002000000000C9
:1011EF00943B04080C00000000000000AE6D0020CE
:1011FF0000000000A83F04080C00000000000000E1
:10120F00A86D002000000000B03F04080C00000093
:10121F0000000000AA6D002000000000B83F040885
:10122F000C00000000000000B46D00200000000062
:10123F00C03F04080C00000000000000B66D002045
:10124F0000000000C03C0408010000000000000086
:10125F000000000000000000000000000E00000071
:10126F00000000000000000000000000C83F04085C
:10127F00000000000000000000000000000000005F
:10128F00D83F04080500000000000000C86D0020D2
:10129F0000000000C03C0408010000000000000036
:1012AF000000000000000000000000000E00000021
:1012BF00000000000000000000000000E03F0408F4
:1012CF00000000000000000000000000000000000F
:1012DF00903704080000000000000000F800002014
:1012EF00040000001C3B04080D00000071370208C9
:1012FF00E404002000000000604504080D00000019
:10130F0065310208D804002000000000FC3E0408EC
:10131F000D00000031310208CC0400200000000055
:10132F00EC3F04080800000000000000C00400208B
:10133F0004000000683F04080D0000001D31020882
:10134F00B404002000000000F43F0408090000006E
:10135F0000000000A804002004000000FC3F040867
:10136F0003000000D98B0308900400200000000048
:10137F00C03C040801000000000000000000000055
:10138F0000000000000000000E0000000000000040
:10139F0000000000000000000040040800000000F2
:1013AF0000000000000000000000000010400408D2
:1013BF000D00000000000000FC04002000000000F1
:1013CF00184004080A000000000000002C6F0020E5
:1013DF0000000000244004080A0000000000000084
:1013EF00346F0020000000002C4004080A000000A9
:1013FF00000000003C6F0020000000003440040893
:10140F000800000000000000F004002000000000B1
:10141F003C4004080400000089B5020800000000E9
:10142F0000000000C03C04080100000000000000A4
:10143F000000000000000000000000000E0000008F
:10144F0000000000000000000000000048400408F9
:10145F00000000000000000000000000000000007D
:10146F005C4004080D00000000000000140500207F
:10147F00000000006C40040804000000E1B3020803
:10148F000000000000000000744004080D00000080
:10149F00000000000805002000000000884004083C
:1014AF0004000000BDB302080000000000000000AF
:1014BF00C03C040801000000000000000000000014
:1014CF0000000000000000000E00000000000000FF
:1014DF000000000000000000904004080000000021
:1014EF00000000000000000000000000A4400408FD
:1014FF000700000000000000500500200000000061
:10150F00B04004080800000000000000440500205F
:10151F0000000000BC4004080800000000000000AC
:10152F003805002000000000C84004080800000033
:10153F00000000002C05002000000000D44004082B
:10154F00080000000000000020050020000000003F
:10155F00C03C040801000000000000000000000073
:10156F0000000000000000000E000000000000005E
:10157F000000000000000000E04004080000000030
:10158F00000000002B03002000000000EC400408C6
:10159F000B00000000000000B80500200000000054
:1015AF00F44004080B00000000000000AC05002010
:1015BF0000000000004104080B00000000000000C4
:1015CF00A0050020000000000C4104080B000000E3
:1015DF0000000000940500200000000018410408DE
:1015EF000B00000000000000880500200000000034
:1015FF00244104080B000000000000007C050020BF
:10160F00000000002C4104080B0000000000000047
:10161F007005002000000000384104080B00000096
:10162F000000000064050020000000004441040891
:10163F000800000000000000580500200000000016
:10164F00C03C040801000000000000000000000082
:10165F0000000000000000000E000000000000006D
:10166F0000000000000000005041040800000000CE
:10167F0000000000000000000000000064410408AA
:10168F000800000000000000E80500200000000036
:10169F00704104080800000000000000DC05002075
:1016AF00000000007C41040808000000000000005A
:1016BF00D005002000000000884104080800000049
:1016CF0000000000C405002000000000C03C04081A
:1016DF0001000000000000000000000000000000FA
:1016EF00000000000E0000000000000000000000DD
:1016FF0000000000904104080000000000000000FE
:10170F002803002000000000A04104080B00000087
:10171F00000000001806002000000000AC41040883
:10172F000B000000000000000C060020000000006D
:10173F00B841040807000000000000000406002064
:10174F0000000000C4410408070000000000000072
:10175F00FC05002000000000D04104080700000035
:10176F0000000000F405002000000000C03C040849
:10177F000100000000000000000000000000000059
:10178F00000000000E00000000000000000000003C
:10179F0000000000DC410408000000000000000011
:1017AF002803002000000000E841040807000000A3
:1017BF00000000006406002000000000F041040853
:1017CF0007000000000000005C0600200000000081
:1017DF00F841040807000000000000005406002034
:1017EF000000000000420408070000000000000095
:1017FF004C0600200000000008420408070000000B
:10180F000000000044060020000000001042040801
:10181F0007000000000000003C0600200000000050
:10182F0018420408070000000000000034060020E2
:10183F000000000020420408070000000000000024
:10184F002C060020000000002842040807000000BA
:10185F00000000002406002000000000C03C040827
:10186F000100000000000000000000000000000068
:10187F00000000000E00000000000000000000004B
:10188F0000000000304204080F00000000000000BC
:10189F0099AE0208000000006C060020C66D002003
:1018AF001700000030FE0308C56D00200A3201004A
:1018BF00C46D002001FA0100C06D002000C80100B6
:1018CF00BE6D0020E803D0070100000046465F46CA
:1018DF004F5254494E49463400000000686D0020B5
:1018EF0000030100676D0020000301003842040867
:1018FF000F000000BDAD020899AD02080000000006
:10190F0048070020444204080F00000061AD0208A0
:10191F0021AD020800000000C0070020504204085B
:10192F000F000000F9AD0208E1AD02080000000051
:10193F00740800205C4204080F000000AFAE0208DC
:10194F00000000008DB302086C0B002064420408F5
:10195F000F0000007D3002080000000000000000B2
:10196F00BC0B00206C4204080F00000065B5020894
:10197F0009B1020805B10208980C0020744204084E
:10198F000F000000D5AE02080000000000000000AC
:10199F004C0D00207C4204080F00000079AF0208B4
:1019AF0049AF020800000000D80D0020844204084F
:1019BF000F000000F5AF02083DB002080000000064
:1019CF00780E0020D06E0020010301009042040821
:1019DF000F00000015AF0208E9AE0208000000007A
:1019EF00680F0020984204080F000000A9AF0208FA
:1019FF0005B4020800000000F40F0020A442040800
:101A0F000F00000069B0020851B402080000000086
:101A1F0094100020CA6E002001030100AC4204089C
:101A2F0000000000000000000000000000000000A7
:101A3F00B84204080800000000000000C011002098
:101A4F0000000000C0420408070000000000000072
:101A5F00B811002000000000D04204080700000069
:101A6F0000000000B011002000000000DC4204085C
:101A7F000700000000000000A81100200000000077
:101A8F00E84204080D000000000000009C11002037
:101A9F0000000000F442040803000000D98B030883
:101AAF008411002000000000C03C04080100000069
:101ABF000000000000000000000000000000000017
:101ACF000E000000000000000000000000000000F9
:101ADF00FC420408000000000000000000000000AD
:101AEF00000000000C4304080A0000000000000082
:101AFF003409040800000000144304080A00000021
:101B0F00000000007C090408000000001C430408CA
:101B1F000A000000000000000C6F00200000000011
:101B2F00244304080A00000000000000CC1100202C
:101B3F0000000000C03C040801000000000000008D
:101B4F000000000000000000000000000E00000078
:101B5F000000000000000000000000002C430408FB
:101B6F000000000000000000000000000000000066
:101B7F003843040803000000D98B03081C1200200F
:101B8F00000000004842040803000000D98B03083E
:101B9F0004120020000000003C4204080300000073
:101BAF00D98B0308EC110020000000004443040807
:101BBF000500000000000000666D0020000000001E
:101BCF004C4304080700000000000000E41100204F
:101BDF000000000058430408070000000000000048
:101BEF00DC11002000000000C03C040801000000D0
:101BFF0000000000000000000000000000000000D6
:101C0F000E000000000000000000000000000000B7
:101C1F006443040800000000000000000000000002
:101C2F00000000007843040803000000D98B03086C
:101C3F006412002000000000844304080300000029
:101C4F00D98B030844010020000000008C430408D6
:101C5F0003000000D98B03084C1200200000000085
:101C6F009443040803000000D98B030834120020AA
:101C7F0000000000C03C040801000000000000004C
:101C8F000000000000000000000000000E00000037
:101C9F00000000000000000000000000A043040846
:101CAF000000000000000000000000000000000025
:101CBF00AC430408070000009DB402081413002071
:101CCF00000000008C3F040803000000D98B0308BC
:101CDF00FC12002000000000B843040803000000BD
:101CEF00D98B0308E412002000000000C043040851
:101CFF0003000000D98B0308CC1200200000000065
:101D0F00C84304080700000081B40208C412002071
:101D1F00000000007C45040803000000D98B030875
:101D2F00AC12002000000000D443040803000000A0
:101D3F00D98B03089412002000000000E043040830
:101D4F0003000000D98B03087C1200200000000064
:101D5F00C03C04080100000000000000000000006B
:101D6F0000000000000000000E0000000000000056
:101D7F000000000000000000EC4304080F0000000A
:101D8F0055AE020811AE0208000000001C1300201F
:101D9F00F44304080F000000D9B00208000000004F
:101DAF0000000000D0130020004404080F000000C2
:101DBF0005AD0208E9AC0208000000005C14002029
:101DCF00084404080F00000000000000000000009D
:101DDF000000000010150020184404080F00000038
:101DEF00B1B00208B9B40208000000009C15002031
:101DFF002044040800000000000000000000000064
:101E0F00000000002C44040803000000D98B0308D5
:101E1F00D8160020000000000C4404080300000046
:101E2F00D98B0308C01600200000000004440408EA
:101E3F0003000000D98B0308A81600200000000043
:101E4F003444040803000000D98B030890160020C7
:101E5F00000000004044040803000000D98B030871
:101E6F00781600200000000048440408020000001B
:101E7F00D5B502080000000000000000504404081F
:101E8F0002000000D5B502080100000000000000AC
:101E9F005C44040802000000D5B5020802000000EF
:101EAF0000000000000000000E0000000000000015
:101EBF000000000000000000626D002088130C1766
:101ECF0001000000646D002088130C170000000053
:101EDF00684404080000000000000000000000003B
:101EEF000000000078440408080000000000000013
:101EFF00C4170020040000008444040808000000F8
:101F0F0000000000B817002000000000FC3F04088C
:101F1F0004000000A1B10208000000000000000052
:101F2F00C03C040801000000000000000000000099
:101F3F0000000000000000000E0000000000000084
:101F4F000000000000000000606D002088130C17D7
:101F5F00010000005E6D002088130C1700000000C8
:101F6F00C04404080F00000079AC02080000000014
:101F7F0000000000D0170020266F00200100000095
:101F8F0090FE03085D6D0020010000009CFE030819
:101F9F003C72002002000000A4FE030826AD0020C2
:101FAF00000000000000000024AD00200000000031
:101FBF000000000022AD0020000000000000000023
:101FCF0020AD002000000000000000001EAD00202A
:101FDF0000000000000000001CAD00200000000009
:101FEF0000000000FC1B00200000000000000000AB
:101FFF005C6D002002000000B0FE0308C844040816
:10200F0000000000000000000000000000000000C1
:10201F007844040808000000000000005418002055
:10202F0004000000844404080800000000000000C1
:10203F004818002000000000FC3F040804000000C6
:10204F0059AC02080000000000000000C03C04086A
:10205F000100000000000000000000000000000070
:10206F00000000000E000000000000000000000053
:10207F0000000000D8440408000000000000000029
:10208F000000000000000000E84404080D000000FC
:10209F0045B202089018002004000000F444040820
:1020AF000D0000009DAC0208841800200400000001
:1020BF00004504080D00000005B202087818002042
:1020CF00000000000C4504080300000081B1020865
:1020DF0060180020080000001845040803000000E5
:1020EF00D98B0308B81B002000000000C03C040877
:1020FF0001000000000000000000000000000000D0
:10210F00000000000E0000000000000000000000B2
:10211F0000000000B83C04080000000000000000B0
:10212F0000000000000000008E3C040804000000C6
:10213F00A5B202080000000000000000C03C040827
:10214F00010000000000000000000000000000007F
:10215F00000000000E000000000000000000000062
:10216F0000000000684504080000000000000000A7
:10217F000000000000000000500E04080D000000D9
:10218F0000000000F018002004000000784504084B
:10219F000800000000000000E41800200400000008
:1021AF00844504080800000000000000D818002033
:1021BF00040000008C450408080000000000000027
:1021CF00CC1800200400000094450408080000000B
:1021DF0000000000C0180020040000009C45040807
:1021EF000800000000000000B418002004000000E8
:1021FF00A44504080800000000000000A8180020F3
:10220F0004000000AC4504080800000000000000B6
:10221F009C18002004000000C03C040801000000CE
:10222F00000000000000000000000000000000009F
:10223F000E00000000000000000000000000000081
:10224F00B44504080F00000069AC0208000000004C
:10225F0000000000FC180020BC4504080F0000001F
:10226F0000000000000000000000000074190020B2
:10227F00C44504080F00000000000000000000002B
:10228F0000000000141A0020256F00200400000039
:10229F00BCFE030858580020E0150C170000000082
:1022AF005B58002008000000ACFB03085A580020C0
:1022BF0005000000D0FE0308CC4504080F00000005
:1022CF00000000000000000000000000641A002061
:1022DF0000FFFF0000000000AA5503009FAA55054C
:1022EF00010000AA550701000001AA550B010000CB
:1022FF00AA5509020000000001000000C0120100F1
:10230F00C157030879570308C95603080000000096
:10231F00B95303083D550308BD550308A5540308D9
:10232F000000000000000000AD53030891530308A4
:10233F008D530308895303087D530308795303080A
:10234F008553030881530308A153030895530308CA
:10235F007D54030891540308695403085554030826
:10236F00415403080100000060350408000000001C
:10237F00000000004D9E0108A0860100040000002F
:10238F00000000000000000000000000000000003E
:10239F000000000000000000000000008C3F040857
:1023AF00C034040800000000D11201087D000000B5
:1023BF000600000000000000000000000000000008
:1023CF0000000000000000000000000000000000FE
:1023DF00FC460408000000000000000021780308FC
:1023EF00E8030000030000000000000000000000F0
:1023FF0000000000000000000000000000000000CE
:10240F000000000004470408000000000000000066
:10241F004DB8010810270000030000000000000065
:10242F00000000000000000000000000000000009D
:10243F000000000000000000F03D04080000000054
:10244F0069FA0108D57A0108204E00000500000046
:10245F00000000000000000000000000000000006D
:10246F000000000000000000000000002C0D040818
:10247F000000000000000000DD72030810270000BC
:10248F00010000000000000000000000000000003C
:10249F00000000000000000000000000000000002D
:1024AF0010470408000000000000000071610108DF
:1024BF00E80300000500000000000000000000001D
:1024CF0000000000000000000000000000000000FD
:1024DF00000000001C47040800000000000000007E
:1024EF0071A00108204E0000030000000000000052
:1024FF0000000000000000000000000000000000CD
:10250F0000000000000000002C470408000000003D
:10251F0000000000799E0108204E0000030000001B
:10252F00000000000000000000000000000000009C
:10253F000000000000000000000000003C470408FD
:10254F0000000000000000006D700308400D030044
:10255F000300000000000000000000000000000069
:10256F00000000000000000000000000000000005C
:10257F0014360408000000000000000029160308AC
:10258F001027000001000000000000000000000004
:10259F00000000000000000000000000000000002C
:1025AF0000000000340D04080000000000000000CF
:1025BF002956020810270000030000000000000049
:1025CF0000000000000000000000000000000000FC
:1025DF000000000000000000400D04080000000093
:1025EF000000000049CB0008A00F00000100000010
:1025FF0000000000000000000000000000000000CC
:10260F000000000000000000000000004C4704081C
:10261F000000000000000000BD7D02081027000030
:10262F00010000000000000000000000000000009A
:10263F00000000000000000000000000000000008B
:10264F00044404080000000000000000551A0308AD
:10265F001A4100000100000000000000000000000F
:10266F00000000000000000000000000000000005B
:10267F0000000000BC0D0408000000000000000076
:10268F0049DB0208102700000100000000000000D5
:10269F00000000000000000000000000000000002B
:1026AF000000000000000000303C040800000000A3
:1026BF00000000002DB702081A41000001000000C1
:1026CF0000000000000000000000000000000000FB
:1026DF000000000000000000000000005847040840
:1026EF00000000000000000021050308400D03005A
:1026FF0000000000000000000000000000000000CB
:10270F0000000000000000000000000000000000BA
:10271F00604704080000000000000000DD0403080B
:10272F00400D03000000000000000000000000004A
:10273F00000000000000000000000000000000008A
:10274F0000000000684704080000000000000000BF
:10275F0079A20108A086010003000000000000001C
:10276F00000000000000000000000000000000005A
:10277F000000000000000000000000000102030440
:10278F0001020304060708090060024010600240BE
:10279F0000000000000B00000000200000000000FF
:1027AF0000000000006002402860024000000000AE
:1027BF00060C0000000020000000000000000000D8
:1027CF00006002404060024000000000100D000059
:1027DF000000200000000000000000000060024028
:1027EF005860024000000000160E0000000020009C
:1027FF000000000000000000006002407060024016
:10280F0000000000200F000000002000000000006A
:10281F0000000000006002408860024000000000DD
:10282F002610000000002000000000000000000043
:10283F0000600240A0600240000000003011000064
:10284F0000002000000000000000000000600240B7
:10285F00B860024000000000362F0000000020008A
:10286F0000000000000000000064024010640240FD
:10287F0000000000003800000000400000000000D1
:10288F0000000000006402402864024000000000C5
:10289F0006390000000040000000000000000000AA
:1028AF00006402404064024000000000103A000043
:1028BF000000400000000000000000000064024023
:1028CF005864024000000000163B0000000040006A
:1028DF00000000000000000000640240706402402D
:1028EF0000000000203C000000004000000000003D
:1028FF0000000000006402408864024000000000F5
:10290F00264400000000400000000000000000000E
:10291F0000640240A0640240000000003045000047
:10292F0000004000000000000000000000640240B2
:10293F00B86402400000000036460000000040006E
:10294F00000000000000000004030904120100024F
:10295F0002020040830440570002010203010000FD
:10296F0009024300020100C0320904000001020203
:10297F0001000524001001052401000104240202B6
:10298F000524060001070582030800FF0904010062
:10299F00020A00000007050102400000070581023E
:1029AF0040000000FF000000A9580308E955030884
:1029BF007D2F0308FD530308555803080D540308D2
:1029CF0029540308ED530308DD53030800000000EA
:1029DF0000000000000000010000000000000000E7
:1029EF00000000000800010043000000000000008C
:1029FF0000000000000000000000000000000000C8
:102A0F000000000000000000430000000000000074
:102A1F0000000000000000000000000000000000A7
:102A2F000000000000000000430000000000000054
:102A3F000000000000000000000000000000000087
:102A4F000000000000000000430000000000000034
:102A5F000000000000000000000000000000000067
:102A6F000000000000000000430000000000000014
:102A7F000000000000000000000000000000000047
:102A8F0000000000000000004300000000000000F4
:102A9F000000000000000000000000000000000027
:102AAF0000000000000000004300000000000000D4
:102ABF000000000000000000000000000000000007
:102ACF0000000000000000008DB00308CDAE030829
:102ADF00000000007C490408893C0408A71604087C
:102AEF00A7160408A7160408A7160408A7160408B3
:102AFF00A7160408A7160408A7160408A7160408A3
:102B0F00FFFFFFFFFFFFFFFFFFFFFFFFFFFF0000C4
:102B1F00010041534349490000000000000000003C
:102B2F000000000000000000000000000000000096
:102B3F00000041534349490000000000000000001D
:102B4F000000000000000000000000000000000076
:102B5F0000000000582400200000000000000000CA
:102B6F000000000000000000000000000000000056
:102B7F000000000000000000000000000000000046
:102B8F000000000000000000000000000000000036
:102B9F000000000000000000000000000000000026
:102BAF000000000000000000000000000000000016
:0C2BBF0000000000000000000100000009
:10800000152303701623C370172383713A238370DB
:108010003B2343713C230372704730B4846814B12E
:108020002368A5885D83436840F2E93001E00028B9
:1080300032D01D89013815F0020F80B2F7D089B215
:10804000998140F2E93101E0002947D018890139CE
:1080500010F0010F89B2F7D0998940F2E93100E0C0
:1080600059B31889013910F0020F89B2F8D092B2D1
:108070009A8140F2E93201E0002A3FD01989013AA1
:1080800011F0010F92B2F7D09B8914B12368A28836
:108090001A83012030BC704720498B4204D0A1F5DF
:1080A00074418B42D9D102201D4901EB0010418956
:1080B000013189B241814189CFE7184A934204D006
:1080C000A2F574429342E0D10221154B03EB01115A
:1080D0004B8901339BB24B814B89D6E70F488342D2
:1080E00003D010498B42B8D102210D4800EB011199
:1080F0004889013080B248814989AEE707498B42FF
:1081000003D0084A9342C0D10222054B03EB02126E
:10811000538901339BB253815389B6E70030014044
:10812000C07B0020003C0040F0B484894FF6FF760D
:108130004FF47A7443B3002938D00F78013101E04D
:10814000B4421AD00589013C15F00205A4B2F7D05B
:10815000BCB284814FF47A7402E0BCB2B4420CD059
:10816000058915F0010504F1FF37F6D08589ADB218
:108170000AB115700132013BDCE70D4B984207D084
:10818000A3F57443984202D00120F0BC7047022549
:10819000084B03EB05156B8901339BB26B81688932
:1081A00080B2003018BF0120F0BC7047FF27C9E73C
:1081B00000300140C07B002070B50546806810B1DA
:1081C00004688088608341F08001686840F2E93487
:1081D00000E0E4B10689013C16F0020FA4B2F8D029
:1081E00089B2818140F2E93100E009B304890139A3
:1081F00014F0010F89B2F8D081890021FFF794FFB4
:10820000AB6813B11A689B881383012070BD1049B5
:10821000884204D0A1F574418842EED102240D4970
:1082200001EB04146189013189B261816189E4E75C
:10823000074CA04203D008498842DED10221054CF8
:1082400004EB01114C890134A4B24C814989D4E773
:1082500000300140C07B0020003C0040002870B589
:108260001EDB0928044620DD012303EB83035B00AA
:10827000B0FBF3F2092AF8D87BB10E4EB4FBF3F051
:108280000928CCBF57223022A6FB03E5024403FB9A
:108290001044EB0801F8012BF0D100230B7070BDE6
:1082A0002D230B7040420131DBE7303001F8010B28
:1082B000F3E700BFCDCCCCCC884230B44FF0010402
:1082C0002ED301FB04F4B0FBF4F58D42F9D284B156
:1082D000AAB901E0B0FBF4F5092DCCBF572230223A
:1082E0002A4404FB150003F8012BB4FBF1F4002C25
:1082F000F0D100221A7030BC7047B0FBF4F5092DA4
:10830000CCBF372230222A4404FB150003F8012B8E
:10831000B4FBF1F4002CF0D100221A7030BC70478D
:108320000546002AEBD1D7E703685A1C0260197092
:1083300070472DE9F047089C2578002B8046894638
:108340000CBF4FF0200A4FF0300A661C35B3002AEC
:1083500029DD334601E0024698B113F8011B501E97
:108360000029F8D1971E60B13D46013D5146404677
:10837000C8476B1C002BF8DC257827EAE770013032
:1083800055B1041B29464046C847301916F8015B11
:10839000002DF7D1BDE8F087BDE8F087002A04DCA6
:1083A0002846BDE8F0870020EBE7571EDCE783682E
:1083B0004268D0ED037A00EB83010133934281EDF3
:1083C000040A836004BF0023836000EB830393ED02
:1083D000047A036870EE277A9A42C0ED037A77EE4A
:1083E000C77AC0ED037A0CDA013307EE103AF8EEE3
:1083F000C76AB7EE007A87EEA60A036030EE070A76
:10840000704707EE102AB8EEC77A87EE870A7047E2
:1084100090ED057A90ED004AD0ED066AD0ED014A64
:10842000D0ED047A90ED035AD0ED025AA4EE007A12
:10843000B0EE406AB0EE470AB0EE667AA6EE247A55
:1084400067EEC07AA0EE457AE6EE257A80ED057AF1
:10845000C0ED067A7047D0ED057A90ED013AD0ED87
:10846000003AD0ED064A90ED024A90ED077A90ED81
:10847000035A90ED086AD0ED045AC0ED067AF0EE8A
:10848000406A27EE830AC0ED056AA3EEA60A80EDD6
:10849000087AA4EE240AA5EE470AA5EEC60A80EDE6
:1084A000070A7047D0ED007A90ED017A30EE670A46
:1084B000E7EE007AB0EE670AC0ED007A70477047C9
:1084C0000A44914214D030B40139551E41F22102C0
:1084D00011F8014F082380EA042004044CBF82EA0B
:1084E00040004000013B80B2F7D18D42F0D130BC5A
:1084F00070474FF40063838270474FF400638382B8
:1085000070474FF40063838270474FF48053838237
:108510007047BFF34F8F0549054BCA6802F4E0620C
:108520001343CB60BFF34F8F00BFFDE700ED00E0CA
:108530000400FA0570B4037B04681F2B08D9203BA4
:108540002021626801FA03F31A421CD170BC704703
:108550002021226801FA03F31A42F7D04269144934
:10856000582000FB021251685689CD6808682968B6
:1085700021F001012960828992B222EA06028281F9
:10858000A36070BC704742690949582000FB021281
:1085900051685689CD680868296821F00101296071
:1085A000828992B222EA06028281E36070BC70473F
:1085B0007C73002030B4094B1C786CB1084A00254C
:1085C00002EBC404116893884D6288890832034322
:1085D0009BB2A2428B81F5D130BC70473C76002023
:1085E0004076002010B4037B01681F2B09D9203B83
:1085F00020224C6802FA03F31C4214D15DF8044BAC
:10860000704720220C6802FA03F31C42F6D00C4A91
:1086100040680024147002685DF8044B22F00102E7
:1086200002608B607047064A40680024147002683C
:108630005DF8044B22F001020260CB60704700BF7E
:108640006F68002070B5044682B01430E56D0623D3
:108650006A464321A847B0B19DF804009DF8006028
:108660009DF801109DF802509DF803209DF80530FB
:1086700041EA062143EA002342EA0522A187E28774
:10868000A4F84030012002B070BD70B5044682B03D
:108690000830656A06236A463B21A847A8B19DF8C1
:1086A00004009DF800609DF801109DF802509DF8AF
:1086B00003209DF8053041EA062143EA002342EAFF
:1086C0000522E18222836383012002B070BD50F84D
:1086D000043C012280F84520103803B11847704748
:1086E000F8B50468C4F30D0405460E4604B32F68BC
:1086F0002BF0ECF8092840F08880454C236923F4DE
:1087000040732361236943F400732361236943F0B9
:10871000010323613E602BF0D9F82369092823F077
:108720000103236171D12B6804332B600020F8BD55
:10873000384B394A93422BD902F58042934226D9CD
:1087400002F5804293422AD902F58042934228D909
:1087500002F58032934226D902F50032934224D9A1
:1087600002F50032934222D902F50032934220D919
:1087700002F5003293421ED902F5802293421CD9A1
:10878000B3F1016F1BD3052007F0B4FDFBE708240C
:108790002BF09CF8092814D04FF0FF30F8BD1024BE
:1087A000F6E71824F4E72024F2E72824F0E7302441
:1087B000EEE73824ECE74024EAE74824E8E75824C9
:1087C000E6E7134F3B6923F440733B613B6943F495
:1087D00000733B613B6923F0F8033B613B6943F065
:1087E00002031C433C613B6943F480333B612BF043
:1087F0006DF83B6923F002033B613B69092823F0D4
:10880000F8033B613FF473AFC6E76FF00100F8BDBA
:10881000003C024000400008FF3F0008F8B5044655
:108820000D468E180027B54201D12069F8BDE368D6
:10883000591CE160234415F8012B1A720429F2D166
:10884000206918B9A1682046FFF74AFF2061E76058
:10885000E9E7024B186808F0A7BA00BFD0900020E3
:10886000F8B5057B466903681F2D29D9A5F12004B9
:108870005F682021A1400F422A4613D01022A24057
:10888000D960DA605A68E240D10703D5012202FAC2
:1088900004F4DC600446304608F012FA227B2368B8
:1088A0001F2A20D9A2F1200008215A6881401142D4
:1088B00000D0D9600422596882400A4221D1F8BD13
:1088C00020211C68A9400C422A460CD01022AA4044
:1088D00099609A601A68EA40D207DBD5012202FA51
:1088E00005F59D60D6E7082118689140014200D047
:1088F00099600421186801FA02F2024203D09A60DA
:10890000F8BDDA60F8BDF8BD70B582B004466946BE
:1089100014302BF0F3F9B0B19DF805009DF801601B
:108920009DF802109DF803509DF804209DF8063034
:1089300041EA062143EA002342EA0522A187E287B1
:10894000A4F84030012002B070BD38B590F859301D
:1089500003B938BD0446184607F09EFA054608F0EC
:10896000ADFC01460028F4D1D5B12023E871AB71EC
:10897000284608F093FB21460F4B41F8103F28464C
:108980002BF050F9AB88B3FA83F3C3F11F03012234
:1089900012FA03F3DDD009490A6813430B6038BDAE
:1089A000294608F07BFB2146034B41F8103F28463F
:1089B000BDE838402BF036B9CF860008003C0140B6
:1089C00038B5044600F11405FFF7BFFF236E80227F
:1089D0006B2128469847642007F082FF236E072208
:1089E000682128469847642007F07AFF236E00220A
:1089F0006B2128469847642007F072FF236E0122FE
:108A00006B21284698470F2007F06AFF94F85320FF
:108A1000236E032A8CBF1A2218221B21284698474E
:108A20000F2007F05DFF236E18221C21284698476F
:108A30000F2007F055FF236E94F852201A21284684
:108A400098470F2007F04CFF236E94F8542019210B
:108A500028469847642007F043FF236E10223721F1
:108A6000284698470F2007F03BFF2846236E012237
:108A7000382198470F20BDE8384007F031BF2DE975
:108A8000F0410B4E346873691C400FD0DFF824802E
:108A90000127B4FA84F3C3F11F0307FA03F558F86A
:108AA000230003689847AC437561F2D1BDE8F081BB
:108AB000003C0140608500202DE9F0410B4E3468F8
:108AC00073691C400FD0DFF828800127B4FA84F3C3
:108AD000C3F11F0307FA03F558F82300036898470A
:108AE000AC437561F2D1BDE8F08100BF003C0140AC
:108AF000608500202DE9F0410B4E346873691C40FD
:108B00000FD0DFF828800127B4FA84F3C3F11F03E4
:108B100007FA03F558F8230003689847AC437561DA
:108B2000F2D1BDE8F08100BF003C0140608500202B
:108B30002DE9F0410B4E346873691C400FD0DFF80B
:108B400028800127B4FA84F3C3F11F0307FA03F561
:108B500058F8230003689847AC437561F2D1BDE82B
:108B6000F08100BF003C0140608500202DE9F0410C
:108B70000B4E346873691C400FD0DFF82880012742
:108B8000B4FA84F3C3F11F0307FA03F558F823007E
:108B900003689847AC437561F2D1BDE8F08100BF2E
:108BA000003C0140608500202DE9F0410B4E346807
:108BB00073691C400FD0DFF828800127B4FA84F3D2
:108BC000C3F11F0307FA03F558F823000368984719
:108BD000AC437561F2D1BDE8F08100BF003C0140BB
:108BE000608500202DE9F0410B4E346873691C400C
:108BF0000FD0DFF828800127B4FA84F3C3F11F03F4
:108C000007FA03F558F8230003689847AC437561E9
:108C1000F2D1BDE8F08100BF003C0140608500203A
:108C2000084A094808B5536C43F480435364002153
:108C3000402234F072FC054B4FF0FF321A60C3F84B
:108C4000032008BD0038024060850020A085002078
:108C500003685B6A18472DE9F041044618460D4643
:108C60001646984631F006FA2768E6722844A07244
:108C700029467D69434632462046AC46BDE8F04170
:108C80006047036810B504461B6898472368204670
:108C90009B689847A37B0133A37310BD10B503688D
:108CA00004469B689847FF2301226373227310BD1B
:108CB00008B507F0F1F840B12C2282710022C27190
:108CC0002021BDE8084008F0E9B908BD40F2E933C9
:108CD00000E0A3B10289013B12F0020F9BB2F8D071
:108CE00089B2818140F2E93300E043B10289013B5E
:108CF00012F0010F9BB2F8D08089C0B27047094AC8
:108D0000904205D0084B984201D0FF2070470223C3
:108D1000064A02EB03135A89013292B25A815889EA
:108D2000C0B2704700300140003C0040C07B0020D2
:108D300038B5054600BF084C2368986808F066FA05
:108D4000236829465868FFF7C1FF2368986808F030
:108D500063FA00BF38BD00BF3C890020144B984225
:108D600024D003F58063984220D0028822F040028C
:108D70001204120C0280028822F038031B041B0C20
:108D800059B141F48071002991FAA1F2B2FA82F14D
:108D900008BF4FF0FF310139C9000B439BB203807C
:108DA00003889BB243F04003038070474908DCE727
:108DB0000038004038B5044600F11405FFF7C5FD42
:108DC000A0694FF48071FFF7C9FF236E80226B21E9
:108DD00028469847642007F083FD236E032268210C
:108DE00028469847642007F07BFD236E01226B2103
:108DF000284698470F2007F073FD94F85320236E00
:108E0000032A8CBF1A2218221B21284698470F20BC
:108E100007F066FD236E18221C21284698470F2074
:108E200007F05EFD236E94F852201A2128469847D9
:108E30000F2007F055FD236E94F854201921284681
:108E40009847642007F04CFD236E102237212846F6
:108E500098470F2007F044FD2846236E3821012251
:108E60009847A0690821BDE8384077E710B5802110
:108E700004468069FFF772FF012007F0D7FC204607
:108E8000FFF79EFD10226A2104F11400FFF7C5F8D8
:108E9000642007F025FDA0690421FFF75FFF012092
:108EA000BDE8104007F0C2BCF8B5464E0446FFF7D7
:108EB0004CFD3778DFB104F114054FF48071A069DF
:108EC000FFF74CFF94F852201A212846FFF7A5F827
:108ED000012007F0ABFC0421A069FFF73FFF20460B
:108EE000FFF7B0FB94F93E30013362D0F8BD04F1D6
:108EF00014054FF48071A069FFF730FF80226B21C9
:108F00002846FFF78AF8962007F0EAFC032268213A
:108F10002846FFF782F8962007F0E2FC03226B2137
:108F20002846FFF77AF80F2007F080FC10226A210C
:108F30002846FFF772F80F2007F078FC3A466C21BC
:108F40002846FFF76AF80F2007F070FC94F85420C9
:108F500019212846FFF761F80F2007F067FC182257
:108F60001B212846FFF759F80F2007F05FFC10225D
:108F70001C212846FFF751F80F2007F057FC10225C
:108F800037212846FFF749F80F2007F04FFC012250
:108F900038212846FFF741F80F2007F047FC04214D
:108FA000A069FFF7DBFE012007F040FC01233370CE
:108FB00083E794F93C30013398D10620BDE8F840AE
:108FC00007F098B9BC240020F8B5654C0601A71934
:108FD0000546387A2AF004FE3B7A03F01F015B094C
:108FE0000122032B02FA01F26DD0042B66D0022B72
:108FF0005CD0A3190135187906F04EFFEDB2074693
:1090000010B11223C5718371A319587906F044FF7A
:1090100010B11323C5718371A319987906F03CFF31
:1090200010B11423C5718371A5190A21EA79384654
:1090300006F09AFD687906F02FFFEA790A2106F01A
:1090400093FDA87906F028FFEA790A2106F08CFD45
:10905000A359444A934247D0434A934250D0434A8B
:10906000934259D0424A934262D0424A93426BD0D3
:10907000414A93422CD03444227BE2B9012002229F
:10908000198801F4415141F445710A4302431A80A1
:109090009A8B22F400621204120C07219A8319821F
:1090A0001A8892B242F040021A80F8BD334B596AD6
:1090B0000A435A629DE700200246E1E72F4B1969F7
:1090C0000A431A6195E72D4B196A0A431A6290E721
:1090D00002F564424FF40010536A43F400135362E4
:1090E0002AF0EEFAA359C6E702F584324FF4805015
:1090F000536A43F4805353622AF0E2FAA359BAE761
:1091000002F500324FF48040136A43F48043136247
:109110002AF0DEFAA359AEE702F5FE324FF4004022
:10912000136A43F4004313622AF0D2FAA359A2E768
:1091300002F582324FF40050536A43F400535362F5
:109140002AF0BEFAA35996E702F568424FF4801060
:10915000536A43F4801353622AF0B2FAA3598AE7A0
:10916000C07B00200030014000380040003C00403F
:1091700000340140005001400054014000380240DA
:10918000427A02B9704710B504460368406804F19A
:109190000A0198470023637210BD437A5A1C0344A6
:1091A000D2B242729972037A934200D802B97047E0
:1091B00010B504460368406804F10A01984700238B
:1091C000637210BD302827D0312827D0322827D00D
:1091D000332827D0342827D0352827D0202827D057
:1091E000212827D0102827D0112827D0122827D0AF
:1091F000132827D0142827D0152827D0162805D0C3
:10920000172808BF0F2202D0002070470E22104BF3
:1092100003EB4203587870470022F8E70122F6E793
:109220000222F4E70322F2E70422F0E70522EEE748
:109230000622ECE70722EAE70822E8E70922E6E748
:109240000A22E4E70B22E2E70C22E0E70D22DEE748
:1092500084D6030870B5448806460D46C4F30B0453
:1092600022460021284634F058F93369094A9342CE
:1092700009D3094A934206D2224628461946BDE838
:10928000704031F035BE23B121462846BDE870401C
:10929000184770BD100600080F070008064B074965
:1092A0008B4202D30023184670471A88C2F30B0280
:1092B0009042F8D01433F3E7880100081006000844
:1092C000024A136823EA000010607047286F0020EC
:1092D000F8B5174D2B78A32B28D16B78BE2B25D151
:1092E000022229464FF6FF70FFF7EAF8114FAC1C37
:1092F00022884AB1A618BE4218D2052A16D921469C
:10930000FFF7DEF83446F3E721460222FFF7D8F8EC
:109310000222A118FFF7D4F80634074B641B1C8007
:1093200041F60F53C31A58425841F8BD0020F8BD0A
:109330000040000800800008244A00202DE9F04F7A
:10934000DFF84C914D4F8BB00326A7EB090718228D
:10935000002104A834F0E1F8494BCDF810900597AE
:109360001A69002A04DA474A5A6002F188325A60C0
:1093700001228DF82420F322DA60434B434C1B88F2
:10938000ADF800300222694604A8FFF747FA02222E
:1093900069464FF6FF70FFF793F8DFF8F8A08046B4
:1093A0004FF0000B544539D30AAC002524F8245D56
:1093B0000222214604A8FFF731FA02222146404644
:1093C000FFF77EF840BAC043ADF80800022202A9B8
:1093D00004A8FFF723FA079878B106ABC0F104029E
:1093E0002946184434F099F8089818B9069904A841
:1093F000FFF776F90023089007939DF82430089A28
:1094000023B11F490B6943F000430B61013E2DD08E
:10941000002A9CD1FFF75CFF50B32CE065888DF8E3
:109420000DB0C5F30B05AB1DADF808302388C3F3B1
:109430000B02ADF80A201B0B062202A904A88DF826
:109440000C30FFF7EBF9062202A94046FFF738F887
:10945000616880462A4604A8FFF7E0F96168404643
:109460002A46FFF72DF8143480469BE7002AD1D016
:10947000052006F03FFF0BB0BDE8F08F008000082C
:10948000003C024023016745A4D603088801000878
:1094900000400008100600080378202B024600F167
:1094A0000100F9D0092BF7D02D2B2CD02B2B03BF8B
:1094B0005378B7EE000A0246B7EE000AA3F1300176
:1094C000C8B209289FED467A10D8F2EE046A07EE7A
:1094D000901AF8EEE77A12F8013FE7EE267AA3F148
:1094E0003001C8B20928B0EE677AF0D92E2B4CD0E3
:1094F00003F0DF03452B0BD0F7EE007A67EE276A07
:1095000020EE260A70475378BFEE000A0246D5E7E0
:1095100010B451782D2959D02B290ABF9178501CAD
:10952000901C0024A1F13003092B53D8002303EB36
:10953000830301EB430310F8011FA1F13002092A54
:10954000A3F13003F3D9B3F59A7F28BF4FF49A7390
:10955000072B42D9DFED236A1A46F7EE007A083A64
:10956000072A67EEA67AFAD803F007032BB1F2EECA
:10957000046A013B67EEA67AFBD124B3C7EE276AE3
:109580005DF8044B20EE260A70475378A3F13001B2
:10959000C8B2092802F10102AAD8F2EE046AF0EE7C
:1095A000665A07EE901AF8EEE77A12F8013F87EE56
:1095B000A66AA3F13001C8B2092866EEA56A37EEA3
:1095C000067AEED994E767EE276AD9E7901C91787E
:1095D0000124A7E7F7EE007ACFE7F7EE007AC5E7B8
:1095E0000000000020BCBE4CB5EEC00ADFED317AB1
:1095F000F1EE10FACCBF30EE270A30EE670ADFED4D
:109600002E7A20EE270A30B5FDEEC07A87B017EE2D
:10961000904A054684EAE470002303A9A0EBE470B5
:1096200001930093029326F005FE002CACBF20238B
:109630002D2303A88DF8003030F01CFD012803A96C
:1096400024D002282DD0032805BF30236846684661
:109650008DF8013033F087FF684630F00BFD03389A
:10966000C4B222466946284633F0DBFF00232B555F
:10967000284630F0FFFC2E22431C2A540DEB040137
:10968000E81833F08DFF284607B030BD3023684618
:109690008DF801308DF802308DF8033033F063FF20
:1096A000DAE7302368468DF801308DF8023033F068
:1096B0005AFFD1E76F12033A00007A442DE9F041D6
:1096C000064615460846B6FBF2F43CB905FB1464A1
:1096D000124B1B5D00F8013BBDE8F081B4FBF2F7D3
:1096E00067B90E4B05FB174705FB1464DA5D00F8FC
:1096F000012B1B5D00F8013BBDE8F081B7FBF2F8E0
:10970000B8F1000F02D04046FFF7D8FF05FB1878EC
:10971000024B13F8082000F8012BE3E70C090408BA
:1097200030B402681146531C036011F8024B01600B
:10973000D31C517803609378151D05601B0443EA20
:109740000123D078234343EA006030BC70470368AC
:10975000591C1A46016012F8021B0260587841EA4F
:109760000020704703685A1C02601878704738B5AB
:1097700004460068154631F0BBFB22682A4422608B
:1097800038BD036810B40A0E5C1C04601A700368CC
:109790000A0C5C1C04601A7003680A0A5C1C0460F2
:1097A0001A7003685A1C026019705DF8044B704708
:1097B000036810B40A0A5C1C04601A7003685A1C1F
:1097C000026019705DF8044B704703685A1C026010
:1097D00010B4197003680A0A5C1C04601A700368EC
:1097E0000A0C5C1C04601A700368090E5A1C0260A3
:1097F00019705DF8044B704703685A1C02601970B9
:109800000368090A5A1C0260197070472DE9F04775
:10981000002488B080460F461E46A14605AD531C65
:109820000393117839B3252933D1931CCDF81090C7
:109830000393507830284ED04FF0000AA0F1300347
:10984000DBB2092B42D96C2819D0642800F0938030
:1098500024D825281CD063D9582876D063281BD15A
:1098600031784046B847039A531C03931178043665
:1098700001340029D7D1204608B0BDE8F087039B0A
:109880005A1C03921B78642B7CD02AD8252B54D1E8
:10989000252140460134B847039AC0E7732833D0E6
:1098A00044D975284FD106F1040E30682B460022AA
:1098B0000A217646FEF700FD049A00955346394684
:1098C0004046FEF736FD039A0444A8E704AA03A91C
:1098D0002DF0CEF8B7E7D31C039390784FF0010A30
:1098E000ACE7732B10D05BD9752B3AD0782B96D17F
:1098F000A3F15802B2FA82F2306852092B461021C5
:109900000436FEF7D9FCD7E73368049A009339464A
:1099100000234046FEF70DFD04360444039A7EE71B
:109920000028B9D1204608B0BDE8F0876E28B3D131
:10993000039A336804361C6071E72AD9582BD7D0B4
:10994000632B8DD06BE77828A6D1A0F15802B2FA2C
:1099500082F2306852092B461021FEF7ADFC043626
:10996000AAE706F1040E30682B4600220A2176464B
:10997000FEF7A2FCA0E7331D306829461E46FEF71D
:109980006DFC99E7331D306829461E46FEF766FCDC
:1099900092E7002B7FF443AF204608B0BDE8F08784
:1099A0006E2BC6D03BE70EB400B584B005AB01907A
:1099B00053F8042B0649039301A8FFF727FF019BE7
:1099C00000221A7004B05DF804EB03B0704700BFCA
:1099D000298300080FB430B583B006AB0A490B48A1
:1099E00053F8042B096800680193FFF70FFF084C38
:1099F0000546206807F0C4F90028FAD0284603B0CD
:109A0000BDE8304004B070478C3D0020903D002000
:109A1000D0900020DFED2B7AB4EEE70AF1EE10FAD9
:109A20004ADDDFED296A9FED297A01E0B0EE670A91
:109A3000B4EEC70AF1EE10FA70EE667AF6DC9FED2E
:109A4000247AF4EEC77AF1EE10FA38D5DFED1E6A0B
:109A50009FED207A01E0F0EE407AF4EEC77AF1EE65
:109A600010FA37EEA60AF6D4DFED1B7AB4EEE70A59
:109A7000F1EE10FA14DDDFED137A37EEC00A60EE76
:109A8000006A9FED166A9FED167ADFED167AA6EE54
:109A9000867A20EE266AE6EE877AA6EE270A7047D7
:109AA000DFED117AB4EEE70AF1EE10FA44BFDFED14
:109AB000087A37EEC00AE2E7F0EE407ABFE7B0EE90
:109AC000670AD1E7DB0F4940DB0FC940E4CB164101
:109AD000DB0F49C0E4CB16C1DB0FC93F92E741B9A8
:109AE0009730083C15A82ABEDB0FC9BF09B909E0A9
:109AF000194690FBF1F301FB13030846002BF7D145
:109B0000084670470146FBE7F0EEC07AB0EEE07A17
:109B1000B4EEE77AF1EE10FAB4BFB0EE676AB0EED9
:109B2000476AB5EE406AF1EE10FA46D0B4EEE77A35
:109B3000F1EE10FA8CBFF0EE675AF0EE475AC5EE20
:109B4000866A9FED1F3A9FED1F6A9FED1F4A9FEDAA
:109B50001F5ADFED1F3ADFED1F4ADFED1F5AA6EE59
:109B6000C36AE6EEA34AA6EE864AB7EE006AA6EE00
:109B7000845AA6EEA46AE6EE855AC5EE866AB4EE6D
:109B8000E77AF1EE10FA48BFDFED147AF5EEC00A7D
:109B900048BF77EEE66AF1EE10FA48BFDFED107AC3
:109BA000B5EEC00A48BF77EEE66AF1EE10FA48BF9C
:109BB000F1EE666AB0EE660A7047DFED076ADEE72F
:109BC00039094E3DE3B59E3E88FA163E45FE7F3F7D
:109BD00099FB243F69A2163EA7DFA834DB0FC93FDB
:109BE000DB0F4940DFED317A30EE277AFDEEC76AB0
:109BF00016EE903A2033402B02D99FED2D0A704784
:109C0000B4EEE70AF1EE10FA4DDD9FED2A6ADFEDC2
:109C10002A6A01E0B0EE677AB4EEE67AF1EE10FA65
:109C200077EE467AF6DC9FED257AF4EEC77AF1EE10
:109C300010FA35D5DFED1F6A9FED217A01E0F0EED5
:109C4000407AF4EEC77AF1EE10FA37EEA60AF6D4AF
:109C5000DFED167AB4EEE70AF1EE10FA1BDCDFED69
:109C6000197AB4EEE70AF1EE10FA44BFDFED137A89
:109C700037EEC00A60EE006A9FED136A9FED137A1B
:109C8000DFED137AA6EE867A20EE266AE6EE877A74
:109C9000A6EE270A7047DFED0F7A37EEC00AE9E734
:109CA000B0EE670AD4E7F0EE477ABCE7DB0FC93FB6
:109CB00000000000DB0FC940E4CB1641DB0F49C0B8
:109CC000E4CB16C1DB0FC9BF92E741B99730083C1E
:109CD00015A82ABEDB0F4940FDEEC07A17EE903A78
:109CE0002033402B51D8DFED2D7AB4EEE70AF1EEA8
:109CF00010FA50DDDFED2A6A9FED2A7A01E0B0EE1E
:109D0000670AB4EEC70AF1EE10FA70EE667AF6DC76
:109D10009FED257AF4EEC77AF1EE10FA38D5DFED33
:109D2000206A9FED227A01E0F0EE407AF4EEC77AE5
:109D3000F1EE10FA37EEA60AF6D4DFED1D7AB4EE96
:109D4000E70AF1EE10FA1BDCDFED1A7AB4EEE70A4F
:109D5000F1EE10FA44BFDFED147A37EEC00A60EE80
:109D6000006A9FED156A9FED157ADFED157AA6EE74
:109D7000867A20EE266AE6EE877AA6EE270A7047F4
:109D8000DFED067A37EEC00AE9E79FED0E0A70476D
:109D9000B0EE670AD1E7F0EE407AB9E7DB0F494051
:109DA000DB0FC940E4CB1641DB0F49C0E4CB16C141
:109DB000DB0FC93FDB0FC9BF92E741B99730083CC1
:109DC00015A82ABE0000000010B507EE901A2DED70
:109DD000028BB8EE678ADFED217A28EE008A04460E
:109DE00028EE278AB0EE480A31F0D6FAF0EE408A23
:109DF000B0EE480A31F032FAF7EE007A9FED187AA9
:109E0000F0EE675AE8EE875A0023A361B0EE676A66
:109E1000C7EEA56A63612362E361A8EEC76ABDEC81
:109E2000028B77EEC07AB6EE007AF8EE005A27EE93
:109E3000877A20EE250A27EE267A26EE266A67EE36
:109E4000A67A20EE260A84ED046AC4ED017A84ED38
:109E5000007A84ED027A84ED030A10BD27D4D2364D
:109E6000F304353F10B44C09012250F8243001F0BE
:109E70001F0102FA01F10B4340F824305DF8044B56
:109E800070474B0901F01F0150F82320012303FA0A
:109E900001F1114214BF184600207047084B1B788F
:109EA000022B03D0074B00229A717047064A1368B1
:109EB00043F480231360034B00229A71704700BF64
:109EC000C424002058720020286F002010B53E20C6
:109ED00005F0E2FF0B4C606018B111220023827183
:109EE000C371202107F0DAF80A2006F09FFC6068B1
:109EF00007F0E4F9044B002814BF012202221A7073
:109F000010BD00BFBC240020C4240020074A084B19
:109F100010781B78074A834296BFC31AC3F18003A7
:109F20000020126818441044704700BF50AF002052
:109F3000CDAE0020CC620020064A074B10781B787B
:109F400083428ABFC3F18003C01AC018C0F17F00EA
:109F5000704700BF50AF0020CDAE002030B5144C8C
:109F6000237883B01BB90120237003B030BD0522D4
:109F700000238DF800208DF8013000BF0D4D2B68B7
:109F8000986807F043F92B6801AA6946586829F0D8
:109F90005BFD2B68986807F03FF900BF9DF805301E
:109FA00003F0010383F00100237003B030BD00BF54
:109FB0004E8900203C89002070B5064C0646256875
:109FC00003E023685B1BB34203D8FFF7C7FF0028F9
:109FD000F7D070BD248600202DE9F04F89B0B2F192
:109FE000000A02900491039340F3B0800B460022D4
:109FF00001EB8A0153F8040B8B420244FAD1039B14
:10A000000592002B00F09A80059B002B6AD0544BE0
:10A01000059A1B68DFF85C9100920099DAB251183A
:10A02000B1F5807F8CBFC2F58072009A01924D4AD3
:10A0300092689A426DD9190C1A0A4FF00204062050
:10A040008DF81F308DF81E208DF81D108DF81C40E6
:10A05000FFF7B2FF0620FEF76BFE434A01231370A1
:10A0600000BFD9F80030986807F0D0F8D9F8003070
:10A0700007A95868002229F09FFC0024049D029E35
:10A08000019FA34629684FEA840800220B46013449
:10A0900071B1B9422AD2D9F8000031684068FEF7A0
:10A0A00043F82A68336813443360BF1AC5F800B018
:10A0B000A24505F1040506F10406E3D1D9F8003004
:10A0C000986807F0A9F800BF254B019900981B6814
:10A0D000421A0092224A0B441360039A32B3009A48
:10A0E000002A9AD1059809B0BDE8F08F029CD9F8F2
:10A0F000003054F80810586800223B46FEF714F868
:10A1000054F808202B683A44DF1B44F808202F60DD
:10A11000D4E70598009C1549154A001B0590059841
:10A1200000230B70137009B0BDE8F08F059B009AF7
:10A130009B1A0593059809B0BDE8F08FFFF70EFF55
:10A1400000287FF461AF039B0593CBE7039C1CB908
:10A15000FFF704FF0594C5E700230593C2E700BF9E
:10A16000CC620020D42200204E89002050AF002075
:10A17000CDAE00203C89002070B5104D104E2B78DC
:10A1800031788B4284B016D00E4A03921A44029260
:10A190008CBF0C46CA1A04A98CBFC3F180020024EC
:10A1A000012341F8102D02A802220194FFF714FFA9
:10A1B000002333702B7004B070BD00BFCDAE002003
:10A1C00050AF0020D0AE002070B5194C194D237847
:10A1D0002978994284B027D0174A03921A440292F0
:10A1E00034BF0E46CA1A04A934BFC3F18002002648
:10A1F000002341F8102D02A802220196FFF7ECFE81
:10A2000023781844C0B203062B7848BF80F0800042
:10A210008342207002D0002004B070BD00230120D2
:10A220002B70237004B070BD012004B070BD00BF5E
:10A23000CDAE002050AF0020D0AE002008B545F2D2
:10A240000820FFF7B9FE0620FEF772FD064B01223B
:10A25000C7201A70FEF76CFD04480549054A002323
:10A2600003700B70136008BD4E89002050AF0020B2
:10A27000CDAE0020CC6200202DE9F04182B0034633
:10A28000060C050A032406208DF807308846174679
:10A290008DF805608DF806508DF80440FFF78CFEB0
:10A2A000C0B100BF0D4C2368986806F0AFFF23686B
:10A2B00001A95868002229F07FFB2368424600214B
:10A2C00058683B46FDF730FF2368986806F0A4FF06
:10A2D00000BF384602B0BDE8F08100BF3C890020D5
:10A2E000F0B5124B9D6885B00DB905B0F0BDED0A13
:10A2F00014D0002704AE7C196410E00210226946D5
:10A30000FFF7BAFF0F2809DD6B4653F8042B013223
:10A310000AD1B342F9D12546AF42ECDBFFF72CFF5F
:10A32000034BED021D60E0E7671CF5E7D422002037
:10A33000CC6200202DE9F84FDFF8B4A0DFF8B4803C
:10A34000DFF8B490274E012308208AF8003029F066
:10A350000BFBD8F8000006F059FF052029F0BCFBE4
:10A36000002029F0B9FB062029F0B6FB002029F0D7
:10A37000B3FB99F80040042044F0010429F0ACFB41
:10A38000204629F0A9FB33888BB1174D174F0024C5
:10A3900015F804B0072029F09FFB584629F09CFBD4
:10A3A0002A5D33883A550134A4B2A342F0D807207D
:10A3B00029F092FBFF2029F08FFB99F80040042040
:10A3C00029F08AFB204629F087FBD8F8000006F028
:10A3D00023FF042029F0C8FA00238AF80030BDE8E2
:10A3E000F88F00BF1801002068580020A85D0020E9
:10A3F000915D0020548F0020374B00202DE9F04163
:10A400004A4E082029F0B0FA306806F0FFFE484BAB
:10A410001B78012B7BD062D3022B0AD1DFF830816D
:10A42000082388F800300D254FF4C373414F3B805B
:10A4300010E0DFF81C813F4F98F8003003F0400334
:10A44000002B14BF4FF4F0734FF4C3733B8014BF61
:10A4500010250D25002404F11000C0B229F03CFBAA
:10A460000134012029F038FBA3B2AB42F3D398F8B2
:10A470000040314D002029F02FFB204629F02CFB15
:10A480002E4B1C78022029F027FB204629F024FBC4
:10A490002B4B1C78032029F01FFB204629F01CFBC6
:10A4A000284B1C780420044329F016FB204629F091
:10A4B00013FB306806F0B0FE042029F055FA3A8804
:10A4C0002148002133F029F82B7833B11F4B1B783A
:10A4D00033B300232B70BDE8F081BDE8F081A020EC
:10A4E00029F0FAFA002029F0F7FA00F00603022B0F
:10A4F000DFF85C8007D000F00500012803D1482375
:10A5000088F8003008E0082388F800308BE7DFF88F
:10A510004080482388F8003010254FF4F07385E719
:10A52000FFF708FF00232B70BDE8F081548F002057
:10A530006C8F00201801002000000020738F002085
:10A54000748F0020374B0020A85D0020915D002013
:10A55000200100200C4B984213D0A3F58063984251
:10A560000FD003F5804398420BD003F580639842E7
:10A5700007D003F58063984203D0044B1868400865
:10A580007047024B18687047000401407890002023
:10A59000F0B5774B774A87B01968914200AF00F069
:10A5A000DB800023744A3B607B60136843F4803394
:10A5B000136003E03B68B3F5A04F09D0136803F4C0
:10A5C00000337B603B6801333B607B68002BF1D03C
:10A5D000694B1B6813F4003318BF01237B607B6851
:10A5E000012B7BD0654D644B654AEA606549586F25
:10A5F000654A0860AA605E6B644C654A654826F04F
:10A6000080065E635E6F46F080765E67196B0C4372
:10A610001C63596B5963996B9963196C41F05B51D9
:10A6200041F47B1141F41F6141F00F011964596C31
:10A6300007F118040A4348F2FF715A6444F8101DE8
:10A64000002621460123FB733E737E73BE7328F000
:10A6500015FF21464FF6FF734F48BB6028F00EFFF1
:10A660004FF6FF7321464D48BB6028F007FF214697
:10A670004B4828F003FF21464A4828F0FFFE2146B8
:10A68000494828F0FBFE2146484828F0F7FE2146BD
:10A69000474828F0F3FE2146464828F0EFFE2046C2
:10A6A00029F0CCF8444B454C1B68BA6844484549EE
:10A6B000A4FB03439B09A0FB0202013B920CB3F1F4
:10A6C000807F0A6007D2404AF0200721536085F856
:10A6D0002300966011601C37BD46F0BD264B3B4CF5
:10A6E0001A6C3B4942F080521A6420688A684D68AF
:10A6F000C96840F4404020609868986098681206E5
:10A7000040F40040986042EA8512986842F4800262
:10A71000490842F00802013942EA014240F4A050DF
:10A7200098605A601A6842F080721A601A68920142
:10A73000FCD52849104A40F205700860996821F05C
:10A7400003019960996841F002019960936803F0F0
:10A750000C03082BFAD145E700221A6062B61E4BA3
:10A760001B6883F308881D4B1B689847FEE700BFF2
:10A77000FCFF0120EFBEADDE0038024000ED00E03E
:10A780000005FA054078002000000008FF916700EE
:10A79000335F07000000024000040240000802404E
:10A7A000000C024000100240001402400018024059
:10A7B000001C02400020024078900020D34D62101F
:10A7C00083DE1B432886002010E000E0007000407C
:10A7D00000000020003C02400000FF1F0400FF1F9B
:10A7E00008B5054B1B6803B19847044B044A1A602F
:10A7F00072B6FDF78EFE00BF34630020FCFF01201F
:10A80000EFBEADDE08B5034B1B6803B1984772B6C7
:10A81000FDF77FFE34630020084B10B507281B6846
:10A82000C8BF143818440C46007D05F035FB20B134
:10A830002146BDE8104006F0F5BC10BDCC850020D7
:10A8400038B50D4B07281B68CCBFA0F11404044693
:10A8500023440546187D05F01FFB58B1013427221B
:10A86000C4718271012106F019FC28460021BDE85F
:10A870003840D1E738BD00BFCC85002070B50F4C03
:10A880000F4DC0EBC00004EB8004286B26693043F9
:10A89000286382B09209667BA1600025012101A88E
:10A8A00063618DF804608DF805208DF806508DF8F1
:10A8B000071023F00BFB02B070BD00BF8820002002
:10A8C00000380240074BC0EBC00030B403EB8000FF
:10A8D000054C0569236B2B4323630176427630BC1C
:10A8E000704700BF88200020003802402DE9F04F5B
:10A8F0005B4C54F8204083B0002C00F0AC80E66D37
:10A90000002E00F0AA809046564A3569226099468A
:10A9100004F2622204F162036361A2614FF40073E6
:10A920007268A1600746E36023616265A246B5B123
:10A930004D4B00205A68954203F11C0376D001303C
:10A940001028F7D100207A1CD2B20C21FFF7BAFFF1
:10A95000636DB168326922630433A1632365F068D3
:10A96000E8B1414B00215A68904203F11C035BD0CF
:10A9700001311029F7D100257A1CD2B20B212846CB
:10A98000FFF7A0FF2346F27F38492846FFF776FFFE
:10A99000636DB168F26862630433E163E36494F861
:10A9A000610005F079FA054694F8600005F074FA44
:10A9B0008346307F00284BD119F0080F38D118F0AA
:10A9C000020F09D045B10B227B1CAA71EB712846FE
:10A9D000727F222105F0C8F818F0010F15D1A36B82
:10A9E0007BB996F82020B17F8DF8063001A8930935
:10A9F00001228DF805308DF804108DF8072023F022
:10AA000065FA504603B0BDE8F08FBBF1000FE6D009
:10AA100001370C238BF807708BF806305846727F8D
:10AA2000222105F0A1F8DAE7CDB2A5E7C0B28AE7A6
:10AA30000137FFB215B10B23EF71AB7119F0100F95
:10AA4000284614BF02211221727F05F08DF8C6E757
:10AA500029F0C6F8B0E7A246D3E7B246D1E700BF77
:10AA6000983D0020A8D603088820002061880008AF
:10AA70000348D0F8AC3113B100F5D27018477047D5
:10AA8000882000200348D0F8903113B100F5C4703D
:10AA900018477047882000200348D0F8743113B15C
:10AAA00000F5B67018477047882000200348D0F89A
:10AAB000583113B100F5A87018477047882000205E
:10AAC0000348D0F83C3113B100F59A70184770472D
:10AAD000882000200348D0F8203113B100F58C7095
:10AAE00018477047882000200348D0F804310BB184
:10AAF000FC301847704700BF882000200348D0F87A
:10AB0000E8300BB1E0301847704700BF88200020C4
:10AB10000348D0F8CC300BB1C4301847704700BFA1
:10AB2000882000200348D0F8B0300BB1A830184777
:10AB3000704700BF882000200348D0F894300BB144
:10AB40008C301847704700BF882000200248836F70
:10AB50000BB1703018477047882000200248C36D41
:10AB60000BB1543018477047882000200248036C0E
:10AB70000BB1383018477047882000200248436ADC
:10AB80000BB11C30184770478820002002488368AA
:10AB900003B11847704700BF882000201549164BA5
:10ABA00016484A6810B4CC681549B2FBF4F203FBAE
:10ABB00002F30360D1F88820124B134C42F4700268
:10ABC000C1F888201A68002042F001021A609860DB
:10ABD0001A6822F0847222F480321A605C601A686B
:10ABE0004FF0006422F480221A60D8608C605DF817
:10ABF000044B70470000002040420F007890002076
:10AC000000ED00E00038024010300024044B4FF407
:10AC1000F07002210A225860D9609A60FFF7BEBF27
:10AC2000000000202DE9F04F9DB0B0F908500D81D3
:10AC3000EDB2442D00AF0C46904600F0D08206469F
:10AC400043D9812D00F0088200F29A80542D00F043
:10AC5000CF8040F2ED816E2D00F08F82802D40F08C
:10AC60001A81C04B93F800A00AF1020A1AF0FF0AF9
:10AC700000F09A80BC4BDFF82C83BC4EDFF828B381
:10AC80009A4403F101090A2516E0322D00F0D8821A
:10AC9000A5F13C00C0B2132840F2D88200232268FC
:10ACA000511C216015702268D14502F1010121601B
:10ACB000137079D019F8015B0A2DE6D1BBF800308A
:10ACC000FF2BA8BFFF23DBB2E9E7052D00F075825B
:10ACD00021D8022D00F0848040F29781032D00F0EE
:10ACE0004282042D40F0D7802A46A1492046FEF733
:10ACF0003EFDA04B20461978FEF77EFD226802211A
:10AD0000531C0125236028462B467437117063813C
:10AD1000BD46BDE8F08F242D60D040F20481282D7F
:10AD200000F0E381382D40F0B6800A68924B01258F
:10AD3000511C216015702268052150192060117086
:10AD400022680A21501920601170226800215019D0
:10AD500020601170226819785019206011702268E3
:10AD6000597850192060117022689978531923601E
:10AD70002B461170284674376381BD46BDE8F08FBD
:10AD8000A02D19D040F21681B82D00F0EA81FE2DD9
:10AD900040F08180794D05F1080635F8021B204608
:10ADA000FEF72AFDB542F8D101252B462846743717
:10ADB0006381BD46BDE8F08F714B08461968FEF708
:10ADC00004FD704B20461968FEF7FFFC6E4B1968B6
:10ADD00020460125FEF7F9FC2B46E7E76B4BF6E72B
:10ADE00004226B4920460125FEF7C1FC2B46C1E732
:10ADF0000B68684ADFF8B481581C11212060197073
:10AE000023681278591C21601A70236898F85B2017
:10AE1000591C21601A70236898F85A20591C216027
:10AE20001A70B8F856102046FEF7E6FC00212046BE
:10AE3000FEF7E2FCB8F858102046FEF7DDFCA8F15A
:10AE4000020508F1480635F8021F2046FEF7D4FC3B
:10AE5000B542F8D12268504B0C21501C20605D187F
:10AE60001170226813F8011F501C9D422060117060
:10AE7000F7D123680222591C21601A70B8F85C10BF
:10AE80002046FEF7B9FC0125B8F85E102046FEF713
:10AE9000B3FC2B466EE7214628460BF0E3F9034648
:10AEA000002881D1742D00F0C980772D0DD1326832
:10AEB000716891421EBF531C33601178374A08BF36
:10AEC000194620462CF04AFF6EE7F52D01F0B883B5
:10AED000762D00F08C81472D00F07D823268392D6F
:10AEE000114600F0648300F20B82212D01F068838B
:10AEF000292D40F07983531C336013780A2B01F01D
:10AF00004B84502B40F07F853046FEF720FCDFF865
:10AF1000A080A8F800003046FEF719FC0125A8F82B
:10AF200002002B4626E7202DB5D10B681C4D591C7D
:10AF30006A7821601A7023682A78591C21601A7077
:10AF40002368AA78591C21601A7029892046FEF7C7
:10AF500053FC23686A79591C21601A702268A97908
:10AF6000CEE600BF4D710020D0D60308082B00208C
:10AF7000668F0020C4240020C16D00207071002065
:10AF8000107AFF1F147AFF1F187AFF1F286F002006
:10AF900034090408708F002069790020617003086B
:10AFA0009888002067666666302B00202079002094
:10AFB000F02A0020822D7FF46EAF0B68BB4ABC4D97
:10AFC0001178BC4A581C2060197011892046FEF780
:10AFD00013FCB94B22681B88FF2B02F10101A8BFAB
:10AFE000FF2321601370A96881F3100189B2204604
:10AFF000FEF702FC296801F30F0189B22046FEF733
:10B00000FBFBAE4B226819787AE6012D7FF443AF43
:10B010000B680022591C21601A7023685A1C226098
:10B020001D7022682421531C23602B461170A1E659
:10B03000522D7FF430AF2268002161E632687168DA
:10B0400091421EBF531C336011789D4A08BF1946B8
:10B0500020462CF083FEA7E69A4B1E78033616F0A6
:10B06000FF063FF4A1AE984BDFF88C821E4403F13B
:10B07000010A4FF00A0920E0B9F1500F00F0DE801C
:10B08000B9F1320F00F0F780A9F13C00C0B21328EB
:10B0900040F2F4800025294623685A1C226020468D
:10B0A00083F80090FEF7A8FB29462046FEF7A4FB94
:10B0B00056453FF479AE1AF8019BB9F10A0FDBD17E
:10B0C000824B9D68196805EB85054FF6FF736D008F
:10B0D0009D42A8BF1D469942A8BF194625EAE575BD
:10B0E00021EAE171ADB289B2D6E70B68DFF80C92C4
:10B0F000774E591C022221601A7023684FF006080F
:10B100005A1C226083F8008023680A22591C21609F
:10B110001A70236801255A1922601D70B9F80010B1
:10B120002046FEF769FBB9F802102046FEF764FBE3
:10B1300023685A19226083F8008023685022591925
:10B1400021601A7023680022591921601A70318811
:10B150002046FEF751FB71882046FEF74DFB2B463B
:10B1600008E65C4B33E60B685A1C0A601D700B68DE
:10B170000222591C21601A705DE74F4B0A681B8838
:10B180004B4DFF2BA8BFFF23511C21601370A968F2
:10B1900081F3100189B22046FEF72EFB4E4B20466C
:10B1A0001988FEF729FB296801F30F0189B22046AF
:10B1B0000125FEF721FB2B46DCE50B224749204603
:10B1C000FEF7D5FA082246492046FEF7D0FA0125B7
:10B1D000072244492046FEF7CAFA2B46CAE5002A50
:10B1E0003FF4E2AD404B136001252B46C2E53268C7
:10B1F000511C31601278002A01F0D582102A07BF55
:10B200003A4B93E822001D4629462368581C2060CB
:10B210001A702046FEF7D9FA29462046FEF7D5FADD
:10B22000334B20465968FEF7D0FA20460021FEF73E
:10B23000E3FA00212046FEF7DFFAFCE62D4B40E75B
:10B240003388FF2BA8BFFF23DBB228E523F0C2FB26
:10B2500000283FF423AD03780A2B25D8B0F902303B
:10B2600088FB0312DB17C3EBA2039BB2FF2BA8BF23
:10B27000FF23DBB213E598E8220024E723F0AAFBC2
:10B2800000283FF407AF03780A2B3FF603AFB0F96D
:10B290000430B0F9061003EB830383F3500521EA71
:10B2A000E171ADB289B2F7E60023E2E766720020F1
:10B2B000788600209888002050720020C8790020ED
:10B2C000097C03084D710020E0D60308BC2A002049
:10B2D000F02A00208C3E00208E7900203C090408D2
:10B2E000480904085409040845620108A42A0020FA
:10B2F000C4240020F42A0020002B002040620020FB
:10B30000552D00F02D81572D40F06E81531C336078
:10B3100012F8378B07F12F010133336013F8010C5A
:10B3200001F8010F9342F7D1DFF8B0A29AF800506C
:10B33000002DFDD1DFF8A8B2012608208AF80060B0
:10B3400028F012FBDBF8000005F060FFA04B284658
:10B350001E7028F0C1FB284628F0BEFB092028F00B
:10B36000BBFB404628F0B8FB07F13008454607F123
:10B370006609A5EB0806F6B20A2028F0ADFB3046B8
:10B3800028F0AAFB15F8016B0B2028F0A5FB30462E
:10B3900028F0A2FB002005F01BFD4D45E9D1082057
:10B3A00028F09AFBA02028F097FBA02028F094FB1F
:10B3B000002028F091FB10F02000F6D10646DBF8C3
:10B3C000000005F029FF0125042028F0CDFA8AF8B5
:10B3D00000602B46CEE4726835687B623046551BB0
:10B3E000FEF79EF9052D38627B6A01F2C88180263E
:10B3F000B346012594E80600521A103A9642C8BF97
:10B400001FFA82FB734A396A92683A61521A93456D
:10B41000396A7B622046FA6088BF1FFA82FBFEF71A
:10B42000D4F97B6A002B01F08981002D41F0658100
:10B430002368C7F800D05D71C0B00533C7F804D0E9
:10B44000FB61BBF1000F01F07D823B6A3A699342D8
:10B4500081F0D3823E6A7D62AA46A846BC60802500
:10B46000FB68A3EB08085B4BB8F5807F9B6828BF9F
:10B470004FF4807806EB08029A4288BFA3EB0608D7
:10B48000FEF77AFE7C68424621463046FEF7F4FE1F
:10B49000F969B86104EB000C0B787B6164452ED22E
:10B4A000DFF840910CF1FF3C04F1FF3E1EF8013F34
:10B4B00009EB830219F823405688ECB100234FF4BE
:10B4C000004204F1FF3816424FEA520202D00878D7
:10B4D000284308706D0806D10AF1010A4D701FFA61
:10B4E0008AFA01318025D34503D8E64532D3984501
:10B4F00030DC01339C42E6D1E645D7D1F9617B6A65
:10B50000BA6913449BB2D3457B6206D97B6A3A6A17
:10B510009846D6183B699E42A2D3BC68802D1CBFBA
:10B520000AF101031FFA83FA0AF1020189B22046E7
:10B53000FEF762F92368796A01255A1922602046CC
:10B540001D70FEF759F92368534423602B46D7F842
:10B5500000D00FE4FB69BC681A463B7D1370DDE741
:10B56000531C336092F80080B8F1FF0F01F0B881EE
:10B57000B8F1FE0F01F060813046FEF7E8F896E87A
:10B580000C009B1A002B07DD531C336013781BB98A
:10B59000B8F10B0F41F28881B8F1240F00F2C98590
:10B5A0000D4B012523F818002B46FFF7E3BB531C76
:10B5B000336013780A2B01F0FB803046FEF7D2F897
:10B5C0003046FEF7CFF83046FEF7CCF8FFF7ECBB7D
:10B5D000995D0020D422002020790020915D002078
:10B5E000548F0020F0D6030870680B3D831AEF2DAE
:10B5F00000F29F850FF2040E5EF825F05DC300088F
:10B6000033C1000833C1000833C1000833C100084A
:10B6100033C1000833C1000833C1000833C100083A
:10B6200033C1000833C1000833C1000833C100082A
:10B6300033C1000833C1000833C1000833C100081A
:10B6400033C1000833C1000833C1000833C100080A
:10B6500033C1000833C1000833C10008D3C2000859
:10B6600033C10008B1C2000833C1000887C2000816
:10B6700033C1000833C1000833C100085FC20008AD
:10B6800033C10008DFC1000833C10008ADC10008A4
:10B6900033C1000839C2000833C10008D3C0000814
:10B6A00033C100083DC1000833C10008E5C00008EF
:10B6B00033C1000833C1000833C1000833C100089A
:10B6C000A9AD000833C1000891C1000833C10008CA
:10B6D00033C10008D7BE000833C10008BDB9000857
:10B6E00033C1000833C1000833C1000833C100086A
:10B6F0007FBF000833C1000833C1000833C1000810
:10B700003FBF000833C10008F1BE000833C1000884
:10B7100033C1000891C0000833C1000833C10008DC
:10B7200033C1000833C1000833C1000833C1000829
:10B7300033C10008BDBF000833C1000863BE000864
:10B7400033C10008F1BD000833C100083DBD000849
:10B7500033C1000815BD0008AFBC000833C10008A4
:10B7600033C1000833C1000833C1000833C10008E9
:10B7700033C1000833C1000833C1000833C10008D9
:10B7800033C1000833C1000833C1000833C10008C9
:10B7900033C1000833C1000833C1000833C10008B9
:10B7A00033C1000833C1000833C1000833C10008A9
:10B7B00033C1000833C1000833C1000833C1000899
:10B7C00033C1000833C1000833C1000833C1000889
:10B7D00033C1000833C1000833C1000833C1000879
:10B7E00033C1000833C1000833C1000833C1000869
:10B7F00033C1000833C1000833C1000833C1000859
:10B8000033C1000833C1000833C1000833C1000848
:10B8100033C1000833C1000833C1000833C1000838
:10B8200033C1000833C1000833C1000833C1000828
:10B8300033C1000833C1000833C1000833C1000818
:10B8400033C1000833C1000833C1000833C1000808
:10B8500033C1000833C1000833C1000833C10008F8
:10B8600033C1000833C1000833C1000833C10008E8
:10B8700033C1000833C1000833C1000833C10008D8
:10B8800033C1000833C1000833C1000833C10008C8
:10B8900033C1000833C1000833C1000833C10008B8
:10B8A00033C1000833C1000833C1000885BC00085B
:10B8B00033C10008D5BD000833C1000833C10008FA
:10B8C00033C1000833C1000833C1000833C1000888
:10B8D00033C1000833C1000833C1000833C1000878
:10B8E00033C1000833C1000833C1000833C1000868
:10B8F00027BC0008D5BB00089DBB000833C1000869
:10B90000FBBA0008E1BA0008C5BA000833C1000854
:10B91000ABBA00083FBA000817BA00080DBA000811
:10B9200061C5000833C1000831C5000833C10008F3
:10B9300033C1000807C50008D9C40008C5C4000801
:10B940009DC400087DC4000853C4000827C4000833
:10B9500033C1000833C1000833C1000833C10008F7
:10B9600033C1000833C1000833C1000833C10008E7
:10B9700033C1000833C1000833C1000833C10008D7
:10B9800033C1000833C1000833C1000807C40008F0
:10B9900033C1000833C10008ADC3000833C100083B
:10B9A00033C1000833C1000833C1000833C10008A7
:10B9B00033C1000833C1000893C30008531C33602F
:10B9C000C24B1278DFF844831A700023C8F80030A5
:10B9D0003046FDF7A5FE3368D8F80020BC49BD4DC0
:10B9E00010435A1CC8F8000032601B780B723046B6
:10B9F000FDF7ADFE28603046FDF7A9FE68603046D1
:10BA0000FDF7A5FEA8603046FDF7A1FE3046FDF724
:10BA10009EFEFFF7C9B9531C33601078060601F18A
:10BA20006380AD4B1B78DD073FF5BEA9032828BF17
:10BA3000002001250BF092FC2B46FFF79BB9531C0D
:10BA40003360304692F800A0FDF76AFE814630462A
:10BA5000FDF766FE05463046FDF762FE804630463D
:10BA6000FDF775FE3046FDF772FE3046FDF77AFEB3
:10BA7000BAF1000F01F02180BAF1100F7FF494A900
:10BA8000964BC3F800905D60B8F1000F02D0944B64
:10BA9000C3F804809349944B0222081F01251A70B1
:10BAA00017F0F0FE2B46FFF765B98B4B1B78D807D4
:10BAB0003FF57AA901250BF005FF0BF01DFD2B4684
:10BAC000FFF758B9844B1B78DA073FF56DA9874A11
:10BAD0001378012543F0040313702B46FFF74AB98E
:10BAE0007D4B1B78D9073FF55FA9814B4FF4C87296
:10BAF00001251A802B46FFF73DB9092B40F3198326
:10BB0000DFF80C821346511CD8F80050316013F84E
:10BB1000021B297033605378AB70D31C3360937869
:10BB2000642B02F10401A8BF64236B713160D378E8
:10BB3000642B02F10501A8BF6423AB713160137956
:10BB4000EB71931D33605379642B02F10701A8BF99
:10BB500064232B7231609379EB7002F10803336038
:10BB6000D3792B713046FDF7F2FD72683368688136
:10BB7000D11A00290CDD591CD8F800003160521A86
:10BB8000002A1978417203DD9A1C32605B78437099
:10BB900001252DF00DFF2B46FFF7ECB8554B18682B
:10BBA000D31C014621329D1E356013F8035C0D70D5
:10BBB0005D1E356013F8025C4D70336013F8015C54
:10BBC0008D7003339A4201F10301ECD111F0B4F806
:10BBD000FFF7EAB8531C336013784449002B00F098
:10BBE0008E870B7843F00203901C0B70424D30603F
:10BBF00053782B753046FDF793FD28603046FDF7EE
:10BC00008FFD68603046FDF7A2FD28813046FDF7C4
:10BC10009EFD3A4AE8811378012543F00203137030
:10BC20002B46FFF7A7B8C3F34705122D00F2818218
:10BC3000C5B107F1700307F12E0A03EB4508D146A1
:10BC4000A8F142083046FDF782FD29F8020FC845E9
:10BC5000F8D12B4B3AF8022F23F8022FD145F9D116
:10BC6000112D09D8274A6B00023B134400212232D0
:10BC700023F8021F9A42FBD1234A01231D46137069
:10BC8000FFF778B81346511C316013F8025B33603C
:10BC9000D31C507833609178002D00F0FD86012D83
:10BCA0007FF482A80EF0EEFD2B46FFF763B80A4B37
:10BCB0001B7813F0010140F03C82531C3360107874
:10BCC00001250EF021FD2B46FFF754B8D06200206D
:10BCD00014780020C03D0020DC710020A42A002040
:10BCE000C4240020A82A00208E5A0020B0880020FA
:10BCF0000AB10020B8680020B48800208C5A0020C7
:10BD0000AE470020B0470020D4470020286F002015
:10BD1000ECB000201346511C31609C4913F8020B13
:10BD2000C87033609A4953784B71D31C3360994B78
:10BD30009278DA7001252B46FFF71CB83046FDF7E4
:10BD400006FD3046FDF703FD3046FDF700FD3046A9
:10BD5000FDF708FD3368904D1946581C2A6830607D
:10BD600011F8020B82F82C003160597882F83610F5
:10BD7000D91C31609B7882F837303046FDF7F2FCF1
:10BD80003046FDF7EFFC3046FDF7ECFC3046D5F8C9
:10BD90000080FDF7DCFCA8F83A003046D5F80080BA
:10BDA000FDF7D5FC96E80C00991A0129A8F838008F
:10BDB0000ADD511C2B683160127883F82E20304642
:10BDC000FDF7D0FC96E80C009B1A032B00F39C8631
:10BDD0002868FBE6DFF8DC8100233046C8F8003035
:10BDE000FDF79EFC0125C8F800002B46FEF7C2BFF8
:10BDF000531C3360684DDFF8C081137888F8053034
:10BE00003046D5F80090FDF7A2FCA9F82000304696
:10BE1000D5F80090FDF79BFC96E80C00991A0729CD
:10BE2000A9F81E0000F31C86991A032900F30A865C
:10BE30009B1A002B05DD511C2B683160127883F8AA
:10BE400026200BF0B1FA23F053FA544B1B68002B59
:10BE500000F028862868012510F014FC2B46FEF718
:10BE600089BF1346511C3160DFF84C8113F8021B67
:10BE700088F8021033604A4953780B70D31C336042
:10BE8000484D93782B71131D3360D378092BA8BFCD
:10BE900009233046AB70FDF75AFC96E80C00991A5E
:10BEA0000129288005DD3046FDF751FC96E80C009D
:10BEB000E881934240F0BC850BF076FA33687268F3
:10BEC0009A423EF471AF5A1C32601B78EB70012528
:10BED0002B46FEF74FBF344B03F10801501C306076
:10BEE000127803F8012F99423EF45EAF3268F5E70D
:10BEF000531C336092F80080B8F1110F00F21981E1
:10BF0000931C3360294D537805F818303046FDF7FF
:10BF10001EFC40F6CA039842A8BF184640F2EE2322
:10BF2000984205EB4801B8BF18460125A0F2EE2261
:10BF30002B46192092FBF0F24A70FEF71BBF134606
:10BF4000511C1B4D316013F8021B2971336053786B
:10BF50006B713046FDF7FBFB336828805A1C32605A
:10BF60001B78AB713046FDF7F2FB336868805A1CD2
:10BF700032601B78EB7101252B46FEF7FBBE0125D5
:10BF8000FEF75CF92B46FEF7F5BE00BF50620020BD
:10BF9000987B002060620020B8680020C862002002
:10BFA000446200205473002013780020F4490020DC
:10BFB000544500208C3E0020847600203046FDF75A
:10BFC000C6FB054617F06CFDFF283EF4EDAE3F2D95
:10BFD00000F2178507F17008002308F8403D4FEA8A
:10BFE000D509414607F12F0087F82F3009F10109E3
:10BFF00017F036FD97F82F305FFA89F905F007053D
:10C000004B4505F1010503D197F83030AB4203D021
:10C010002946484617F030FD33687268D21A012A63
:10C020007EF7C2AE5A1C07F17000326000221D7804
:10C0300000F8412D17F008FD97F82F30AB420AD0D9
:10C04000B94B1B683BB19A79AA4204D31B681B69A0
:10C050000BB12846984733685A1C3260404600228C
:10C060001D7887F8302017F0E3FC97F83030AB42AA
:10C070003EF49AAEAC4B1B68002B3EF495AE1B68A9
:10C080005B69002B3EF490AE28469847FEF78CBEC5
:10C09000A64B1B78012B3EF687AE1146531C33602E
:10C0A000DFF8AC8211F8023B88F802303160D31C13
:10C0B00092F801E03360C31A012B917840F3918428
:10C0C0003046FDF744FB0125A8F800002B46FEF79B
:10C0D00051BE531C3360964B12785A7501252B467E
:10C0E000FEF748BE0722B3FBF2F2C2EBC2055B1BB0
:10C0F0001FD1D2B202F1FF395FFA89F9002A3EF46A
:10C1000053AEDFF830A209F101091D464B1C336024
:10C1100091F90020874B4FF0000893F902109142EB
:10C1200003F1080300F09B8308F10108B8F1050F43
:10C13000F3D14FF0FF352B46FEF71CBE531C336086
:10C1400013780E2BF5D8911C31605578032DF0D85B
:10C150007948062101FB03F1431802F1030E5D71DA
:10C16000C6F800E095784554111D3160D1785970BA
:10C17000511D316011799970911D31605179D970DB
:10C18000D11D316092791A7101252B46FEF7F2BD5F
:10C190001346511C3160694913F8020B88703360F3
:10C1A00053784B7001252B46FEF7E4BD644D05F135
:10C1B00040083046FDF7CBFA3368A5F88000591CDB
:10C1C0001A46316012F8021B85F8821032605B78E3
:10C1D00085F883300435A845EBD1FEF7E5BD531C47
:10C1E000534D336013782B723046FDF7B0FAA883B5
:10C1F0003046FDF7ACFA28833046FDF7A8FA3368DD
:10C2000068835A1C32601B78EB7473689A1A032A8D
:10C2100000F3C8833268991A052900F3B3839B1A87
:10C22000002B7EF7C1AD531C3360137885F82130A5
:10C2300001252B46FEF79EBD511C316015781F2D40
:10C240003FF677AF052B7FF474AF3046FDF768FA01
:10C250003B4B43F8250019F081FEFEF7A5BD531CAA
:10C260003360384915780D70C31A002B7EF79CADEA
:10C27000931C33605378003318BF012301254B70A2
:10C280002B46FEF777BD3046FDF761FADFF8C48034
:10C29000C8F800003046FDF75AFAC8F804003046E6
:10C2A000FDF755FA0125C8F808002B46FEF762BDD8
:10C2B000DFF8A4800023C8F800303046FDF730FADC
:10C2C000D8F8003001250343C8F800302B46FEF7AC
:10C2D00051BD531C33601578132D3FF62AAF931CC4
:10C2E000336050787A622BF073FD00283FF421AF61
:10C2F0007A6A154B017803F82510D11C316003EBE5
:10C30000850391785970111D3160D0789870501D57
:10C3100030600E491279DA70086801252DF0D6FADE
:10C320002B46FEF727BD00BFB4680020136F002026
:10C33000147800207C8F0020983E00206C62002042
:10C340006C670020D0620020D4620020B868002012
:10C3500088790020C03D0020286F0020A84A102BBB
:10C360004FF0000128BF1023116051609160D1602F
:10C370001174002B3EF418AD3168013A0B440131C1
:10C38000316011F8010C02F8010F9942F7D1FEF764
:10C390000BBD9C4B1B78DB073FF5CBAE01250AF0AC
:10C3A000F9FF0BF0A9F82B46FEF7E4BC531C3360F1
:10C3B00013780F2B3FF6BDAE911C3160C3EBC30366
:10C3C00091495078C854D01C30600B449178597012
:10C3D000111D3160D1789970511D31601179D9707A
:10C3E000911D316051791971D11D31609179597167
:10C3F00002F108013160D2799A7101251EF07CFBAF
:10C400002B46FEF7B7BC3046FDF7A1F9DFF80482F2
:10C41000A8F80E003046FDF79AF90125A8F80C009F
:10C420002B46FEF7A7BC1146531C3360774B11F81F
:10C43000020B1870316051785970D11C31609178BD
:10C440009970111D3160D278DA7001252B46FEF704
:10C4500091BC3046FDF77BF9DFF8D481A8F81000D5
:10C460003046FDF774F9A8F812003046FDF76FF971
:10C470000125A8F814002B46FEF77CBC1346511C7E
:10C48000316013F8020B3360D31C5178336092781B
:10C490001DF0B0F800287EF487AC4AE61346511C24
:10C4A00031605B4913F8020B0870336059495378C7
:10C4B0008B70D31C3360584B92789A7001252B46B1
:10C4C000FEF758BC554B564918684E2201252EF0F0
:10C4D0000FFD2B46FEF74EBC1146531C3360514BEB
:10C4E00011F8020B1870316051785970D11C31600D
:10C4F00092789A703046FDF72AF94B4B0125D88087
:10C500002B46FEF737BC3046FDF721F9DFF81881DE
:10C51000A8F800003046FDF71AF9A8F802003046E6
:10C52000FDF715F90125A8F804002B46FEF722BCFB
:10C53000DFF8009199F80030002B3EF435ACDFF8BD
:10C54000F88000253046FDF702F910F04BFD99F810
:10C550000030A8EC010A01359D42F3DBFEF724BC54
:10C560000D2B7FF4E6AD531C33601578072D3FF695
:10C57000E0ADDFF8C89030464FF00C08FDF7E7F863
:10C5800008FB05F809EB0805A8803046FDF7DFF841
:10C59000E8803046FDF7DBF8336828811A46591CDD
:10C5A000316012F8021BA97232605B78EB72304680
:10C5B000FDF7B6F8012549F808002B46FEF7DABB6F
:10C5C0001346511C3160194D13F8021B697033601A
:10C5D00053782B70D31C33609378AB703046FDF7E3
:10C5E000B6F833682881591C1A46316012F8021BCC
:10C5F000697132605B78AB7101252B46FEF7BABBDF
:10C60000A0680020DC710020146C0020A05B0020DA
:10C61000847600205062002060620020B86800200C
:10C6200080E00308486200203C45002098880020F4
:10C63000547300204D71002094440020206B002092
:10C64000336872689A4240F0C480C14BFF225A702E
:10C650004FF0000ABF4D20F0EBFD51462022BE48AE
:10C6600085F800A030F059FF87F830A097F83030F7
:10C67000072B00F25781DFF80493B74E524697F824
:10C68000303003EB430309EBC3035B7CE3B197F862
:10C69000303003EB430309EBC30320215B699BB1FB
:10C6A00097F8303003EB430309EBC303586946F8AE
:10C6B000220004F0F3FC2B7856F8230004F0ACFDC4
:10C6C0002A780132D2B22A7097F830300133DBB2C7
:10C6D00087F8303097F83030072BD0D92368591CB1
:10C6E00021601A70B8F1000F3EF45EAB9B4BC8F8A6
:10C6F000003001252B46FEF73DBB994B3A6A9B68FB
:10C70000D4F800905A449A4200F2D980FDF734FDE3
:10C710005A464946386AFDF7AFFD23680344236053
:10C7200086427EF741AB002100E0236801305A1CAD
:10C73000864222601970F8D1FEF736BB002DDCD19D
:10C7400059462046FDF758F823685A1C22601D7090
:10C75000834B26689D683B6A0BEB0302954280F091
:10C76000E3803B6AED1AFDF707FD2A463146386A39
:10C77000FDF782FD236803442360FEF715BB3046B6
:10C78000FCF7E5FF326871687B6A9142834649D1C4
:10C7900006461D46FEF72EBE3046FCF7D8FFDFF8F2
:10C7A000E081FEF7B6BB6F4B93E82200FEF72DBD8C
:10C7B000931C33606C4B51781970D11C31609178A7
:10C7C0005970111D3160D2789A7001252B46FEF701
:10C7D000D1BA5A1C194632605D4811F8022B4270DA
:10C7E00031605B788370042A03D9FF2A7EF423AC7E
:10C7F0002EE75E490978994205D8022A7EF41BACDF
:10C80000FF2B7EF418AC236801255A1922601D7095
:10C81000B8F1000F3EF4C8AA554BC8F800302B46BB
:10C82000FEF7A8BA511C316012781D46131C06464B
:10C8300018BF0123FEF7DEBD931C33605578022D2F
:10C840003FF677AC3046FCF782FF4A4B03EB4503DB
:10C850004FF0FF35A3F85C002B46FEF78BBA0AEBCE
:10C86000C80B30468BF80220FCF771FF33682AF8BA
:10C8700038001A46591C316012F8021B8BF803105D
:10C8800032605A788BF80420DA1C32609A788BF880
:10C890000620191D31600135DB788BF80530A9457C
:10C8A0007FF434ACFEF780BA324B0030984418BFA6
:10C8B0000120012588F84A002B46FEF75BBA3A6A48
:10C8C000A3EB0208FDF758FC42464946386AFDF7DB
:10C8D000D3FC236803442360002D3EF465AA1FE7C0
:10C8E000931C3360244B51781970D31C3360DFF8EC
:10C8F0008480937888F85B30131D3360D37888F890
:10C900005A303046FCF723FFA8F856003046FCF7B3
:10C910001EFF3046FCF71BFF0125A8F858002B46E8
:10C92000FEF728BA5246D9E6FDF726FC5A463146AC
:10C93000386AFDF7A1FC23680125034423602B46D8
:10C94000FEF718BADA46C7F824B0FEF7EDBD00BF0F
:10C95000C4240020FA690020C8690020E19C020874
:10C96000D4220020D05A0020C16D00204D7100203B
:10C970005162010820790020708F002094720020FD
:10C9800040620020531C33601378EB723046FCF792
:10C99000C7FE3368E8605A1C32601B782B7496E837
:10C9A0000C003CE43046FCF7D2FEA8843046FCF78D
:10C9B000CEFE96E80C00991A0329E8847FF72BAC89
:10C9C0001346511C316013F8021BA977336053786A
:10C9D00085F820303046FCF7BAFE96E80C006884F3
:10C9E00019E4504B1A88012512FB0EF22B4692FBDC
:10C9F000F1F2A8F80020FEF7BDB97D62AA46FEF765
:10CA000093BD07F13008404617F006F83B8EAB4265
:10CA10003FF402AB444B1B68002B3FF4FDAA1B689C
:10CA20009B69002B3FF4F8AA28469847FFF7F4BA11
:10CA3000531C33601378003318BF012388F8073084
:10CA4000FFF73ABA3046FCF782FEA8F80E003046EF
:10CA5000FCF77DFE96E80C00A8F81000FFF7E8B997
:10CA60003046FCF774FEA8F80A003046FCF76FFE6B
:10CA7000A8F80C003046D5F80090FCF768FEA9F83D
:10CA800022003046D5F80090FCF761FE96E80C00D5
:10CA9000A9F82400FFF7C8B901250FF0BBFF2B460A
:10CAA000FEF768B921482249224A234B0360012539
:10CAB0000B6013602B46FEF75DB9204B1020C3F8C6
:10CAC00000905D6024F09AFE1D4A137843F0010344
:10CAD0001370B8F1000F3EF467A91A4B0125C3F893
:10CAE00004802B46FEF746B900F07F00032828BFDC
:10CAF000002001250DF0E2FE2B46FEF73BB90B7836
:10CB000003F0FD03FFF770B83046D5F80080FCF75E
:10CB10001EFEA8F8320030462E68FCF718FEB086DC
:10CB2000FFF756B964AF0020B4680020B83F00207A
:10CB30000C4000200C440020BF840008D05A002084
:10CB4000B0880020C42400202DE9F04F2DED028B89
:10CB500093B0834625F01AFD914B1D7825B113B093
:10CB6000BDEC028BBDE8F08F8E4B1B685905F6D5E6
:10CB70008D4B8E4E1B6863B18D4A31681368CB1A9A
:10CB80007C2B06D98B48116003780133037028F0A1
:10CB90000FF9894B1B78002B72D0884C884AD4F847
:10CBA0001031ABEB0303934201F2548394F81891D4
:10CBB000B9F1000F35D1DFF83C82D8F8000004F05D
:10CBC000EFF8C0B201280FD902287E4F42F06680EC
:10CBD0003B78002B42F0B181D4F81C31ABEB03035E
:10CBE000B3F57A6F82F0EF82D4F82031002B47D072
:10CBF00094F81831C3B9744B1B689B7801211E3B14
:10CC000000228B4284F8181184F82C2142F296827B
:10CC1000D8F800000221043028F07CF894F8243180
:10CC200011E0D4F820315BB3D4F8283140F6B732A4
:10CC3000ABEB0303934223D994F82431002B01F08A
:10CC4000F986DFF8B081013BDBB284F82431002B98
:10CC500001F02684D4F8207194F82C2117F8011BD8
:10CC600094F82D31D8F80000C4F820710A4401333B
:10CC700084F82C2184F82D3104F096F8C4F828B1FA
:10CC8000524B37681B7853B1DFF86C81D8F800003D
:10CC900028B14F4B1B78013B012B41F211844D4BC6
:10CCA0001B7873B1DFF85481D8F800304BB133688A
:10CCB000424C02931A46D4F84431D31A632B01F242
:10CCC000B281DFF83C8198F80030022B01F08A86AF
:10CCD0003C4F97F87430032B01F0CC833E4B1B780C
:10CCE00073B13E4D2B685BB1344C03F053FDD4F867
:10CCF0005031029044F61F62C31A934200F2308111
:10CD0000374B1B78002B7DD1364B1B7843B12B4C16
:10CD1000D4F8A03203F5C333A0339B4581F03E82A3
:10CD2000314B1B78002B3FF41AAF244E2F4C304D63
:10CD300006F2C127206804F033F800283FF40FAF53
:10CD4000206804F025F82B7880465A1E33B12068FD
:10CD50002A7004F025F80028F2D100E703223946B2
:10CD6000781E30F0C0FB96F8C03296F8C12286F8E3
:10CD7000C38283F47F4383F0FF039B1A1FFA88F872
:10CD80009BB2B8EB132FD5D196F8C222DBB29A42F0
:10CD9000D0D1781E21F098FE2B7818442870C9E76E
:10CDA000905D0020A87600206C860020248600205C
:10CDB0008C88002088880020667A0020CC240020FF
:10CDC0003F0D0300200000203C880020687A0020EE
:10CDD000707A0020787A0020807A0020847A0020FF
:10CDE000F07A0020017B00208A7A0020907A0020CF
:10CDF000947A002038880020708600203088002037
:10CE00003E490020484C2278A2B1484B9B7A53B14E
:10CE100003F0C0FC464B1B68C31AA3F57A73B3F545
:10CE2000FA6F07D82278434B4349186803F084FF10
:10CE300000232370414CD4F8983203F5C333A03358
:10CE40009B45FFF461AF3E4DC4F898B22B78002BA0
:10CE500041F035873B4D2B78002B41F08D8694F8BF
:10CE60009C2239498D5CEA0701F1E787AF0701F1A0
:10CE7000A787680702F12B802A0748D5334B344F28
:10CE80000B9312AA1146A3F13D0241F8202D002078
:10CE9000A3F140020D4603F8400C03910223112137
:10CEA0005170937028463968FCF76BFC2846796806
:10CEB000FCF767FCFB89274903EBC3039B000533A1
:10CEC00081FB0321DB17C3EBA101284689B2FCF7E4
:10CED0006FFC3B8A03EB8303590089B22846FCF7B9
:10CEE00067FC1D4B039D1B789B0743BF398901F5E8
:10CEF0007A7189B24FF47A712846FCF759FC0A9B83
:10CF00003A7D591C0A9128461A7025F0CFFA134A27
:10CF100094F89C321178013393FBF1F201FB123348
:10CF200084F89C32F0E600BF587A00201478002084
:10CF3000AC480020F47A0020187A0020CC2400208D
:10CF4000F87A0020F97A0020FC7A0020187A002074
:10CF5000B488002067666666B0880020007B0020E9
:10CF600094F85631002B41F08A85DB4B1A6802F0A9
:10CF70000803002B4AF60B4048F603414BF60F43DB
:10CF800049F6074704BF03460F4612F0040F4FF05F
:10CF9000190118BF1F46900684F8561103D547F4AF
:10CFA000804747F02007CD4B5A79C7F30909002A7B
:10CFB00042F031819B79002B42F03D8298466420FB
:10CFC0004FF0FF3A4FF0000C0A970B97ADF834C0C2
:10CFD000CDF83AC0CDF83EC0CDF842C0CDF8309083
:10CFE000ADF83680ADF838A08DF846000AAF0FCF07
:10CFF000DFF800E384F805C0AEE80F0097E80F0003
:10D00000AEE807002EF8023B71464FF0010C1B0CF6
:10D01000FE271F20C82201F81E39A770A27184F8CC
:10D0200007C0E07094F86601207180F0F10383EA94
:10D030000313DAB2130983F0E70343EA022383EA16
:10D04000C2031BB283EA0312D2B2C3F3072383EAFB
:10D05000121343EA022383EAC2031BB283F0C8021D
:10D0600082EA0212D2B2C3F3072383EA121343EA1D
:10D07000022383EAC2031BB283EA0C0787EA07177D
:10D08000FFB2C3F3072282EA171242EA072200EB3B
:10D090000C0382EAC7070EEB0C0084F86631278088
:10D0A00011F8013B7B4083EA0313DBB21A0982EAE1
:10D0B000172242EA032282EAC3031BB29FB28142D3
:10D0C0002780EDD183F07C0383EA0313DBB24FEAC0
:10D0D000131E8EEA172E8EEA032E8EEAC30E0FFA67
:10D0E0008EFE1FFA8EF9DFF810C2A4F800905FFAE6
:10D0F0008EFE4FEA192984F8289084F827E00CF571
:10D10000C77804F1220ADCF80000DCF80410DCF82F
:10D110000820DCF80C3047460FC70CF1100CD44542
:10D12000B846F0D1DCF8000038606D4F9CF8043050
:10D1300088F8043007F1270884F8B5E184F8B6913F
:10D1400017F8011F286803F02FFEB845F8D194F8AE
:10D150005731002B41F08E846249326809780A20E9
:10D1600084F85701002901F021865F4F0129388892
:10D17000069042F257810229B7F802E002F065807A
:10D18000B8880590032902F05D81F888049004298D
:10D1900002F06E810529388902F065810629B7F809
:10D1A0000A9002F05C810729B7F80C8002F05481E4
:10D1B000FB89039394F866110A920B4683F03002C0
:10D1C00082EA0212D2B217094849079387F07A0718
:10D1D00047EA02270988237187EAC202444FC1EB5C
:10D1E000012187FB013A069B4FF0000C63F30F0C03
:10D1F000059B6EF31F4C4FF0000E63F30F0E049B64
:10D20000CDF82CC012B28A440027C91763F31F4E11
:10D21000C1EB6A2A039BCDF830E082EA021160F389
:10D220000F070020C9B268F30F00C2F3072269F3A9
:10D230001F4782EA111263F31F404FF000090D9758
:10D240008DF83DA00E908DF83C9042EA01220DF140
:10D25000280C82EAC107BCE80F003FB287F0C8087B
:10D2600088EA0818DFF88CE084F805905FFA88F8FF
:10D27000C7F30727AEE80F0087EA181747EA082325
:10D280009CE8030083EAC8031BB283F023024EF834
:10D29000040B82EA0212D2B2C3F30723079F83EA88
:10D2A0001213704643EA022383EAC20207F1010C1B
:10D2B00020F814194FF023081621FE27C82384F8FC
:10D2C00066C1228084F807800EF1020EA770E1701B
:10D2D000A371114612E000BFAC880020988800209E
:10D2E0005B260020A0470020987900208E7900203E
:10D2F00003082080D4240020CE24002010F8013B15
:10D300004B4083EA0313DBB21A0982EA112242EA94
:10D31000032282EAC3031BB299B270452180EDD18A
:10D3200083F0F40383EA0313DBB24FEA131E8EEAA1
:10D33000112E8EEA032E8EEAC30E0FFA8EFE1FFA0E
:10D340008EF8CA4FA4F800804FEA182C5FFA8EFEC0
:10D3500084F81EE084F81FC07968BA683868FB68F2
:10D3600007F5C778A8E80F0038697969BA6904F247
:10D370008F17A8E8070004F2AD1884F8ADC184F84F
:10D38000ACE117F8011F286803F00EFDB845F8D18D
:10D3900094F85A31002B41F07783B54B1B68192262
:10D3A000990684F85A2140F1FC82B24BB24F1B78A7
:10D3B0009A0741F128873B7D042B8CBF4FF003086F
:10D3C0004FF0020803F0E6F93B8A3A890A9003EB32
:10D3D00083035B00ADF842304FF47A703B680C93E6
:10D3E000F98997F814E07B688DF8448000FB02F21D
:10D3F0004FF0000C0AA84FF0FF398DF845E0CDF84A
:10D400002CC0CDF83C900E920D93ADF840108046A4
:10D410000390B8E80F00DFF870E2AEE80F0098E87C
:10D420000F00AEE807007246182122F81C39E1719E
:10D4300094F8661184F805C081F0780383EA031339
:10D44000D8B2030983F0F60343EA002383EAC0035A
:10D450001BB283EA0310C0B2C3F3072383EA10139D
:10D4600043EA002383EAC0031BB283F0C80080EACA
:10D47000001C5FFA8CFCC3F3072080EA1C1040EA12
:10D480000C2080EACC0000B280F0180383EA03137A
:10D49000DBB2C0F3072080EA131040EA032080EAE1
:10D4A000C30301F101081E204FF0FE0C4FF0C80924
:10D4B000E0700EF1020E217184F86681238084F8F9
:10D4C00002C084F80690184612F8011B414081EA18
:10D4D0000111C9B20B0983EA102343EA012383EA4D
:10D4E000C10109B288B272452080EDD181F01801E6
:10D4F00081EA0111C9B20A0982EA102383EA0123F1
:10D5000083EAC1031BB29AB2DFF860A12280DBB2CA
:10D51000120A0592049384F8272084F82630D64610
:10D520000AF5C77904F12208DEF80000DEF80410DD
:10D53000DEF80820DEF80C30CC46ACE80F000EF127
:10D54000100EC645E146EFD1DEF80000CCF8000031
:10D550009DF81030DFF8348184F8B4319DF8143030
:10D5600084F8B531C14619F8011F286803F01CFC86
:10D57000424B4B45F7D103F00DF9414B414AB3F90A
:10D580000410B7F808E03B680B930A907B680C9393
:10D5900082FB01274FF47A70C9174FF0000C00FB93
:10D5A0000EF0C1EBA701DDF80CE0ADF83CC0ADF822
:10D5B0003EC0ADF840C0ADF842100D900E90BEE8F0
:10D5C0000F00314F84F805C00FC79EE807004FF0E9
:10D5D000210C87E807001C23C8224FF0FE0EE370E1
:10D5E00084F807C084F802E0A27194F866112171F2
:10D5F00081F06A0383EA0313DAB2130983F0D503D7
:10D6000043EA022383EAC2031BB283EA0312D2B2C3
:10D61000C3F3072383EA121343EA022383EAC20314
:10D620001BB283F0C80282EA0212D2B2C3F307230C
:10D6300083EA121343EA022383EAC2031BB283EA9A
:10D640000C0282EA0210C0B2C3F3072282EA10126F
:10D6500042EA0022013182EAC0020C3784F86611E6
:10D660002280A7F11C01104612E000BFCE2400204A
:10D67000AC880020B0880020B488002081260020DB
:10D680009088002067666666D42400205B26002010
:10D6900011F8013B434083EA0313DBB21A0982EA23
:10D6A000102242EA032282EAC3031BB298B2B942B3
:10D6B0002080EDD183F0680383EA0313DBB21909FC
:10D6C00081EA102282EA032282EAC3031BB29AB2E1
:10D6D000DB4F2280DBB24FEA122C049384F8243013
:10D6E00004F1220384F825C007F5C7790593FB6888
:10D6F00038687968BA68CE46AEE80F00059B1037E7
:10D700009F42F146F3D13B88AEF800309DF81030CF
:10D71000CC4F84F8B231C14684F8B3C119F8011F67
:10D72000286803F041FB4F45F8D194F866C1C64A1A
:10D73000C64F84F804C08CF0EB0383EA0313D9B21C
:10D740000B0983F0C50343EA012383EAC1031BB23B
:10D7500083EA0310C0B2C3F3072181EA101141EA42
:10D76000002181EAC0010CCA09B281F0C80E8EEA1C
:10D770000E1E5FFA8EFE4FF000090A92C1F30721D8
:10D78000039A0B93CDF8309081EA1E1343EA0E23DF
:10D7900007CA83EACE031BB283F0310E87E8070085
:10D7A0008EEA0E1E5FFA8EFEC3F3072383EA1E1372
:10D7B00043EA0E2383EACE0394F808E0607AA17A64
:10D7C000E27A277B84F805901BB28EEA030E8EEA7C
:10D7D0000E1E5FFA8EFEC3F3072383EA1E1343EA8D
:10D7E0000E2383EACE031BB2584080EA0010C0B279
:10D7F000C3F3072383EA101343EA002383EAC00339
:10D800001BB2594081EA0110C0B2C3F3072181EA7B
:10D81000101141EA002181EAC00109B24A4082EABE
:10D820000212D2B2C1F3072383EA121343EA02239E
:10D8300083EAC2031BB25F4087EA0717FFB2C3F354
:10D84000072383EA171343EA0723607BA17BE27B6C
:10D8500094F810E094F8119083EAC7031BB2584083
:10D8600080EA0010C0B2C3F3072383EA101343EA2F
:10D87000002383EAC0031BB2594081EA0111C9B2F7
:10D88000C3F3072383EA111343EA012383EAC103A5
:10D890001BB25A4082EA0212D2B2C3F3072383EAD0
:10D8A000121343EA022383EAC2031BB28EEA030E79
:10D8B0008EEA0E1E5FFA8EFEC3F3072383EA1E1361
:10D8C00043EA0E2383EACE031BB289EA030989EAFD
:10D8D00009195FFA89F9C3F3072383EA191343EAA5
:10D8E000092383EAC903A17CE27C594F1BB259404A
:10D8F00081EA0111C9B2C3F3072383EA111343EA92
:10D90000012383EAC1031BB25A4082EA0212D2B257
:10D91000C3F3072383EA121343EA022383EAC20311
:10D920001BB283F0270989EA0912D2B2C3F307298F
:10D9300089EA121949EA022989EAC2090FFA89F922
:10D940001FFA89F20CF101034FEA122E5FFA89F9EE
:10D9500031204FF0FE0C0C2184F86631C823228060
:10D96000E07184F802C0E170A37184F8149084F827
:10D9700015E0DAF80410DAF80820DAF80C30DAF8F2
:10D980000000BAF810C00FC727F803CB84F8A3E152
:10D9900084F8A29118F8011F286803F005FA47459A
:10D9A000F8D194F85EC1BCF1000F41F07880294BAA
:10D9B00094F866E1B3F90010B3F90220B3F904302A
:10D9C0009FED256A214F84F805C007EE103A3368B1
:10D9D0000A938EF06A0383EA031306EE901AD9B213
:10D9E0000B0983F0D50343EA012383EAC1031BB289
:10D9F00083EA03115242C9B207EE902AC3F3072308
:10DA000083EA111343EA0123F8EEE77AF8EEE66AB7
:10DA1000B8EEC77A83EAC1031BB267EE867A66EE78
:10DA2000866A27EE067A002083F0C808CDED0C7ACE
:10DA3000CDED0B6A8DED0D7A0E900F900EE000BFCC
:10DA4000CE2400207F260020D05A0020D42400209D
:10DA50005C2600209088002088C3E43A109088EA71
:10DA600008160DF12809F6B2C3F30728B9E80F002C
:10DA700088EA161848EA062888EAC6080FFA88F8DD
:10DA80000FC788F01E0699E8070086EA0616F6B268
:10DA9000C8F3072383EA161343EA062387E807003F
:10DAA00083EAC606C8214FF005084FF01E0CFE237E
:10DAB0001C200EF10102A17184F85E8184F807C078
:10DAC000A370E070A7F1100184F804E00C37268001
:10DAD00084F8662111F8013B734083EA0313DBB23B
:10DAE0001A0982EA162242EA032282EAC3031BB21F
:10DAF0009EB2B9422680EDD183F0270383EA031357
:10DB0000DBB24FEA131E8EEA162E8EEA032E8EEA41
:10DB1000C30E0FFA8EFE1FFA8EFCD94FA4F800C078
:10DB20005FFA8EFE4FEA1C2C84F825C084F824E0AE
:10DB300007F5C77804F1220938687968BA68FB6884
:10DB400046460FC610374F45B046F5D1CD4E3B88FF
:10DB5000A8F8003006F1240784F8B2E184F8B3C1D4
:10DB600016F8011F286803F01FF9B742F8D194F89E
:10DB70005F81B8F1000F40F08C87C34B1B68052212
:10DB80009B0684F85F2141F10B81C04BDFEDC06A39
:10DB9000DA891B8907EE902A07EE103AF8EEE77A49
:10DBA000B8EE477A67EEA67A94F866C1B94BBA4ADE
:10DBB000B3F90410B2F90620B84EB948CDED0B7A8E
:10DBC0008CF0220383EA0313DFB23B0983F059038D
:10DBD00043EA072383EAC703B2F5FA6F1BB2A8BF73
:10DBE0004FF4FA6283EA0317FFB2B2F57A7FC3F308
:10DBF000072383EA1713B8BF4FF47A724FF0640E0D
:10DC000043EA0723A2F57A720EFB02F283EAC70702
:10DC100086FB02E680FB01E03FB2C917D217C2EBD8
:10DC2000A612C1EBA0034FF000090AA987F0C806AD
:10DC30008DED0C7AADF83A20ADF83830CDF828905B
:10DC4000CDF834908E4686EA0616F6B20391C7F3F5
:10DC50000727BEE80F0087EA161747EA062787EA74
:10DC6000C606904FDEF800E084F804C00FC736B255
:10DC700086F04A0383EA0313DBB2C6F3072181EA85
:10DC800013113A4641EA03210CF1010C81EAC30366
:10DC9000142042F810E9FE264FF04A0E002184F8C5
:10DCA00066C14FF0C80CE0702380043784F807E0A9
:10DCB000A670617184F806C0184612F8011B414035
:10DCC00081EA0111C9B20B0983EA102343EA012357
:10DCD00083EAC10109B288B2BA422080EDD181F055
:10DCE000140181EA0111C9B24FEA111E8EEA102E09
:10DCF0008EEA012E8EEAC10E0FFA8EFE1FFA8EF604
:10DD0000DFF87CA126804FEA162C5FFA8EFE84F89D
:10DD10001CE084F81DC0DAF80410DAF80000DAF824
:10DD20000820DAF80C30BAF818900AF5C7770FC750
:10DD3000DAF81000DAF8141003C704F28F16A7F807
:10DD40000090374684F8ABC184F8AAE104F2AB191D
:10DD500017F8011F286803F027F8B945F8D1524B8E
:10DD6000524A1B781278013B12F00100DBB214BF5B
:10DD7000C0214021172B03D84D4A134493F830801B
:10DD80004C4B1A8897071ABF002341F0100101235A
:10DD900012F4027F18BF022312F0100F18BF0623DF
:10DDA00012F0200F18BF1023002841F002824FF01C
:10DDB000030C94F866E10A938EF0460383EA03139A
:10DDC000DAB2130983F0920343EA022383EAC2031F
:10DDD0001BB283EA0310C0B2C3F3072282EA101217
:10DDE00042EA002282EAC00212B282F0C80787EA41
:10DDF0000717FFB2C2F3072282EA171200238DF839
:10DE00002FC0032042EA072C039A8DF82C808DF84E
:10DE10002D308DF82E108DF8300007CA8CEAC70C13
:10DE20000FFA8CFC1F4FE3718CEA0C1803C75FFAE2
:10DE300088F8CCF3072C8CEA181C4CEA082181EAFC
:10DE4000C80894F808C03A700FFA88F88CEA080CF1
:10DE50008CEA0C1C5FFA8CFCC8F3072282EA1C12C5
:10DE600042EA0C22607AA17A94F80B80637182EA0C
:10DE7000CC0212B2504080EA001C5FFA8CFC1BE01E
:10DE8000CE2400205B260020AC880020B48800202F
:10DE90000AD7233C9088002098790020D34D621047
:10DEA00067666666D4240020D0620020DC71002002
:10DEB000F4DA030898680020C2F3072080EA1C10F7
:10DEC00040EA0C2080EACC0000B2414081EA011116
:10DED000C9B2C0F3072282EA111242EA012282EAA1
:10DEE000C10212B288EA020888EA08185FFA88F8C4
:10DEF000C2F3072282EA181242EA082294F80CC000
:10DF0000607BA17B84F804E082EAC80212B28CEA4A
:10DF1000020C8CEA0C1C5FFA8CFCC2F3072282EA2A
:10DF20001C1242EA0C2282EACC0212B2504080EA71
:10DF30000010C0B2C2F3072282EA101242EA0022A5
:10DF400082EAC00212B2514081EA0111C9B2C2F3A1
:10DF5000072282EA111242EA012282EAC102E17B2F
:10DF600094F8108013B281EA030282EA0212D2B25C
:10DF7000C3F3072383EA121343EA022383EAC203AB
:10DF80001BB288EA030282EA0212D2B2C3F3072369
:10DF900083EA121343EA022383EAC2031BB283F02B
:10DFA000320282EA0212D2B2C3F3072383EA1213C7
:10DFB00043EA022383EAC2031BB29AB24FF0FE0C7B
:10DFC0000920C8210EF1010EDBB284F802C04FEA2D
:10DFD000122CE070A17184F866E1228084F812C0EE
:10DFE0006374DAF80000DAF80410DAF80820BAF8F6
:10DFF0000C9007F5C07EAEE8070007F5C8778EF8ED
:10E000000280AEF8009084F8A0C184F89F3116F821
:10E01000011F286802F0C8FEB742F8D1029BC4F87D
:10E020005031FEF76DBEDFF824A27C4FDFF820925E
:10E03000412026F01BFEBAF9023087FB0320DB17D4
:10E04000C3EBA00080B226F0F5FDBAF9003087FBE3
:10E050000320DB17C3EBA00080B226F0EBFDBAF97A
:10E06000043087FB0320DB17C3EBA00080B226F04F
:10E07000E1FD99F80010D8F8000002F095FE94F840
:10E0800048A11AF0010700F01085654B1B689A063D
:10E0900072D5644B644F1B789B0741F14B803B7DED
:10E0A000042B8CBF4FF0030A4FF0020A472026F0E2
:10E0B000DDFD386826F08AFD786826F087FDFB894B
:10E0C0005A4AD8F80000A2FB0323C3F347131946AA
:10E0D000039302F069FE3A8999F80010039B6420CB
:10E0E0004B4000FB02F089F8003026F06FFD3F7DC9
:10E0F000D8F800004AEA8707FFB2394602F054FE1A
:10E1000099F80030D8F800005F40394689F800706F
:10E1100002F04AFE94F848A1BAF1000F2CD1444F06
:10E120004F2026F0A3FD386826F050FD786826F0D1
:10E130004DFD504626F04AFD0121D8F8000002F0BE
:10E1400033FE384A99F800301778D8F8000007F005
:10E150000107394683F0010389F8003002F024FEFC
:10E1600099F80030D8F800005F40394689F800700F
:10E1700002F01AFE94F848A1029B2E4AC4F84431DA
:10E180000AF10103DBB2A2FB0312D20802EB820206
:10E19000A3EB420384F84831FEF793BD94F8A43210
:10E1A000254AC4F8A0B202EB8302926C42B312ADCE
:10E1B00004F2AB23214E45F8203D002104F2BD239B
:10E1C00031800B9380211523A52784F8AA32284695
:10E1D00084F8A91284F8A872904728463188FBF782
:10E1E0000BFB0A9D164804F52A716D1A152DA8BF60
:10E1F00015252A462CF07CFE124A94F8A43215709C
:10E20000114A013382FB0312A2EBE37202EB4202DA
:10E210009B1A84F8A432FEF783BD00BF676666666A
:10E22000AC880020B0880020B48800201F85EB5106
:10E23000D05A0020CDCCCCCCF4DA0308D67900201B
:10E24000884600209D460020565555559088002050
:10E2500034880020C24AC34BD4F8141130681B889C
:10E2600092F80BE0C04A401A4FF47A71DFB201FB1A
:10E270000EF11B0A9777177588424FF00007D37786
:10E2800053759770177180F0F784B849DFF808C3A9
:10E290000B688968B648B74F007897F814A08CFBD4
:10E2A00003E8DB178CFB01EC4FEAE17EC3EBA8012E
:10E2B00011770912CEEBAC0E5177F4214FEA2E2CD8
:10E2C00082F820E091764FF0010E302182F81BE0B9
:10E2D00082F82210A84B82F821C04FF0750E7821E9
:10E2E00082F823E082F82410820783F81AA040F114
:10E2F000BF84D7F800C0A14AD7F804E0A04882FB49
:10E300000C194FEAEC7182FB0E82C1EBA9514FEA66
:10E31000EE79C9EBA25200FB01C9029200FB02E0B8
:10E3200009EB4909974A4FEA490982FB098204929D
:10E3300000EB4000934A4000039082FB0008049ADF
:10E340009014029A0490F8893F8902EB820200EB54
:10E35000C00002EB820207F5FA770692BAF1050FC8
:10E360004FEA80021FFA87FA0398049F029201EB9A
:10E3700081014FEAE97201EB810105914FEAE071F9
:10E38000A7EB0200804F83F815A0024607FB12920C
:10E39000059F4FEAA84840B200EB8709A8EB0100AF
:10E3A000794F0399804607FB1010069F77494FFA73
:10E3B00088F84FEADC7C4FEADE7E83F809C083F8F8
:10E3C0000EE0DFF8D8C108EB870E029F81FB0781C2
:10E3D0004FEAE778BCF800700397C8EBA1116C4FC7
:10E3E000029187FB021887FB00170299DFF8B0C182
:10E3F0001FFA89F91FFA8EFE4FEAE2724FEAE070C7
:10E40000C2EB681883F80A90C0EB671283F80FE03C
:10E410004FEA19274FEA1E29C1F3072E0399BCF8CA
:10E420000000DF7283F810904FEA222783F80C80F7
:10E430005A749DF80820DA714FEA282C4FEA1A2AFC
:10E440004FEA112934BF4FF032084FF033089DF8DE
:10E450000C2083F80DC09F7483F816A083F808E0A1
:10E46000DA7483F8149083F81B801877C4F810B11D
:10E47000FEF79CBBDFF82C91D9F8000002F080FC7D
:10E4800000283EF42BACD9F80000012102F074FC06
:10E490000222002387F8742088F80030FEF71EBCA3
:10E4A00094F82C1194F82D31D8F800004A1C01334F
:10E4B00084F82C2184F82D3102F076FCFEF7DEBBC7
:10E4C000344CDFF8E4904FF0000A0BE01B2B00F017
:10E4D0009F820D2B00F079814FF0010389F8013004
:10E4E000D8F8000002F05CFC00285FD0D8F80000EB
:10E4F00002F04EFC83B27E2B32682AD099F80110CC
:10E500000029EDD194F82E21002ADFD07D2B00F0D8
:10E51000648294F83CE1BEF1000F04D080F0200347
:10E52000DBB284F83C11511CC9B22244092984F899
:10E530002E1182F8303100F044820829D0D8B4F886
:10E540003A21134403EB132303F0FF03A4F83A31F9
:10E55000C6E784F82EA184F82FA189F801A0BFE7AF
:10E560005872002050720020987A0020788600208F
:10E57000B0880020B4880020C47A00206BCA5F6B8A
:10E58000806967FF83DE1B4340420F00D34D62105A
:10E590001F85EB51CC2400206766666692790020C7
:10E5A0009E6800209C4900202000002094F83D3106
:10E5B00033B194F8313184F83D01302B00F0D78528
:10E5C00094F82F21BA4BBB49DFF818A3DFF8189352
:10E5D00002954FF0010E90464246002A00F05B8300
:10E5E0003268D21B012A00F21F8294F83E21002AD1
:10E5F00040F0348294F83FC133F81C00F0B984F83D
:10E600003FE10A689506E7D59AF800209007E3D520
:10E61000A94FAA49FA89029D4FF4F36303FB02F361
:10E6200081FB0321DB17C3EB61114FF4036026F07C
:10E6300057FB002384F82F31FEF731BB0CF1010C9E
:10E640005FFA8CFCB0F5E06F84F83FC100F09A806F
:10E650001BD8B0F5047F00F0498136D8B0F5887F2B
:10E6600000F0D380B0F5007F00F0B880B0F5807F77
:10E67000B2D10A685207AFD50021029D26F030FBC7
:10E68000002384F82F31FEF70ABBB0F5026F00F0CB
:10E690005E816CD8B0F5E46F00F08480B0F5006F57
:10E6A00000F0DD80B0F5E26F96D1854B029DDA6B0C
:10E6B000998A642303FB02F393FBF1F126F010FB2C
:10E6C000002384F82F31FEF7EABAB0F5826F00F02C
:10E6D0005581B0F5C06F00F02981B0F5806F7FF4EF
:10E6E0007BAF94F84031029D0133DBB2032B00F283
:10E6F000AF8142F2107184F8403101FB03F1714B9C
:10E700001B88002B40F0A28101316F4B1B78DB0787
:10E710006E4B1B8848BF0431DF0748BF0A3198079A
:10E7200048BF14311A0648BF2831DF0548BF2831D9
:10E73000580748BF64311A0748BFC8319F0548BF12
:10E7400001F5C871980648BF01F57A71DA0648BF2D
:10E7500001F5FA615F0648BF01F57A614FF4806008
:10E7600026F0BEFA002384F82F31FEF798BAB0F5F0
:10E77000046F1CD0B0F5116F56D0B0F5036F7FF465
:10E780002BAF3EE74E4B029D90469A6B998A6423CD
:10E7900003FB02F393FBF1F126F0A2FA84F82F8138
:10E7A000FEF77DBA464B029D90461A6CEEE7484B49
:10E7B000029DB3F9041001EB81019046490026F057
:10E7C0008FFA84F82F81FEF76ABA4FF0010184F8BE
:10E7D0002E1184F83031A4F83A2181E699F8062008
:10E7E000002A3FF4F9AE3B4B3B491B68029D81FB7D
:10E7F0000321DB17C3EBA1014FF4007026F070FA80
:10E80000002384F82F31FEF74ABA0A6852077FF5D1
:10E81000E3AE00214FF48870029D26F061FA0023D8
:10E8200084F82F31FEF73BBA99F80520002A3FF40F
:10E83000D3AE2A4A107800283FF4CEAE284B029D72
:10E840001B8803EB8303590091FBF0F14FF4116037
:10E8500026F046FA002384F82F31FEF720BA0A6822
:10E8600095067FF5B9AE9AF8002090077FF5B4AE13
:10E870001CF0010F029D104F104900F068847A6867
:10E8800082EAE273A3EBE27303EB5303A1FB0331D0
:10E89000C908002AACBF41F0004141F040414FF4AB
:10E8A000006026F01DFA002384F82F31FEF7F7B937
:10E8B000F4DA0308AC880020B48800201F85EB51EF
:10E8C00040880020D4790020DC7100209868002066
:10E8D0009088002078860020676666666672002051
:10E8E00050720020B08800209888002099F80520F8
:10E8F000002A3FF471AEC64A107800283FF46CAE8F
:10E90000C44B029D5B7B002B00F08184C24B1B88B3
:10E9100093FBF0F000EB800041004FF4047026F010
:10E92000DFF9002384F82F31FEF7B9B999F80620F2
:10E93000002A3FF451AEB94B029D99684FF4C06074
:10E9400026F0CEF9002384F82F31FEF7A8B90D6820
:10E95000AD067FF541AE9AF800C01CF0020F3FF4FF
:10E960003BAEAF4F029D3B896421904601FB03F112
:10E9700026F0B6F984F82F81FEF791B90A6890065F
:10E9800040F10181A74BA64F1878397D029D00F018
:10E990000203002B0CBF00234FF47A7340F6B83209
:10E9A00008BF4FF4FA6210F0010F18BF1346194464
:10E9B0004FF4826026F094F9002384F82F31FEF79B
:10E9C0006EB9B4F83A21C2F1FF0293427FF484ADEC
:10E9D0004FF0010384F83D317EE54FF0010384F8E8
:10E9E0003C317DE501F0D6FE8F4B1B68C01A40F626
:10E9F000B833984200F25881DFF858A29AF80430F0
:10EA00003A2B00F0C782002388F80030FEF766B981
:10EA1000D8F8000002F0C4F900287FF45DAD4FF093
:10EA2000010384F82F315BE50023029D84F82F3128
:10EA3000FEF735B9C4F8203184F81831DFF81882B0
:10EA400026F09CF994F82431FEF7FDB802315CE61B
:10EA5000012384F8403142F2107150E67349029D5F
:10EA6000062025F027FF002384F83E0184F82F318B
:10EA7000FEF715B9013B84F85731FEF789BC013B1D
:10EA800084F85631FEF763BB013B84F85A31FEF738
:10EA900088BF08F1FF3884F85F81FFF7BFBA0CF137
:10EAA000FF3C84F85EC1FFF762B8614B1B88D80554
:10EAB00013D4D90600F17B839A0600F1DA83580655
:10EAC00000F1DC83190700F1DB83DA0700F1EC8346
:10EAD00013F0020F0CBF04270C27564B564A1B7825
:10EAE000D27803F001030AB143F0020353200393E9
:10EAF00026F0BCF8484A128802EB820202EB82023E
:10EB0000900080B226F096F8002026F093F84B4A49
:10EB10004B491288D8F80000C2EBC212520081FBA8
:10EB2000023111444FEAE27ACAEB612A5FFA8AFAAB
:10EB3000514602F039F999F80020039BD8F80000FB
:10EB40001F438AEA020A002189F800A002F02CF98A
:10EB50003946D8F8000002F027F999F80030D8F8C3
:10EB600000007B40DBB2194689F8003002F01CF946
:10EB700094F848A1FFF7D0BA32493A2025F09AFE1E
:10EB80002870FEF7C1B8304A1268120600F1F78209
:10EB9000204A127B002A3FF41FAD94F84111029DD8
:10EBA000032900F28383DFE801F059281902274B7B
:10EBB0001B6859799A79DB7901F1407101EB0221E7
:10EBC00001EB0341002384F841314FF4826026F0C9
:10EBD00087F8002384F82F31FEF761B81C4B1A68C0
:10EBE000137A507992781B0403EB002313444A1CD8
:10EBF00084F8412103EB0161E7E7154B1A68D379EB
:10EC0000107952781B0403EB00231344EFE700BF95
:10EC10006672002058720020507200207886002012
:10EC2000B4880020B088002044490020D94C030853
:10EC300098680020DC710020EC6100208E790020B3
:10EC4000030820800D250308A8760020ECB00020E2
:10EC5000B86800202C49002038880020BA4B1A6878
:10EC60009379D07812781B0403EB00231344BEE79A
:10EC70002D22DA76FFF7FABBB44B31681B78C4F863
:10EC80001411013B012B3FF600AB102102239170C0
:10EC90001371FFF7FABA029DFEF701B826F05EF88D
:10ECA00001233B70FDF7A0BFA94AB2F84A31002109
:10ECB0000133A2F84A3188F80010FEF70FB8A54ECC
:10ECC000A54B00930024A6F13F01A44BA44A089150
:10ECD00006F8404CA34909960AA8FAF764FE089E74
:10ECE000731C08933470089B2922591C08911A70D0
:10ECF000089BEA22591C08911A70089BC822591CCB
:10ED000008910AA81A702BF0B5F9471C0AA93A46CF
:10ED100008982CF0EDF8089AD31901330893D455CC
:10ED2000089B5A1C08921C70089B5A1C08921C7065
:10ED3000089B5A1C08921C70089B5A1C08921C7055
:10ED4000089B5A1C08921C70089B5A1C08921C7045
:10ED5000089B5A1C08921C70089B5A1C08921C7035
:10ED6000089B5A1C08921C70089B5A1C08921C7025
:10ED7000089B5A1C08921C70089BFF22591C089182
:10ED80001A70089B0122991812A808911A7050F85D
:10ED9000283D9B1B337023F089FB2C70FDF7B4BF1B
:10EDA000DFED717AB0EE677AFEF7FEBE88468946DF
:10EDB0000846049105918E4606910391FEF7FAB933
:10EDC000644A6A4B0B9212AEA2F13D0046F8200D48
:10EDD0001988674FA2F1400300204FF00A0E02F895
:10EDE000400C082283F801E030469A70FAF7E0FC04
:10EDF0003B686049DA1781FB0313C2EBA30399B2A6
:10EE00003046FAF7D5FC0BF06DFDBF680A9B3A0C53
:10EE1000591C0A911A700A9B3A0A591C0A911A70D5
:10EE20000A9B5A1C0A921F700A9B5A1C0A9218705D
:10EE3000304623F03BFBFEF71CB84F4F9FED4F8A47
:10EE4000B7F9022043480B9007EE902AF8EEE77AD4
:10EE500012AE67EE887AA0F13D01FDEEE77A46F842
:10EE6000201D00F8403C0823CDED027A00F83F3C1D
:10EE70001E23BDF8081000F83E3C3046FAF798FC17
:10EE8000B7F9003007EE903AF8EEE77A304667EED1
:10EE9000887AFDEEE77ACDED027ABDF80810FAF730
:10EEA00087FCB7F9043007EE903AF8EEE77A30467F
:10EEB00067EE887AFDEEE77ACDED027ABDF80810AC
:10EEC000FAF776FC304623F0F1FAFDF7CFBF2C4A73
:10EED000204B12680B93A3F14007002103F8401C5C
:10EEE0002123D100BB7040F1B88126490326264B6F
:10EEF0001B885A0500F1A681D80700F1BC8103F0F8
:10EF00000203224A002B1CBF03261146DFF8808033
:10EF1000324640462BF0ECFF06EB080312A8013303
:10EF2000A8F1020140F8203D00225B1A06F80820F3
:10EF30007B7023F0BBFAFDF79FBFC4F81CB187F8C4
:10EF40000090FDF751BE00BFB8680020C8790020CE
:10EF5000CC240020187A0020668F00207C09040849
:10EF60008409040890090408000000005072002081
:10EF700078860020676666669088002058A08B41DE
:10EF8000CC790020680904089868002078090408F2
:10EF9000DB7900209AF80240C4B1013CE4B20134AC
:10EFA00054445146002211F8013B534083EA0313B5
:10EFB000DBB2120ADF0042EA03228C4287EA131313
:10EFC00082EA0302EFD1002A7FF41DADBC4ABD4F97
:10EFD000BD4B1288BD4CFA61DFF824931A68FA62BF
:10EFE0009B68B4F84A21F8660021FB64D9F8000058
:10EFF000F963FA6500F0DAFA029000287DF469AE50
:10F000000221D9F8000001F0B7FE94F84C319AF8CB
:10F0100003200392642B4FF0040287F8742040F021
:10F02000738194F84D31072B04BF9DF8083084F8A4
:10F030004D3194F84D31069307EB031ADAF80410BA
:10F04000029108462BF016F8DAF8081005915FFADD
:10F0500080FA08462BF00EF8C0B204900AEB0002CA
:10F06000069B9B48029902900832C27123F00F025E
:10F0700086468272049803F00F0300EBCA008EF8F4
:10F080000D3052468EF80E000EF10F002BF030FFBF
:10F09000904B049A05990AF1090018442BF028FFB7
:10F0A0000298C37903F1010ACBB1013B5FFA83FCFB
:10F0B0000CF1080CDFF84CE284440023073010F810
:10F0C000011B59408B00CA0883EA410302F0180271
:10F0D0004B404EFA02F253408445DBB2EFD17D4AF9
:10F0E00003980AF8023029F071FA94F84D310022A1
:10F0F000013384F84D3184F84C21029BDDF808A0DF
:10F100009B785BB11AF80510D9F8000001F04CFEAD
:10F1100001359AF80230EDB2AB42F3D894F84C3195
:10F120000322013384F84C3187F8742088F80020DA
:10F13000FFF7A2B94FF0010AFEF7B8BF0221D8F8D5
:10F14000000001F019FE94F82431FDF77CBD3A6807
:10F1500082EAE273A3EBE27303EB5303A1FB0331F7
:10F16000C908002AB8BF41F08041FFF798BB5A494F
:10F17000881F25F043FC84F83E01FFF721BA1023D5
:10F180000027042218460AA9029D8DF828308DF820
:10F1900029208DF82A708DF82B708DF82C708DF841
:10F1A0002D7025F07DFD84F82F71FDF778BD342793
:10F1B00093E44A4AD278002A0CBF4FF0040C4FF077
:10F1C000050CFEF7F6BD0123D8F800003B7001F0F6
:10F1D000DFFD0746D8F8000001F0DAFD7B067DF47C
:10F1E00003AD8A284ED08E287DF4FEAC94F81831F9
:10F1F000002B7DF416AD3A4BC4F820312D2384F852
:10F200002431FDF7F8BC4FF00108FEF7DBB82C4BBA
:10F210001888FFF77FBB2A499A790B8803EB830391
:10F2200003EB83034FEA83081FFA88F8002A00F0F3
:10F230001081254B1B680FFA83FA0BF053FB40B289
:10F24000FDF7C0BE0326274960E698469946184652
:10F25000049305930393FDF7ADBF234B234A1B682B
:10F26000234903F48003002B16BF1146042603260E
:10F270003DE6242731E41F49042647E610272CE405
:10F2800020272AE41C4B1B689F067DF5ADAC94F843
:10F290001831002B7DF4C5AC184BC4F820312D2358
:10F2A00084F82431FDF7A7BC082716E44B1CDBB219
:10F2B000042B84F841314FEA01613FF483AC84E4CC
:10F2C000507200202000002078860020CC240020EE
:10F2D000D4A90020DAA9002004260020EC61002037
:10F2E000987A00206C090408A876002068090408B0
:10F2F0006009040870090408AC880020C47A002062
:10F300009C4900200007090E97F875A05B490495F9
:10F310001AF00F0F04BF0AF1010A5FFA8AFABAF174
:10F32000070F28BF4FF0010A4FEA0A1C07EB0C0336
:10F33000187C534B02930A18002392F82410504A69
:10F3400093725FFA8CF31A464E4B964607EB0C020B
:10F350004EEA000001291870D26803F101000CD9AF
:10F360000239C9B28D1C1D44034603F8012BAB4280
:10F370004FEA1222F9D101310844BC4422F0600363
:10F380000AF1010A9CF811205FFA8AFA1343BAF1D4
:10F39000080F037000F1010340D04FEA0A1C07EB8D
:10F3A0000C01384A087C354901449A1A91F8241016
:10F3B00055180EF1100E132D5FFA8EFEC6DD049D5A
:10F3C0000298DFF8CCE0D2B2931DDBB243F04001EB
:10F3D000C17103F1010CCBB10532D3B20833C318AC
:10F3E00004930EF10100002310F8011B59408B001B
:10F3F00083EA4103CA084B40234902F0180241FA4C
:10F4000002F25340049A8242DBB2EDD103980CF829
:10F410000E3087F875A029F0D9F86EE6194A049DD8
:10F420009A1ACDE7984699461846049305939E4646
:10F430000393FDF7BFBE154B9046B3F900A06420BF
:10F44000FDF7C0BD98469946184604930393FDF70F
:10F45000B1BE4FF0FF33EEE60393FDF7ABBE984627
:10F460000393FDF7A7BE984699460393FDF7A2BE06
:10F470009846994618460393FDF79CBEF4DA0308B4
:10F48000D4A90020E1A900200007090E78860020F9
:10F49000DAA90020436A8269D154436A0169426B48
:10F4A00001338B4228BF00234362002A2FD0EFF3A1
:10F4B0001182502383F31288436B1968C9072CD437
:10F4C00070B45E686EB9456A816A8D4217D08469EE
:10F4D0000C44DC600ED9691A59608562002180F8FD
:10F4E0005810196841F00101D2B2196082F31188F5
:10F4F00070BC70470469611A59608662EEE70123A7
:10F5000080F85830D2B282F3118870BC7047426DD7
:10F51000D36843F08003D3607047D2B282F311887E
:10F52000704700BF026B10B462B1836CC26844695B
:10F53000D11A013B615C5DF8044B08BF134683643C
:10F54000C8B27047016A4369C4685B5C0131A1427B
:10F5500028BF114601625DF8044BD8B2704700BF66
:10F56000436B13B190F858007047836A406A181AC9
:10F57000B0FA80F040097047416A836A99420AD321
:10F58000CB1A416B026961B14968501E0B4483423A
:10F590000AD2C01A704702691144CB1A416B002984
:10F5A000F2D1501EC01A704700207047036B43B160
:10F5B000826C5B6893422FBF981AC0689B1AC01870
:10F5C0007047C269036A9A422FBFD01AC068801878
:10F5D000C01A70470A4B30B503F1100493F90020AC
:10F5E0005D78072AC8BF143A811804338D7213F866
:10F5F000025C855413F8012C0A75A342EED130BD8C
:10F6000048DB030803682DE9F041DF691FB13B4681
:10F61000BDE8F0411847002A164611DD04460D46A4
:10F620000E4400E023689B68204698470028F9D0E4
:10F63000236815F8011B1B6820469847AE42F1D19C
:10F64000BDE8F081002325212622017042708370DD
:10F65000C3707047038A2DE9F0478589ADB21D401C
:10F6600029D00F4606464FF000484FF00009B5FA82
:10F6700085F328FA03F2D24391B21B3B1540318245
:10F68000042B16D8DFE803F03129211903007B6A27
:10F69000002B32D003F1FF3A1FFA8AFAC7F8249000
:10F6A0003C6A34B123682046514698476468002C70
:10F6B000F8D1002DDBD1BDE8F0873868716B0368A5
:10F6C00089B29847002DD2D1F5E77868B16B03680D
:10F6D00089B29847002DCAD1EDE7B868F16B03688D
:10F6E00089B29847002DC2D1E5E7F868316C03680C
:10F6F00089B29847002DBAD1DDE7F36A1FFA83FA81
:10F70000CEE700BF30B50446406D61718389A268C1
:10F7100023F400531B041B0C838185B0A379009252
:10F7200013F0040230D04FF4805213F00203ADF80E
:10F7300004205CD1ADF806304FF480630022ADF8B0
:10F74000083011F00103ADF80C2028D1ADF80A30D3
:10F7500008238D07694648BFADF80A301EF0EEFB5E
:10F76000A279636DD10724D412F0080F9A8A1BD1B5
:10F7700022F008021204120C9A829A8992B242F480
:10F7800000529A8105B030BD13F00203ADF8042099
:10F790002AD04FF400551346ADF80650CEE70423A7
:10F7A000ADF80A300C23D4E792B242F008029A82F4
:10F7B000E3E710498B4215D0A1F548418B420FD0A9
:10F7C00001F580618B4209D00B498B42CCD10520D9
:10F7D0000121FBF721F8A279636DC5E70320F7E764
:10F7E0000220F5E70020F3E7ADF80630A6E74FF476
:10F7F00000539FE7001001400014014010B504467B
:10F80000406DA160838923F400531B041B0C83818A
:10F81000A37984B013F00402009135D04FF48052E4
:10F8200013F00203ADF804205CD1ADF806304FF4BC
:10F8300080636279ADF80830D1074FF00003ADF86E
:10F840000A30ADF80C3045BF0423ADF80A30082368
:10F850000C236946920748BFADF80A301EF06EFBD4
:10F86000A279636DD1071FD412F0080F9A8A16D1BE
:10F8700022F008021204120C9A829A8992B242F47F
:10F8800000529A8104B010BD13F00203ADF80420B9
:10F8900025D04FF400511346ADF80610C9E792B2D7
:10F8A00042F008029A82E8E710498B4215D0A1F590
:10F8B00048418B420FD001F580618B4209D00C4941
:10F8C0008B42D1D105200121FAF7A6FFA279636D01
:10F8D000CAE70320F7E70220F5E70020F3E7ADF8D9
:10F8E0000630A6E74FF400539FE700BF0010014029
:10F8F000001401402DE9F04F7822002183B08A489E
:10F900008A4CDFF84C928A4D8A4E8B4FDFF8448246
:10F910002DF003FE89488A49DFF83CE2DFF83CC25B
:10F9200000221359834200F0D480B3F1804F00F0DD
:10F93000E480AB4200F0E380B34200F0E280BB42DF
:10F9400000F0E180734500F0E080634500F0DF8067
:10F95000434500F0DE80DFF808A2534500F0DB806D
:10F960000AF5806A534500F0D8800AF5806A53454D
:10F9700000F0D580AAF5983A534500F0D2800AF5F8
:10F98000806A53457BD00AF5806A534508BF0D2332
:10F9900076D01832902AC4D1644C6A4E6A4F6B4DAF
:10F9A00004F1900802E01834A04565D0A379002B3B
:10F9B000F9D023794FEA131909F1FF39B9F1030F8F
:10F9C00003F00F03EFD836F8190040FA03F2D2071C
:10F9D000E9D54FF0010A0AFA03F3013B18402BF076
:10F9E00013F817F80930184415EBC002DBD055F8AE
:10F9F0003000DFF870E1217A00F13F4303F57E0328
:10FA00009B0A1EF8033003F01F0E5B09032B0AFA52
:10FA10000EFA60D0042B67D0022B51D0938800934C
:10FA2000B3FA83F3C3F11F039BB2DA0800EB82023F
:10FA300003F00703D2F820E09B004FF00F0C0CFA04
:10FA400003FC2EEA0C0EC2F820E0D2F820E001FA06
:10FA500003F343EA0E0313626946002302221834BB
:10FA60008DF804208DF805308DF806308DF80730BC
:10FA700023F004FDA04599D103B0BDE8F08F0C231D
:10FA800009EBC3034FF0010A1B7D03F01F0B5B0959
:10FA9000032B0AFA0BFA0ED0042B07D0022B7FF4AB
:10FAA00078AF4B6C4AEA03034B6472E70B6B4AEA8C
:10FAB00003030B636DE70B6C4AEA03030B6468E70F
:10FAC000DFF87CE0DEF844304AEA0303CEF8443045
:10FAD000A4E70023D4E7DFF868E0DEF840304AEA24
:10FAE0000303CEF8403099E7DFF854E0DEF8303019
:10FAF0004AEA0303CEF8303090E70123C0E702233F
:10FB0000BEE70323BCE70423BAE70523B8E70623CF
:10FB1000B6E70723B4E70823B2E70923B0E70A23CF
:10FB2000AEE70B23ACE700BF90700020380004085C
:10FB30000004004000080040000C004000000140AC
:10FB400000380240CC000408C8000408D883002014
:10FB500048DB03080004014000100040001400408E
:10FB6000004001401001040800286AD003682DE914
:10FB7000F04F03F13F4404F57E045F4EA40A0125D3
:10FB8000345D04F01F066409032C05FA06F559D00C
:10FB9000042C00F0AC80022C59D08588B5FA85F091
:10FBA000C0F11F0080B2C40803EB840400F007001A
:10FBB000266A80000F27874026EA07062662276A02
:10FBC00001F003068240701E3A430128C1F3810C04
:10FBD000C1F300182262C1F341113DD9002422462D
:10FBE00001274FF0030E03E0102A04F1020426D08F
:10FBF00007FA02F0A84302F10102F5D1D3F800C0E0
:10FC00000EFA04F0C04300EA0C0CC3F800C0D3F8AD
:10FC1000008006FA04FC4CEA080CC3F800C0D3F8D4
:10FC20000CC000EA0C00D860D3F80CC001FA04F054
:10FC300040EA0C00102AD86004F10204D8D1BDE8D3
:10FC4000F08F70472D4C266C35432564A5E72B4C6F
:10FC5000666C35436564A0E7002002464FF0010E54
:10FC60004FF0030904E00132102A00F102003CD0F9
:10FC70000EFA02F737EA0504F5D1D3F800A009FA25
:10FC800000F4E4430AEA040AC3F800A0D3F800B081
:10FC900006FA00FA4AEA0B0AC3F800A0D3F808A053
:10FCA00004EA0A0AC3F808A0D3F808B00CFA00FA6C
:10FCB0004AEA0B0AC3F808A0D3F804A02AEA070707
:10FCC0005F60D3F804A008FA02F747EA0A075F600A
:10FCD000DF683C40DC60DF6801FA00F401323C433D
:10FCE000102ADC6000F10200C2D1BDE8F08F034CA5
:10FCF000266B3543256350E71001040800380240A5
:10FD000003682DE9F04F03F13F4404F57E04604E93
:10FD1000A40A0125345D04F01F066409032C05FACA
:10FD200006F500F0AF80042C00F0A780022C54D020
:10FD30008588B5FA85F0C0F11F0080B2C40803EBD6
:10FD4000840400F00700266A80000F27874026EA17
:10FD500007062662276A01F0030602FA00F0721E07
:10FD60003843012AC1F3810CC1F300182062C1F3AA
:10FD7000411137D90024224601274FF0030E03E03A
:10FD8000102A04F1020426D007FA02F0A84302F177
:10FD90000102F5D1D3F800C00EFA04F0C04300EA26
:10FDA0000C0CC3F800C0D3F8008006FA04FC4CEA3F
:10FDB000080CC3F800C0D3F80CC000EA0C00D860EF
:10FDC000D3F80CC001FA04F040EA0C00102AD86005
:10FDD00004F10204D8D1BDE8F08F2E4C666C354397
:10FDE0006564A5E7002002464FF0010E4FF00309BD
:10FDF00004E00132102A00F102003CD00EFA02F7B2
:10FE000037EA0504F5D1D3F800A009FA00F4E44379
:10FE10000AEA040AC3F800A0D3F800B006FA00FA10
:10FE20004AEA0B0AC3F800A0D3F808A004EA0A0AB9
:10FE3000C3F808A0D3F808B00CFA00FA4AEA0B0A93
:10FE4000C3F808A0D3F804A02AEA07075F60D3F834
:10FE500004A008FA02F747EA0A075F60DF683C403F
:10FE6000DC60DF6801FA00F401323C43102ADC60F8
:10FE700000F10200C2D1BDE8F08F064C266B35437D
:10FE8000256355E7034C266C3543256450E700BFD6
:10FE9000100104080038024010B50409013C032C8D
:10FEA00017D80D4B33F8142000F00F0042FA00F37E
:10FEB00013F001030DD0012303FA00F001381040C4
:10FEC0002AF0A2FD054A064B125D104403EBC00068
:10FED00010BD002010BD00BFCC000408C8000408FD
:10FEE000D883002001490248FFF7B4BBE07000202E
:10FEF0000008004001490248FFF7ACBBB870002081
:10FF00000004004002494FF08040FFF7A3BB00BF50
:10FF100090700020F0B50668B30AA3F58013022B99
:10FF200050D8384CE55C022D4CD84379A8009F0886
:10FF3000002952D09C080223B6F80CE0A3404419D3
:10FF400007EB440743EA0E032F4C07F1040E9BB264
:10FF500044F8271044F82E20B381EFF31181502389
:10FF600083F312884219D200A7183B695BB33B6246
:10FF70000433421904EBC202576917B11F60536979
:10FF80000433421904EBC202976917B11F609369E9
:10FF90000433421904EBC202D76917B11F60D36959
:10FFA00004330022C9B21A6081F31188284404EB9B
:10FFB000C004236A5BB9B38923F001031B041B0C43
:10FFC000B381F0BDF0BD02F120032344D1E7B38932
:10FFD0009BB243F00103B381F0BDB3890A4C4FF0EB
:10FFE000020E0EFA07FE9BB223EA0E0300EB050E8B
:10FFF00007EB4E07B3813B1D44F8271044F823203C
:020000040801F1
:10000000ABE700BFECFE03089070002010B503685A
:1000100082480139834282B089B200F0CA80A0F5DB
:100020008060834200F0C58000F58040834200F08C
:10003000B78000F58060834200F0B28000F58060F8
:10004000834200F0AD80764C188824686408B4FBC5
:10005000F2F4013CA4B282B2B3F1804F0AD07148ED
:10006000834207D000F58060834203D000F58060B2
:10007000834202D122F0700292B26B48834200F0B8
:10008000A18000F58060834200F0A68022F44072D7
:1000900000F56C4092B283421A80D9621C854FD021
:1000A0005E4A93424CD001229A821A8892B242F060
:1000B00001021A80B3F1804F00F09880594A9342B0
:1000C00000F0968002F58062934200F0938002F582
:1000D0008062934200F0908002F58062934200F0CB
:1000E0008D8002F58062934200F08A8002F57042B2
:1000F000934200F0878002F57052934200F08480B2
:1001000002F58062934200F0818002F580629342A2
:100110007ED0A2F5983293427CD002F58062934261
:100120007AD002F58062934208BF0D2215D002A852
:100130004FF0012340F8043D1DF0C8FE02B010BD91
:100140000122002119869A821A88384892B242F018
:10015000010283421A80ADD10A46354B03EBC2033C
:1001600001A85C7D8DF80440012300228DF8053044
:100170008DF807308DF806201DF0A8FE1B2C08D046
:100180002E2CDBD12B4B019301A81DF09FFE02B05A
:1001900010BD294B019301A81DF098FE02B010BDBF
:1001A0001F4C18882468B4FBF2F4013CA4B282B25C
:1001B00052E71B4C18882468B4FBF2F4013CA4B24B
:1001C00082B257E701201A80D9621C8598821A886A
:1001D00092B202431A8071E701201A80D9621C850D
:1001E00098821A8892B202431A8063E70122B4E728
:1001F0000222B2E70322B0E70422AEE70522ACE711
:100200000622AAE70722A8E70822A6E70922A4E710
:100210000A22A2E70B22A0E70C229EE7000401407D
:1002200078900020000400400010004000000140D1
:1002300048DB03082C010001190100012B4B9842F7
:100240003CD0B0F1804F3BD0A3F57C43984239D0ED
:1002500003F58063984237D003F58063984235D028
:1002600003F58063984233D003F58063984231D020
:1002700003F5704398422FD003F5705398422DD068
:1002800003F5806398422BD003F58063984229D010
:10029000A3F59833984227D003F58063984207D09E
:1002A00003F58063984208BF0D2202D000207047FA
:1002B0000C220F4B03EBC203187D70470022F8E7B6
:1002C0000122F6E70222F4E70322F2E70422F0E734
:1002D0000522EEE70622ECE70722EAE70822E8E734
:1002E0000922E6E70A22E4E70B22E2E700000140E8
:1002F00048DB03082DE98048013085B0C3B2039381
:100300008A4D8B4F8B4C8C4E0A230293DFF82C9234
:1003100025F064FE4FF4FA7A4FF0100C4FF47A7027
:10032000D9F80430C3F30803002B40F0C180EFF389
:100330001183002B40F0BC802968A26800BF2B68A5
:100340009942F9D1D7F800E000FB0EF39B1AB3FBFA
:10035000FEF300FB01314FF0010E0191D9F804309A
:10036000C3F30803002B40F08780EFF31183002BC9
:1003700040F082802B68A16800BF2A689342F9D1BF
:10038000D7F800B000FB0BF2521AB2FBFBF200FBF5
:100390000323019A9B1AB3F57A7FDFD3BAF1010ADE
:1003A000BED1039B002B40F0BD804FF47A7ADFF87A
:1003B0008C9150464FF0100CD9F80430C3F3080369
:1003C000002B40F09280EFF31183002B40F08D80E2
:1003D0002968A26800BF2B689942F9D1D7F800E0DC
:1003E00000FB0EF39B1AB3FBFEF300FB01314FF051
:1003F000010E0191D9F80430C3F3080303BBEFF3F6
:100400001183EBB92B68A16800BF2A689342F9D128
:10041000D7F800B000FB0BF2521AB2FBFBF200FB64
:100420000323019A9B1AB3F57A7FE3D3BAF1010A49
:10043000C2D1029B013B02937FF468AFFAF7D0F977
:10044000EFF311888CF31288A1682368DB0344BFA3
:10045000C6F800E0A1682B6832685FFA88F888F374
:100460001188D7F800801A4400FB08F35B1AB3FB2D
:10047000F8F300FB0233D4E7EFF311888CF3128812
:10048000A1682368DB0344BFC6F800E0A1682B68BD
:1004900032685FFA88F888F31188D7F800801A4428
:1004A00000FB08F35B1AB3FBF8F300FB023370E7C1
:1004B000EFF311828CF31288D4F808E02368D90393
:1004C00003D501233360D4F808E02B683168D2B239
:1004D00082F311883A68194400FB02F3A3EB0E0380
:1004E000B3FBF2F300FB013135E7EFF311828CF33C
:1004F0001288D4F808E02368D90303D501233360B8
:10050000D4F808E02B683168D2B282F311883A68D7
:10051000194400FB02F3A3EB0E03B3FBF2F300FB61
:10052000013164E7184623F03FFE3EE724860020B1
:100530002886002010E000E02086002000ED00E08A
:100540002DE9F04F013085B0C3B203930B46029101
:100550008B4C8C4E002B00F099808B4D8B4FDFF82D
:10056000309225F03BFD4FF4FA7A4FF0100C4FF427
:100570007A70D9F80430C3F30803002B40F0DE8012
:10058000EFF31183002B40F0D9802968A26800BFE7
:100590002B689942F9D1D7F800E000FB0EF39B1AC3
:1005A000B3FBFEF300FB01314FF0010E0191D9F8CE
:1005B0000430C3F30803002B40F08780EFF311836E
:1005C000002B40F082802B68A16800BF2A6893420C
:1005D000F9D1D7F800B000FB0BF2521AB2FBFBF2D4
:1005E00000FB0323019A9B1AB3F57A7FDFD3BAF19C
:1005F000010ABED1039B002B40F0BD804FF47A7AF4
:10060000DFF88C9150464FF0100CD9F80430C3F34A
:100610000803002B75D1EFF31183002B71D12968EA
:10062000A26800BF2B689942F9D1D7F800E000FB1F
:100630000EF39B1AB3FBFEF300FB01314FF0010EEA
:100640000191D9F80430C3F3080313BBEFF311830E
:10065000FBB92B68A16800BF2A689342F9D1D7F88B
:1006600000B000FB0BF2521AB2FBFBF200FB0323BB
:10067000019A9B1AB3F57A7FE3D3BAF1010AC4D188
:10068000029B013B0293002B7FF467AF05B0BDE8EE
:10069000F08FEFF311888CF31288A1682368DB03D5
:1006A00044BFC6F800E0A1682B6832685FFA88F89A
:1006B00088F31188D7F800801A4400FB08F35B1A0E
:1006C000B3FBF8F300FB0233D2E7EFF311888CF3AE
:1006D0001288A1682368DB0344BFC6F800E0A16864
:1006E0002B6832685FFA88F888F31188D7F80080A1
:1006F0001A4400FB08F35B1AB3FBF8F300FB023368
:1007000070E7EFF311828CF31288D4F808E02368C5
:10071000D90303D501233360D4F808E02B6831688E
:10072000D2B282F311883A68194400FB02F3A3EBBA
:100730000E03B3FBF2F300FB01317FE7EFF311820D
:100740008CF31288D4F808E02368D90303D5012379
:100750003360D4F808E02B683168D2B282F3118894
:100760003A68194400FB02F3A3EB0E03B3FBF2F368
:1007700000FB013118E7184623F016FD3EE700BFE5
:1007800010E000E02086002024860020288600203B
:1007900000ED00E0204B5B68C3F3080330B4BBB945
:1007A000EFF31183A3B91D4B1D4C1868A16800BF5E
:1007B0001A689042F9D11B4B1C684FF47A7202FB05
:1007C00004F3591AB1FBF4F130BC02FB001070477E
:1007D000EFF31182102383F3128811498C680B68A0
:1007E00013F4803F104B02D0012018608C680B4935
:1007F000D2B20D68186882F311880A4B19684FF459
:100800007A72284402FB01F31B1B30BCB3FBF1F3EB
:1008100002FB0030704700BF00ED00E0248600209E
:1008200010E000E028860020208600202DE9F84F07
:100830008046FFF7AFFF254E2549DFF8A0E0254AA7
:10084000254D844610274FF47A740120DEF80430D9
:10085000C3F30803D3B9EFF31183BBB90B68D2F824
:1008600008A000BFD1F800904B45F7D1D6F800B0F2
:1008700004FB0BF9A9EB0A09B9FBFBF904FB039391
:10088000A3EB0C034345E1D3BDE8F88FEFF3118AE6
:1008900087F31288D2F808B01368DB0344BF2860DE
:1008A000D2F808B00B68D5F800905FFA8AFA8AF39C
:1008B0001188D6F800A0994404FB0AF3A3EB0B03BC
:1008C000B3FBFAF304FB0933DAE700BF2886002004
:1008D0002486002010E000E02086002000ED00E0EB
:1008E0002DE9F04FDFF830C1474A4849484E494D9D
:1008F0008046102718F1FF38C0F08480DCF80430FF
:10090000C3F30803002B5CD1EFF31183002B58D104
:100910000B68946800BF08688342F9D1D6F800904C
:100920004FF47A7000FB09FEAEEB040EBEFBF9FE3D
:1009300000FB03EEDCF80430C3F308034FF47A74D1
:100940000120FBB9EFF31183E3B90B68D2F808A0DB
:1009500000BFD1F800904B45F7D1D6F800B004FBAA
:100960000BF9A9EB0A09B9FBFBF904FB0393A3EB11
:100970000E03B3F57A7FBDD2DCF80430C3F308036D
:10098000002BDFD0EFF3118A87F31288D2F808B07A
:100990001368DB0344BF2860D2F808B00B68D5F8B1
:1009A00000905FFA8AFA8AF31188D6F800A0994479
:1009B00004FB0AF3A3EB0B03B3FBFAF304FB0933C9
:1009C000D5E7EFF3118487F31288D2F80890136803
:1009D000D80303D501232B60D2F808900B68286850
:1009E000E4B284F31188D6F800A04FF47A7400EBD7
:1009F000030E04FB0AF3A3EB0903B3FBFAF304FBB6
:100A00000E3E97E7BDE8F08F10E000E0248600205E
:100A1000288600202086002000ED00E030B4EFF3AF
:100A20001183102282F312880649074C0A6807488E
:100A3000013200250A602560DBB2026883F3118869
:100A400030BC7047248600202086002010E000E0A3
:100A500038B5254B5C69236B73B1636D626BCAB1AA
:100A6000998A1A88C90592B201D5D20700D438BD37
:100A70004FF6F7721A8038BD636D99891A88890616
:100A800092B2EBD59206E9D5E26ACAB1988880B2F3
:100A90009047E2E799891A880D0692B2E0D51006D0
:100AA000DED5A26A616A8A4219D0A1692569885C8B
:100AB00098800132B2FBF5F105FB1122A262CFE76B
:100AC0009B88E2696169DBB28B54E269E068636D1F
:100AD0000132B2FBF0F100FB1122E261BEE7DA68FD
:100AE00022F08002DA60BBE7983D002038B5254B44
:100AF000DC68236B73B1636D626BCAB1998A1A8823
:100B0000C90592B201D5D20700D438BD4FF6F772AD
:100B10001A8038BD636D99891A88890692B2EBD51F
:100B20009206E9D5E26ACAB1988880B29047E2E7B6
:100B300099891A880D0692B2E0D51006DED5A26A10
:100B4000616A8A4219D0A1692569885C988001325E
:100B5000B2FBF5F105FB1122A262CFE79B88E269A7
:100B60006169DBB28B54E269E068636D0132B2FB0C
:100B7000F0F100FB1122E261BEE7DA6822F08002A8
:100B8000DA60BBE7983D002038B5254B9C68236BA5
:100B900073B1636D626BCAB1998A1A88C90592B242
:100BA00001D5D20700D438BD4FF6F7721A8038BD90
:100BB000636D99891A88890692B2EBD59206E9D5B8
:100BC000E26ACAB1988880B29047E2E799891A88A8
:100BD0000D0692B2E0D51006DED5A26A616A8A429D
:100BE00019D0A1692569885C98800132B2FBF5F1C2
:100BF00005FB1122A262CFE79B88E2696169DBB243
:100C00008B54E269E068636D0132B2FBF0F100FBE6
:100C10001122E261BEE7DA6822F08002DA60BBE707
:100C2000983D002038B5254B1C68236B73B1636D6C
:100C3000626BCAB1998A1A88C90592B201D5D207E6
:100C400000D438BD4FF6F7721A8038BD636D9989AC
:100C50001A88890692B2EBD59206E9D5E26ACAB142
:100C6000988880B29047E2E799891A880D0692B277
:100C7000E0D51006DED5A26A616A8A4219D0A16960
:100C80002569885C98800132B2FBF5F105FB1122E1
:100C9000A262CFE79B88E2696169DBB28B54E269AB
:100CA000E068636D0132B2FBF0F100FB1122E261FA
:100CB000BEE7DA6822F08002DA60BBE7983D0020E8
:100CC00070B4EFF31186502383F31288436B1A68D4
:100CD000D20720D45D686DB9446A826A944217D005
:100CE00081691144D9600ED9A21A5A608462002227
:100CF00080F858201A6842F00102F1B21A6081F3BC
:100D0000118870BC704701698A1A5A608562EEE7E3
:100D1000012380F85830F3B283F3118870BC704718
:100D200003685B6A03B11847704700BF03681B6A1A
:100D300003B11847704700BF03682DE9F041DF6930
:100D40001FB13B46BDE8F0411847002A164611DDA9
:100D500004460D460E4400E023689B6820469847F1
:100D60000028F9D0236815F8011B1B682046984716
:100D7000AE42F1D1BDE8F08103689B69184700BF1E
:100D800003685B69184700BF03681B69184700BF09
:100D90000368DB68184700BF03689B68184700BFFB
:100DA00003685B68184700BF03681B68184700BFEB
:100DB00038B50C46097849B1054601342B682846F8
:100DC0001B68984714F8011B0029F7D138BD00BFF4
:100DD000064B53F820302BB11A689B8851690B429F
:100DE00001D1138370475383704700BFF085002003
:100DF000026802F13F4303F57E032DE9F04F9B0AA1
:100E0000544DEB5C03F01F055B090124032B04FA2E
:100E100005F400F09980042B00F09180022B3ED065
:100E200001F00306731E012BC1F3810CC1F30018FE
:100E30008588C1F3411137D90024234601274FF09B
:100E4000030E03E0102B04F1020426D007FA03F08E
:100E5000A84303F10103F5D1D2F800C00EFA04F063
:100E6000C04300EA0C0CC2F800C0D2F8008006FAB9
:100E700004FC4CEA080CC2F800C0D2F80CC000EA2E
:100E80000C00D060D2F80CC001FA04F040EA0C006B
:100E9000102BD06004F10204D8D1BDE8F08F2E4BA6
:100EA0005D6C2C435C64BBE7002003464FF0010EF1
:100EB0004FF0030904E00133102B00F102003CD095
:100EC0000EFA03F737EA0504F5D1D2F800A009FAC3
:100ED00000F4E4430AEA040AC2F800A0D2F800B021
:100EE00006FA00FA4AEA0B0AC2F800A0D2F808A0F3
:100EF00004EA0A0AC2F808A0D2F808B00CFA00FA0C
:100F00004AEA0B0AC2F808A0D2F804A02AEA0707A6
:100F10005760D2F804A008FA03F747EA0A075760B7
:100F2000D7683C40D460D76801FA00F401333C43F1
:100F3000102BD46000F10200C2D1BDE8F08F064B47
:100F40001D6B2C431C636BE7034B1D6C2C431C6413
:100F500066E700BF10010408003802402DE9F04F99
:100F60004A484B494B4B4C4C4FF0010A4FF0020999
:100F70004FF004084FF0080C4FF0100E20274026C9
:100F8000802530F8022B12F0010F03D01960A3F86E
:100F900004A0083312F0020F03D01960A3F80490E4
:100FA000083312F0040F03D01960A3F8048008334B
:100FB00012F0080F03D01960A3F804C0083312F030
:100FC000100F03D01960A3F804E0083312F0200FCB
:100FD00002D019609F80083312F0400F02D01960D0
:100FE0009E80083312F0800F02D019609D80083374
:100FF00012F4807F05D04FF4807B1960A3F804B011
:10100000083312F4007F05D04FF4007B1960A3F879
:1010100004B0083312F4806F05D04FF4806B196070
:10102000A3F804B0083312F4006F05D04FF4006B3E
:101030001960A3F804B0083312F4805F05D04FF4B0
:10104000805B1960A3F804B0083312F4005F05D088
:101050004FF4005B1960A3F804B0083312F4804F1A
:1010600005D04FF4804B1960A3F804B00833D20BBD
:1010700004D04FF4004219609A80083301F5806172
:10108000A1427FF47EAFBDE8F08F00BFCC00040822
:1010900000000240D883002000100240002855D0F4
:1010A000026802F13F4303F57E032DE9F04F9B0AEE
:1010B000544DEB5C03F01F055B090124032B04FA7C
:1010C00005F444D0042B00F09780022B44D001F0AB
:1010D0000306731E012BC1F3810CC1F30018858830
:1010E000C1F341113DD90024234601274FF0030EDF
:1010F00003E0102B04F1020426D007FA03F0A84302
:1011000003F10103F5D1D2F800C00EFA04F0C04398
:1011100000EA0C0CC2F800C0D2F8008006FA04FC09
:101120004CEA080CC2F800C0D2F80CC000EA0C006F
:10113000D060D2F80CC001FA04F040EA0C00102B89
:10114000D06004F10204D8D1BDE8F08F70472E4B77
:101150001D6C2C431C64BAE72B4B5D6C2C435C6408
:10116000B5E7002003464FF0010E4FF0030904E0FD
:101170000133102B00F102003CD00EFA03F737EADE
:101180000504F5D1D2F800A009FA00F4E4430AEA14
:10119000040AC2F800A0D2F800B006FA00FA4AEA3F
:1011A0000B0AC2F800A0D2F808A004EA0A0AC2F8A2
:1011B00008A0D2F808B00CFA00FA4AEA0B0AC2F802
:1011C00008A0D2F804A02AEA07075760D2F804A0C2
:1011D00008FA03F747EA0A075760D7683C40D4602B
:1011E000D76801FA00F401333C43102BD46000F1BE
:1011F0000200C2D1BDE8F08F034B1D6B2C431C6372
:1012000065E700BF100104080038024010B1036810
:1012100082885A83704700BF10B1036882881A839E
:10122000704700BF18B10368828809B95A837047B4
:101230001A8370470E4B1B8801463BB90D4B0E4A73
:101240001B7810680BB981F00101EBE70B4B5A6971
:101250001AB118B91A68106058747047084A1868AB
:101260001188084A92FBF1F201210260597470471B
:10127000FC850020FE8500200086002004860020DA
:101280001C86002020A1070010B40A4B0A4A1C78D3
:1012900001238340234052F8200029B9B3FA83F197
:1012A00049095DF8044BBDE7191C18BF01215DF821
:1012B000044BB7E7EE850020F085002030B10368CD
:1012C00082881B691A4214BF01200020704700BFAA
:1012D0002DE9F04F2DED0A8B444B1B7895B0012B77
:1012E000089001F0F585424C94F80021002A41F065
:1012F0002D80072B3F4D01F0E685002304936B689A
:101300003C489847002800F0CE80B5F8B430002162
:1013100085F85510002B41F02682EB6CB5F9407032
:10132000B5F93CE0686AB5F93E60A96ADFF8D0B06B
:10133000A7EB030C8CEAEC72A2EBEC72B2F5804FD7
:10134000EA6AD8BFEF64AEEB0000D8BF3B46711A23
:101350009B1A28636963284895F85610AB6316F00A
:1013600059F9DBF80030990040F10B87D5ED0D5AA3
:10137000D5ED0C7A214A94ED676AD4ED686A94ED54
:10138000697AD4F8A8311268B8EEE58AD5ED0E5A1C
:10139000F8EEE77AF8EEE58A013377EE867A38EEF2
:1013A000268A78EE878A9342C4ED677A84ED688A4C
:1013B000C4ED698AC4F8A83102F0D7800B4B93F8CA
:1013C0000080B8F1140F03F0BF810023D4F8B0718E
:1013D0000593062F00F2C886DFE817F0DE14C81464
:1013E00065148B1630061A16A11500BF6C7100200B
:1013F00090270020F07B0020207C00203863002014
:10140000A8760020D34EDFF8BC93DFF8BCA306F229
:10141000DC680027D04BD5ED087A1B78172B01F03C
:101420009E8096ED007AB8EEC78A082B28EE278AB0
:1014300007D1B0EE480A059329F062FF059B2AF810
:101440001700DBF8002092000BD5002F04F0E18597
:10145000B0EE480AD5F8783708F170009847B0EE3A
:10146000408AB0EE480AD5F89836A8F1700098473F
:10147000D5F8083740469847B74B1B78032BB0EE9A
:10148000408A01F07980D6F85C06D5F8B830B0EE25
:10149000480A98470137032F08F12408A9EC010AEC
:1014A00006F10406B6D1AC4B1F78072F01F0188265
:1014B00094F8C031002B40F09286A84B5B79002B4A
:1014C00040F0A4850123A44A84F8C0311278072A89
:1014D00002F0368000230B93A14B94ED729A93EDAA
:1014E000007AA04BDFF8E482D3F800A09E4B05936E
:1014F000F7EE007A37EEC9BA9C4B07932BEE07BA8A
:101500009B4B09939B4B0693B4EEE7BA08F1680333
:101510000025F1EE10FA0A93D4ED71BA964BDFF87C
:10152000B0B2DFED968A9FED96AADFED96AADFEDC9
:10153000969ADFF8A092954F049388BFB0EE67BAF1
:101540002E46934B98ED008A2B44D3ED007AF5EEAE
:10155000407AF1EE10FA17D08E4B2B44D3ED006A8F
:1015600038EE667AB0EEC76AF4EEC67AF1EE10FA9B
:1015700008D5B5EEC07AF1EE10FACCBF37EEA68AE8
:1015800036EEE78A83ED008A059B1A8893073FD0E1
:10159000022E3DD0804B9AF82E1033F9163007EE0C
:1015A000103A0A9B07EE901A2B44F8EEE76AB8EE61
:1015B000C77AD3ED007A4B42A6EEA77A700007EE09
:1015C000903AF8EEE77AB4EEE77AF1EE10FA0AD440
:1015D00007EE901AF8EE677AF4EEC77AF1EE10FA99
:1015E00088BFF0EE477A6D4B6D490344085EB3F94E
:1015F0000C30C01A07EE100AB8EEC77AD007E7EE33
:10160000687A40F1F485674B93ED008A27EE888A6B
:10161000069B94F8D8212B44D3ED01CA38EE6CCA4E
:10162000002A3DD0604BD4F8DC2108991B688A1A47
:101630009A4235DD9AF84830022B02F09280022E51
:1016400004F07584594B1B68990740F16F87534B21
:101650005349DFF850E131F916C09EED008ADFF8FA
:1016600078E1C7ED00AA03EB460028EE288AB0F91E
:101670000C00A0EB0C0007EE900AF8EEE77ADEF81B
:10168000000027EE888A904238EE6CCAC1F23E8292
:10169000F7EE007AB4EEE79AF1EE10FA01F10D825E
:1016A000434B2B4493ED000A049B2BEE800A022E41
:1016B00020EE0C0AA3EC010A049304F05284079B69
:1016C0009BED007AD3ED007A3A4BD7ED006A93EDAB
:1016D000006A394B67EE277A2B4427EE8B7AD3EDDD
:1016E000007A67EE277AF0EE665AE7EE8C5AB1EE92
:1016F000467AB4EEE57AF1EE10FA08DCF4EEC65A5A
:10170000F1EE10FA8CBFB0EE467AB0EE657A94ED49
:10171000726AF7EE007AB4EEE76AF1EE10FAACBF47
:101720000123002343B1F0EEE66AF0EEC77AF4EE4F
:10173000E67AF1EE10FA01D587ED007A022E04F078
:10174000DB831E4A1E4B52F826001B68B0EE6C0A63
:1017500044E000BF207C00206C71002084760020D3
:1017600060440020B868002098680020980000209D
:10177000DC7100209876002070620020CDCCCC3D3A
:10178000AE47813F000000000000C8427C6200209C
:10179000544400205C2900202029002050620020B1
:1017A000908800203C44002068440020AC88002041
:1017B00010440020844400201C440020BC3F002032
:1017C000B83F00209C7600207071002094280020F3
:1017D000B43F002088620020644400209847CB4A30
:1017E000CB4B52F826001B6898479AF8373023B144
:1017F000059B1B88002B00F06485B0EE6A8AC54B00
:101800009BED007A38EE400A2B4493ED008A83ED7D
:10181000000A9AF8483030EE480AC0EE077A2BB337
:10182000099B1B78DB0721D5B7EE007AB4EEC79A87
:10183000F1EE10FA04DB94F8D831002B00F04A875F
:10184000D4F8DC31089AD31AB34A12689A420DDDF3
:10185000B24B93ED007AB0EECCCAB4EEC7CAF1EE4B
:1018600010FA41F16F81002384F8D831AC4B94F821
:10187000E8212B4493ED007A2BEE877A67EE277AE6
:10188000C9ED007A32B9049BC7ED00AA43ED01AA65
:10189000C9ED00AA0136032E08F1040809F1040974
:1018A00007F1040705F104057FF44BAE9D4B1B784F
:1018B000072B01F05C83012B01F04786002794F889
:1018C000F031002B40F0FC85974A984B10681B685C
:1018D00010F4805A93F82C3040F05486944A95497D
:1018E00092ED006A498B944A84ED806A92ED007A09
:1018F000924A84ED817A07EE901AF8EEE76AD2ED0B
:10190000037A8F4A84ED7E6A37EE467A77EEE67A7E
:10191000D2ED006A84ED7D7A012284F80822C7EEB8
:10192000A65A8849884A91ED005A88499FED886AED
:1019300091ED004A8749DFED886AD1ED004A92EDCA
:10194000007A35EE045AF7EE007AF4EEE75A35EEF7
:10195000245AF1EE10FA88BFF0EE675A25EE065AC7
:10196000F4EEE65AB1EE476AF1EE10FAB4EEC65A5A
:10197000B8BFF0EE665AF1EE10FAC4ED835A01F1E9
:10198000F080B4EEC75AF1EE10FA88BFB0EE475AB5
:101990006C4ADFED6F6AD2ED017A6C4A92ED014A32
:1019A0006C4A77EE847AD2ED014A77EEA47A67EE3C
:1019B000A67AB4EEE76AF1EE10FA08DCB4EEE77A44
:1019C000F1EE10FA8CBFB0EE676AB0EE476A5D4A7E
:1019D000DFED5F6AD2ED027A5C4AD2ED024A5F4ADD
:1019E00077EEA47A92ED007A67EEA67AB1EE473AE6
:1019F000F4EEC37AF1EE10FA08D4F4EEC77AF1EE01
:101A000010FA8CBFB0EE473AB0EE673A544A5278BB
:101A10000AB9B1EE433A002B41F0C883F7EE003A21
:101A2000504D2A78002A02F044864F4BDFED4A7A67
:101A3000D3ED024AD3ED016A93ED037A66EE244AB0
:101A4000E5EE264AE3EE074A63EEA44AF4EEE74ADF
:101A5000F1EE10FAB4BFB0EE674AB0EE644A98BF38
:101A6000F0EE647A012ACDED0C4A02F0838693ED04
:101A7000067AD3ED052AD3ED076A26EE077AA5EE9E
:101A8000227AA3EE267A23EE877AB4EEE77AF1EE95
:101A900010FAB4EEC47A8CBFF0EE676AF0EE476AD3
:101AA000F1EE10FA88BFF0EE676AB4BFF0EE447A48
:101AB000F0EE477A022A8DED0D7A00F00F8193ED5A
:101AC0000A7AD3ED092A93ED0B4A26EE077AA5EEA2
:101AD000227AA3EE047A23EE877AB4EEE67AF1EE68
:101AE00010FAB4EEE77A8CBFB0EE664AB0EE474A21
:101AF000F1EE10FA98BFF0EE446AA8BFF0EE477A14
:101B0000032A8DED0E7A00F0E9802FE010400020CE
:101B10000C400020702900206844002074440020FC
:101B2000284400206C710020A8760020B8680020AE
:101B300080AF0020147800203462002068720020FA
:101B40004445002070620020884400207C62002010
:101B50006F12833A88620020000000008C4400204D
:101B6000D06200204D710020B444002093ED0E7A25
:101B7000D3ED0D2A93ED0F4A26EE077AA5EE227AD1
:101B8000A3EE047A23EE877AB4EEE67AF1EE10FA49
:101B9000B4EEE77A8CBFB0EE664AB0EE474AF1EE9B
:101BA00010FA98BFF0EE446AA8BFF0EE477A042A14
:101BB0008DED0F7A00F0928093ED124AD3ED112A49
:101BC00093ED137A26EE044AA5EE224AA3EE074AC5
:101BD00023EE844AB4EEE64AF1EE10FAB4EEE74A98
:101BE0008CBFB0EE667AB0EE447AF1EE10FA98BF90
:101BF000F0EE476AA8BFF0EE447A052A8DED104A50
:101C00006CD093ED164AD3ED152A93ED177A26EE94
:101C1000044AA5EE224AA3EE074A23EE844AB4EE14
:101C2000E64AF1EE10FAB4EEE74A8CBFB0EE667AFF
:101C3000B0EE447AF1EE10FA98BFF0EE476AA8BF12
:101C4000F0EE447A062A8DED114A47D093ED1A4AF8
:101C5000D3ED192A93ED1B7A26EE044AA5EE224A0B
:101C6000A3EE074A23EE844AB4EEE64AF1EE10FAF8
:101C7000B4EEE74A8CBFB0EE667AB0EE447AF1EE8D
:101C800010FA98BFF0EE476AA8BFF0EE447A072A30
:101C90008DED124A22D093ED1E7AD3ED1D2A93EDDD
:101CA0001F4A26EE077AA5EE227AA4EE037A27EEE3
:101CB000237AB4EEE67AF1EE10FAB4EEE77A8CBF4E
:101CC000B0EE666AB0EE476AF1EE10FA8DED137A67
:101CD00098BFF0EE466AA8BFF0EE477A77EEE67A54
:101CE000F7EE006AF4EEE67AF1EE10FAC4ED727ADD
:101CF00043F3298686EEA77A022ADDED0D7A67EE98
:101D0000244A67EE877ACDED0C4ACDED0D7A2DD0C1
:101D1000DDED0E7A67EE877A032ACDED0E7A25D0B7
:101D2000DDED0F7A67EE877A042ACDED0F7A1DD0AC
:101D3000DDED107A67EE877A052ACDED107A15D0A1
:101D4000DDED117A67EE877A062ACDED117A0DD096
:101D5000DDED127A67EE877A072ACDED127A05D08B
:101D6000DDED137A27EE877A8DED137AAA4B1E6884
:101D700016F0805601F0C280F6EE005AC4ED835A88
:101D8000002A02F08B84A54BD4ED814A93F803809E
:101D900094F908320999D4ED806A91F800E0DFF8EF
:101DA0008CC29F49DFF88892B1F906109CED007A49
:101DB000049106EE103AFDEEE44A9A4B99F8009031
:101DC000B3F81AB094ED7D5AD4ED7E7A14EE903AC1
:101DD000FDEEE64A00F0100C00F480000EF0010E5B
:101DE000B8EEC66A14EE901A0590B8F1000F41F0F3
:101DF0001F82DFF84082BCF1000F41F0CB8098EDEC
:101E0000007ADDED0C6ADFF830C225EE877AA6EEA7
:101E1000267AF0EE676AE5EE076ABDEEE67A17EE1F
:101E2000106A17EE100A9E42A8BF1846B142C8BFFA
:101E3000084607EE100AB8EEC77A012A8CED007A40
:101E400000F0DC8098ED047ADDED0D6A25EE877AEE
:101E5000A6EE267AF0EE676AE5EE076ABDEEE67A50
:101E600017EE106A17EE100A9E42A8BF1846B1423C
:101E7000C8BF084607EE100AB8EEC77A022A8CEDF2
:101E8000017A00F0BB8098ED087ADDED0E6A25EE50
:101E9000877AA6EE267AF0EE676AE5EE076ABDEE6F
:101EA000E67A17EE106A17EE100A9E42A8BF18468F
:101EB000B142C8BF084607EE100AB8EEC77A032A37
:101EC0008CED027A00F09A8098ED0C7ADDED0F6AC5
:101ED00025EE877AA6EE267AF0EE676AE5EE076AC7
:101EE000BDEEE67A17EE106A17EE100A9E42A8BF02
:101EF0001846B142C8BF084607EE100AB8EEC77AC6
:101F0000042A8CED037A79D098ED107ADDED106A11
:101F100025EE877AA6EE267AF0EE676AE5EE076A86
:101F2000BDEEE67A17EE106A17EE100A9E42A8BFC1
:101F30001846B142C8BF084607EE100AB8EEC77A85
:101F4000052A8CED047A59D098ED147ADDED116AEA
:101F500025EE877AA6EE267AF0EE676AE7EE056A46
:101F6000BDEEE67A17EE106A17EE100A9E42A8BF81
:101F70001846B142C8BF084607EE100AB8EEC77A45
:101F8000062A8CED057A39D098ED187ADDED126AC3
:101F900025EE877AA6EE867AF0EE676AE7EE056AA6
:101FA000BDEEE67A17EE106A17EE100A9E42A8BF41
:101FB0001846B142C8BF084607EE100AB8EEC77A05
:101FC000072A8CED067A19D098ED1C7ADDED136A9C
:101FD00065EE875AE6EE265AE5EE257AFDEEE77ABB
:101FE00017EE900A8342A8BF03468142C8BF0B4642
:101FF00007EE903AF8EEE77ACCED077ABEF1000FE3
:1020000040F06B82002A40F0638266E2064B1B7848
:10201000013BDBB2FFF757BACC790020EC6100201E
:102020009879002014780020446200209044002019
:1020300078730020B4440020A4620020AE4B1A78CC
:10204000D4F8B4E1AD4E9FEDAE7A4FEACE0033182E
:1020500083ED007A002A7CD0AA49B0EE476AF0EE00
:10206000476A0023F1EC017A013367EEA77A05EEA7
:10207000903AB4EEE77AF1EE10FAF8EEE55AB8BF0E
:10208000B0EE677A934276EEA76AA7EEA56AE9D129
:10209000F5EEC06A3318F1EE10FA83ED007A58DDE0
:1020A000C6EE265A984B994A1288B7EE000AD3ED2D
:1020B000007A75EEC05A65EEA77AFDEEE77A17EE64
:1020C000903A812B42F376849342A8BF134607EEE1
:1020D000903AF8EEE77A8E4B00EB0E0103EB8103AA
:1020E00093ED057AD3ED003A93ED066A93ED014A3C
:1020F000D3ED046AD3ED034A93ED025AA3EEA77A17
:10210000A4EE276A66EEC76AA7EE646ABDEEC77AD8
:10211000E5EE276A17EE101A812983ED056AC3EDF3
:10212000066A42F34B848A42A8BF0A4607EE902A09
:10213000F8EEE77AFCEEE77ACDED067ABDF81830D6
:1021400032189380BEF1000F03D1B8F1130F03F0E2
:102150000284B8F1150F41F0FB8530446D4E838841
:1021600026F81E30D4F8B0716B4B013783FB072380
:10217000DA19FB17C3EBA203C3EBC303FF1AC4F8BE
:10218000B071664B1B78002B7FF43CA9644FDFF8DD
:10219000B89107F24C7607F5F768F7EC017A95ED00
:1021A000080AD5F87837F8EEE77A304627EE800A45
:1021B0009847A6F1E000D5F898369847A6F1700048
:1021C000D5F808379847D7F85806D5F8B830984763
:1021D0002436B045A9EC010ADFD1FFF764B9013B11
:1021E00084F8C03115B0BDEC0A8BBDE8F08F94EDDA
:1021F0005E7AB1F90000D4ED5F6AB1F902E0494AB4
:10220000F4EEC76A80EAE0738EEAEE71A3EBE07346
:10221000F1EE10FAA1EBEE71B4BFB0EE476AB0EE8A
:10222000666A8B42B8BF0B4607EE103A1378B8EED9
:10223000C77A27EE287A002B40F0E7813A4BD3ED9E
:10224000005AF4EECA5AF1EE10FA41F10D81B7EEE0
:10225000005A75EE654ADFED356A9FED355A354B0C
:1022600036EEC77A24EE855AD3ED006AE7EE055ABA
:1022700065EEA65AF5EEC05AF1EE10FA40F23A8633
:10228000C9EEA56AB7EE007AF0EE475AE6EE665A56
:10229000F0EE656AF4EEC76AF1EE10FA88BFF0EE70
:1022A000476AF5EEC06AF1EE10FAB8BFF0EE6A6A5E
:1022B000214B93ED007A67EE877AA7EEA68AFFF7A7
:1022C000A7B91E4B1E4A2B4493ED007AD2ED007A3B
:1022D0001C4B67EE277AF7EE006AF4EEE67AF1EE31
:1022E00010FA93ED007A88BFF0EE667A67EE877A8F
:1022F00027EE888AFFF783BA3E6300205C650020E2
:102300000000000090270020406300203C63002074
:10231000746500207071002093244992316300207D
:10232000207C00204844002050440020000034431A
:10233000610BB63B444400204044002008290020A3
:1023400038440020344400209C760020072B02F003
:102350000C820027DFF874B3C34DDBF800305E0554
:1023600001F1E480C14B1B78002B40F0DE81DFF8E7
:102370003C9394F8126126B1BD4B1B88980742F03C
:10238000508194F81821002A41F0738099F81E308A
:10239000002B00F0FF83022B01F07C87032B01F060
:1023A0005583B44B598899F81F300233DBB2002AA9
:1023B00001F06187002901F05E87AF480068B1FB3A
:1023C000F0F10FFA81F8A4F84881002B03F0CF82D6
:1023D00007EE908AF8EEE77AF7EE006A86EEA77AC3
:1023E000A649012BD4ED576AD1ED007A77EEE67A53
:1023F00067EE877AC4ED537A21D0D1ED017AD4ED1E
:10240000586A77EEE67A022B67EE877AC4ED547A43
:1024100015D0D1ED027AD4ED596A77EEE67A032B26
:1024200067EE877AC4ED557A09D0D1ED037AD4ED01
:102430005A6A77EEE67A67EE877AC4ED567A904864
:102440000078092803F0C382B8F1000F40F3A98394
:1024500093B394ED577AD4ED537A77EE877A012BC4
:10246000C4ED577AC1ED007A21D094ED587AD4EDBD
:10247000547A77EE877A022BC4ED587AC1ED017A4F
:1024800015D094ED597AD4ED557A77EE877A032BEF
:10249000C4ED597AC1ED027A09D0D4ED5A7A94ED9F
:1024A000567A77EE877AC4ED5A7AC1ED037A013B0A
:1024B000022BB8BF0223DBB2002A18BF022371E34C
:1024C000099B704D1B78DE0700F128822A7822B123
:1024D00092006D496D4828F00BFD6D4B1B68002B79
:1024E00040F043836B4B1B789BB1287870B1DFF8C9
:1024F0009C81DFF8DC910026F0B2D9F80030B8EC0E
:10250000010A9847287801368642F5DB624B1B6842
:1025100098475B4B1B78072B00F02285012384F83A
:10252000003115B0BDEC0A8BBDE8F08F5B4BC7EDF9
:1025300000AA1B689342BFF6ABA8594B1A88002328
:1025400084F8D831002A41F07D86564A564B1178DE
:10255000186881F00101FEF765FEFFF7A1B896ED5E
:10256000007A05EB4702B8EEC78A928F2AF8172047
:1025700028EE278AFEF765BF28F0C2FE2AF817006A
:10258000FEF781BF099A1278D50703D4474A128B08
:10259000A4F8FC21464A3949128891ED037A07EEE6
:1025A000902AF8EEE77AB4EEE77AF1EE10FA41F20B
:1025B00065814049098807EE901AF8EEE77AB4EE93
:1025C000E77AF1EE10FAC1F2A3803B493B4AD1ED24
:1025D000006A92ED006A3A49C4ED806ABCEEC75ABF
:1025E00076EE665A15EE102AC4ED7E6AC4ED7D5A69
:1025F00084ED816AA4F8FC210122D1ED006A84F8FF
:10260000082277EE677AFFF78AB92E4B93ED005ACE
:10261000B5EEC05AF1EE10FA40F36C842A4BD3EDBC
:10262000006AF5EEC06AF1EE10FA40F3638436EE0C
:10263000C77A66EE695A87EE266AC5EE856AB7EEF6
:10264000007AB4EEC76AF1EE10FA88BFB0EE476ABE
:10265000B5EEC06AF1EE10FA76EE876AB8BFB0EE5A
:102660006A6A66EE266A15E6F07B0020E622002004
:1026700098680020A0470020C862002068720020EF
:102680006C7100204D71002094440020A462002051
:10269000846C002080760020747300206444002045
:1026A000FC850020FE850020008600201478002094
:1026B000484500204A45002034450020346200206F
:1026C00050450020444400204C440020A8760020BF
:1026D0006C730020864A92ED007AF0EEE76AF4EE21
:1026E000C76AF1EE10FA7FF7ABA8824A92ED007A42
:1026F000F0EECC6AF4EEC76AF1EE10FA7FF7A0A80C
:102700007D4A98ED007AD2ED006AB0EEC77AB4EE59
:10271000E67AF1EE10FA7FF593A801220899C4F841
:10272000DC1184F8D821FFF78FB8744BDFF8E891FB
:10273000B3F90620B9F81A309A423FF71AAE704B37
:102740001B78012B01F08885192B01F085850E2B54
:102750003FF40FAE082B3FF40CAE6A4900238B60A8
:10276000C4F80C3105E6684A06924FF47A7E126886
:10277000BEFBF2F2C2EB421802EB88024FEAC2083B
:102780006248634E634F90F801903F78B6F90600B7
:102790001FFA88F8434502F01481D5F888E0B5F9AE
:1027A0003CC0EA6E0EF1010107EE90CA62440129B5
:1027B000C5F88810EA66F8EEE77A02F00D81D5EDEB
:1027C0001E5AD5ED206A07EE101A37EEE56AB8EE0C
:1027D000C75A012B86EE057A37EE257A77EEC77A4F
:1027E00085ED1F7AE7EE866A85ED1E7AF0EE667A51
:1027F000C5ED216AC5ED206A02F0C586D5F89CE0DA
:10280000B5F93EC02A6F0EF1010107EE90CA62448D
:102810000129C5F89C102A67F8EEE77A02F0F580E6
:10282000D5ED235AD5ED256A07EE101A37EEE56A85
:10283000B8EEC75A012B86EE057A37EE257A77EE89
:10284000C77A85ED247AE7EE866A85ED237AF0EE85
:10285000667AC5ED266AC5ED256A02F0BE86D5F812
:10286000B0E0B5F940C06A6F0EF1010107EE90CA01
:1028700062440129C5F8B0106A67F8EEE77A02F001
:10288000DD80D5ED285AD5ED2A6A07EE101A37EE0D
:10289000E56AB8EEC75A012B86EE057A37EE257A3F
:1028A00077EEC77A85ED297AE6EE276A85ED287AF4
:1028B000F0EE667AC5ED2B6AC5ED2A6A02F05686FF
:1028C000F080B5F8B430134A013B1778A5F8B4305E
:1028D00006990023072F4B608B60CB607EF4E8AD38
:1028E000FDF758FF049B0A4EC01A3080FEF7E0BD8A
:1028F00078440020744400207C4400209879002013
:10290000D062002068720020987600208476002033
:10291000707100206C710020147800202B78002B3F
:102920003FF4DBADD4ED5F3A94ED5E4AD4ED7E7AB0
:102930008F4A94ED7D7A92ED005AD4ED5C5A94ED75
:102940005B6ADFF84882DFF848C2F4EEC43AF3EE7F
:10295000046AF1EE10FA77EEA64A00F1C88798ED06
:10296000026A26EE656AB0EE674AA6EE074AB4EE42
:10297000E44A34EE666AF1EE10FA48BFB0EE456AFA
:10298000012B8CED006A3FF4A8AD98ED066A26EEA7
:10299000656AB0EE674AA6EE074AF4EEC44A34EE22
:1029A000666AF1EE10FA88BFB0EE456A022B8CED34
:1029B000016A3FF492AD98ED0A6A26EE656AB0EEC0
:1029C000674AA6EE074AB4EEE44A34EE666AF1EED0
:1029D00010FA48BFB0EE456A032B8CED026A3FF453
:1029E0007CAD98ED0E6A26EE656AB0EE674AA6EEFB
:1029F000074AF4EEC44A34EE666AF1EE10FAC8BF34
:102A0000B0EE456A042B8CED036A3FF466AD98ED99
:102A1000126A26EE656AB0EE674AA6EE074AF4EE41
:102A2000C44A34EE666AF1EE10FAC8BFB0EE456AE9
:102A3000052B8CED046A3FF450AD98ED166A26EE36
:102A4000656AB0EE674AA6EE074AB4EEE44A74EE51
:102A5000666AF1EE10FAB8BFF0EE456A062BCCEDCF
:102A6000056A3FF43AADD8ED1A6A66EEE56AB0EE53
:102A7000674AA6EE874AB3EE046AF4EEC44A74EEDF
:102A8000466AF1EE10FAC8BFF0EE456A072BCCEDAE
:102A9000066A3FF422ADD8ED1E6A66EEE55AE5EE11
:102AA000877AF4EEE74A77EEC67AF1EE10FAC8BFFD
:102AB000F0EE457ACCED077A0FE506992D4BD1ED76
:102AC000017A93ED007AF0EEE77AF4EEC77AF1EE50
:102AD00010FA7EF5E5ADD1ED027AF0EEE77AB4EECC
:102AE000E77AF1EE10FA7EF7DBADD1ED037AF0EE86
:102AF000E77AB4EEE77AF1EE10FA7EF7D1AD1E4B2D
:102B00001B689A077FF519AD1C491D4BB3F90C20C2
:102B1000B1F900E01B48AEEB020E00688EEAEE72DF
:102B2000A2EBEE728242BEF6BBADB3F90E30B1F944
:102B30000220D21A82EAE273A3EBE27398427EF794
:102B4000AFADFAE4104B98ED007AD3ED006AB0EE29
:102B5000C77AB4EEE67AF1EE10FA7EF787AEFEF7AA
:102B600082BEB0EE465AFEF713BF17F015FCB9E46B
:102B70009044002070440020AC8800209088002001
:102B8000506200206C4400207C440020B4440020AB
:102B9000A4620020A4F848319846002A00F072810F
:102BA000D9490223D94ADFEDDA6A1068D94A90F888
:102BB00002E092F800C0027807EE902AF8EEE77A79
:102BC000B0EE007A67EEA67AF4EEC77AF1EE10FA6C
:102BD00040F31D8337EEC77ADFEDCF6AB0EE676A48
:102BE000A7EE266AB0EE467A9FEDCC6AD1ED006A78
:102BF00066EE866AB0EEE66AC4ED5B6A84ED5E6AF4
:102C0000BEF1000F13D005EE90EAB8EEE55ADFED05
:102C1000C05A66EEA64A25EE255AF7EE005A75EE22
:102C2000C55A64EE864AE4EE855A66EEA56ADFED83
:102C3000BC5A427927EE257A27EE267ACAB1DFED13
:102C4000B46ADFEDB85A26EE266A06EE902AF8EE50
:102C5000E66A26EE266AB4EEE56AF1EE10FA00F3B3
:102C60003486F7EE005A35EEC66AC5EE866A27EE60
:102C7000267ABCF10C0F9FEDAC8ADFEDAC6A00F058
:102C8000D985B4EEC87AF1EE10FA98BFB0EE478A53
:102C9000B4EEE68AF1EE10FAB8BFB0EE668A84EDC3
:102CA000418A002B00F0E280B0EE007AF4EEC77AA1
:102CB000F1EE10FA05DD37EEC77ADFED976AE7EE41
:102CC000267A91ED017ADFED956A27EE267AB0EE4D
:102CD000C76A84ED5C7A84ED5F6ABEF1000F13D0A1
:102CE00006EE90EADFED8A5AF8EEE66A27EE075A1A
:102CF00066EEA56AF7EE005A75EEE65A25EE065A1C
:102D0000E5EE265A27EE257ADFED856A827967EEB1
:102D1000A67A67EE877AAAB107EE102AB8EEC77ACC
:102D2000DFED7B5ADFED7F6A27EE067A27EE257A04
:102D3000B4EEE67AF1EE10FA40F3CB85DFED7C6A73
:102D400067EEA67ABCF10C0F00F02485DFED766A01
:102D50009FED767AF4EEE67AF1EE10FA88BFF0EEA7
:102D6000667AF4EEC77AF1EE10FAB8BFF0EE477A61
:102D7000012BC4ED427A79DD4378DFED656A07EE19
:102D8000903AF8EEE77AB0EE007A67EEA67A437AE8
:102D9000F4EEC77AF1EE10FA05DD37EEC77ADFED13
:102DA0005E6AE7EE267A91ED027ADFED5C6A27EE45
:102DB000267AB0EEC76A84ED5D7A84ED606A9BB1D5
:102DC00006EE903ADFED525AF8EEE66A27EE075A21
:102DD00066EEA56AF7EE005A75EEE65A25EE065A3B
:102DE000E6EE855A27EE257ADFED4D6AC37967EE68
:102DF000A67A67EE877A0BB307EE103AB8EEC77A79
:102E0000DFED435ADFED476A27EE067A27EE257A93
:102E1000B4EEE67AF1EE10FA0CDCB5EEC07AF1EE23
:102E200010FA01F12482B7EE006A36EE477AC6EE58
:102E3000076A01E0DFED3E6A67EEA67ABCF10C0F8F
:102E400000F0A084DFED386A9FED387AF4EEE67A80
:102E5000F1EE10FA88BFF0EE667AF4EEC77AF1EE82
:102E600010FAB8BFF0EE477AC4ED437ABCF1090F0F
:102E700000F06D8499F82160002E40F00384002357
:102E800084F818312B4B1B68990609D52A4B1B88EF
:102E900003F0300323B1294B1B78DA0702F13F809E
:102EA000274B1B7823B9274EB378002B41F0F981CB
:102EB000184B1B78072B00F0D8840022072B84F8CE
:102EC00000217EF41AAAFDF765FC0490FEF717BAFC
:102ED0001D4B1E4C1A681E4B1E4E94F80001D26901
:102EE0001B883280738000287FF433AA04901A4D27
:102EF000FEF705BADFED196AFFF7DAB941023EF5D0
:102F00003BAFFEF73DBF00BF68720020ECB0002071
:102F10000AD7233C6C710020D7A368416F12033B92
:102F200000004843A4707D3F00C0F94400C0F9C4CC
:102F30000000C842AC88002098680020B0880020BB
:102F4000905D002088790020AC7B00209027002035
:102F5000264A002070710020F07B00200000000055
:102F6000FDF718FCAB4BC01BD880FFF7D7BAFDF7B5
:102F700011FCA94B0B9A1B78A64E801A012B70806E
:102F800000F0E482072B7EF499ACFDF703FC0746C2
:102F9000FEF795BCBEF1000F41F0FE8398ED007A7C
:102FA000DDED0C6ADFF884C225EE877AA6EE867A1C
:102FB000F0EE676AE7EE056ABDEEE67A17EE106A94
:102FC00017EE100A9E42A8BF1846B142C8BF084675
:102FD00007EE100AB8EEC77A012A8CED007A3FF4AA
:102FE00077AA98ED047ADDED0D6A25EE877AA6EED4
:102FF000867AF0EE676AE7EE056ABDEEE67A17EECE
:10300000106A17EE100A9E42A8BF1846B142C8BF08
:10301000084607EE100AB8EEC77A022A8CED017A4C
:103020003FF456AA98ED087ADDED0E6A25EE877A10
:10303000A6EE867AF0EE676AE7EE056ABDEEE67AFE
:1030400017EE106A17EE100A9E42A8BF1846B1424A
:10305000C8BF084607EE100AB8EEC77A032A8CEDFF
:10306000027A3FF435AA98ED0C7ADDED0F6A25EE71
:10307000877AA6EE867AF0EE676AE7EE056ABDEE1D
:10308000E67A17EE106A17EE100A9E42A8BF18469D
:10309000B142C8BF084607EE100AB8EEC77A042A44
:1030A0008CED037A3FF414AA98ED107ADDED106AE6
:1030B00025EE877AA6EE867AF0EE676AE7EE056A75
:1030C000BDEEE67A17EE106A17EE100A9E42A8BF10
:1030D0001846B142C8BF084607EE100AB8EEC77AD4
:1030E000052A8CED047A3FF4F3A998ED147ADDED0E
:1030F000116A25EE877AA6EE867AF0EE676AE7EE29
:10310000056ABDEEE67A17EE106A17EE100A9E42C7
:10311000A8BF1846B142C8BF084607EE100AB8EE6D
:10312000C77A062A8CED057A3FF4D2A998ED187A71
:10313000DDED126A25EE877AA6EE867AF0EE676AF2
:10314000E7EE056ABDEEE67A17EE106A17EE100A92
:103150009E42A8BF1846B142C8BF084607EE100AF3
:10316000B8EEC77A072A8CED067A3FF4B1A998ED3C
:103170001C7ADDED136A65EE875AE6EE265AE5EE17
:10318000257AFDEEE77A17EE900A8342A8BF034640
:103190008142C8BF0B4607EE903AF8EEE77ACCEDD5
:1031A000077A002A7FF494A9FFF797B91B4B5A7945
:1031B000002A3EF433AC1A4A1278002A3EF42EACB0
:1031C0001B78DFED184A07EE903A174BB8EE677A96
:1031D0001B8807EE902A06EE903AF8EEE77AF8EEB2
:1031E000666A67EE277AB7EE007AC7EEA63AF4EE83
:1031F000E43AF1EE10FA88BFF0EE643AF4EEC73A22
:10320000F1EE10FAB8BFF0EE473AFEF709BCB0EEA7
:10321000677AE9E4707100206C71002098880020C2
:1032200066720020713DAA3F50720020A462002007
:10323000BCF1000F00F02284BEF1000F42F05F806D
:10324000DFF8E485B9F1000F41F00087D8ED006A9E
:10325000DDED0C4ADFF8D4C565EEA66ABDEEC77A8F
:1032600017EE101AB0EE667AA4EE867AF0EE676A70
:10327000E7EE056ABDEEE67A17EE106A17EE100A61
:103280009E42A8BF1846B142C8BF084607EE100AC2
:10329000B8EEC77A012A8CED007A3FF419A998EDAF
:1032A000047ADDED0D6A25EE877AA6EE867AF0EED9
:1032B000676AE7EE056ABDEEE67A17EE106A17EE6A
:1032C000100A9E42A8BF18468E42B8BF084607EEB5
:1032D000100AB8EEC77A022A8CED017A3FF4F8A8FA
:1032E00098ED087ADDED0E6A25EE877AA6EE867AED
:1032F000F0EE676AE7EE056ABDEEE67A17EE106A51
:1033000017EE100A9E42A8BF18468E42B8BF084664
:1033100007EE100AB8EEC77A032A8CED027A3FF462
:10332000D7A898ED0C7ADDED0F6A25EE877AA6EE28
:10333000867AF0EE676AE7EE056ABDEEE67A17EE8A
:10334000106A17EE100A9E42A8BF18468E42B8BFF8
:10335000084607EE100AB8EEC77A042A8CED037A05
:103360003FF4B6A898ED107ADDED106A25EE877A65
:10337000A6EE867AF0EE676AE7EE056ABDEEE67ABB
:1033800017EE106A17EE100A9E42A8BF18468E422A
:10339000B8BF084607EE100AB8EEC77A052A8CEDCA
:1033A000047A3FF495A898ED147ADDED116A25EEC4
:1033B000877AA6EE867AF0EE676AE7EE056ABDEEDA
:1033C000E67A17EE106A17EE100A9E42A8BF18465A
:1033D0008E42B8BF084607EE100AB8EEC77A062A32
:1033E0008CED057A3FF474A898ED187ADDED126A39
:1033F00025EE877AA6EE867AF0EE676AE7EE056A32
:10340000BDEEE67A17EE106A17EE100A9E42A8BFCC
:1034100018468E42B8BF084607EE100AB8EEC77AC3
:10342000072A8CED067A3FF453A898ED1C7ADDED5F
:10343000136A65EE875AE6EE265AE5EE257AFDEE2A
:10344000E77A17EE900A8342A8BF03468142D8BFAD
:10345000194607EE901AF8EEE77ACCED077A002AC3
:103460007FF436A8FFF739B8DA4BD3ED005AFEF7F0
:1034700001BFD94BD949D3F8EC30096844F6206034
:103480008342A8BF0346B3F57A7FB8BF4FF47A737F
:1034900098B2C906A4F81A01DBF8003041F1858220
:1034A000DB0400F19286CE4BD3F800E0BEF9326027
:1034B000CC49DFF87CC3D1ED037AD4F81C31ACFBE6
:1034C00000108009642191FBF0F11429BDEEE77A28
:1034D00004EB430CA8BF142101338B42C4F81C3108
:1034E00017EE108AA4BF0023C4F81C3104EB430379
:1034F000ACF82081B3F9203107EE103AB8EEC77A64
:1035000077EEC77AFDEEE77ACDED047ABDF91010BB
:1035100081EAE173A3EBE173B34202F30582B24B9C
:1035200019464FF07E530B60FEF730BFAB68002B9F
:103530003EF418AF05F1500128469847FEF712BF38
:10354000FDF728F90B90FDF7C7BFA84EFDF722F94C
:10355000A74AD4F8EC311268C4F8EC01C31A9A1ADD
:103560000746B380F280FEF7AAB907EE103AA14BE6
:103570009E4E1B78B6F9040095ED080AB4F8AC81AC
:10358000B8EEC77AF7EE006A0022132B86EE879A10
:10359000C4F8A82101F0F983974B984A02EB8807F9
:1035A0000021C4F89C11C4F8A01167EE897A93ED4C
:1035B000001A93ED053A93ED122A93ED176AD3EDB5
:1035C000091A93ED0E4AD3ED015AD3ED063A93ED65
:1035D0000A7A93ED0F5AD3ED132AD3ED186AD3ED7F
:1035E000044AD3ED030A69EE288A29EE088AA1EE7F
:1035F000273AA2EE286AA1EE884AE5EEA73AA7EE9E
:10360000085A93ED167AD3ED0D5A93ED021AD3EDC5
:103610000C1A87ED003AE2EEA86A64EEC34A27EE80
:10362000467A93ED0B2AD3ED152A87ED204AE0EE7A
:10363000C33A65EEC45A93ED143AC3ED053AE1EE90
:10364000274AF0EE477AA1EEC45AE2EE085AE2EEBB
:10365000C66AE3EE287AC3ED064A83ED0E5AC3ED3F
:103660000F5A87ED406AC3ED176AC3ED187AC4F8A4
:10367000A41108F1010303F01F03A4F8AC31B080DA
:10368000FDF79CBE1E215548F6F7FBFB00283FF4D2
:10369000F6AB5B4B1B8858063FF5F1AB94F88431D1
:1036A000B34242F0F981504BD4ED627AD3ED016A16
:1036B00094ED435ADFED535A9FED536A27EEC57AD6
:1036C00068EE277AA8EE267AE5EE267AB4EEE57A59
:1036D000F1EE10FA88BFB0EE657AB4EEC67AF1EE7C
:1036E00010FAF4EEE57AB8BFB0EE467AF1EE10FAD1
:1036F00088BFF0EE657AF4EEC67AF1EE10FAB8BF44
:10370000F0EE467A84ED417AC4ED437AFFF7B7BB19
:10371000B4F8FC11914240F264853C493C4AD1ED39
:10372000007A92ED007A3B49C4ED807A77EE676AC1
:10373000C4ED7E7A0122C4ED7D6A84ED817AD1EDFB
:10374000006ADFED357A84F80822FEF7E8B8FDEE6E
:10375000C87A264E17EE903AA6F80480F380FFF759
:1037600089BB2E4B1B88002B40F05A852C4A2D4BD1
:1037700011781868FDF756FDD4F8DC21089B9A1AD9
:10378000FDF75DBFBDEEE77A184E17EE103AB38035
:10379000FFF758BB9FED1B7ADFED1B6A134EF4EE6B
:1037A000C77AF1EE10FA98BFB0EE677AFDEEE77ACD
:1037B000B4EEE67AF1EE10FA17EE902AB8BFB0EE4A
:1037C000667A012B84ED427A72803FF7D5AAFFF723
:1037D00051BB00BF44440020681C0020CC7900206D
:1037E000B8680020687200209800002070710020E6
:1037F000C86200206C710020E06500205C6300203E
:103800009868002000C0F94400C0F9C43445002085
:10381000346200205045002000000000FC8500209C
:10382000FE85002000860020B4440020A462002011
:10383000D34D6210B4EEC87AF1EE10FA98BFB0EE34
:10384000478ABDEEC77AB4EEE68A854EF1EE10FAED
:1038500017EE102AB8BFB0EE668A84ED418A328036
:10386000002B7FF421AAFFF705BBFCF793FF7C4EEA
:103870007C4BC01B1B78B080FFF71FBB7A4A7B498B
:10388000D2ED006A7A4A91ED006A1278C4ED806A3E
:1038900084ED816A002A40F0A08476EEC65AF0EEEC
:1038A000466ABCEEC76A7349C4ED7D5A16EE102A0B
:1038B000C4ED7E6AA4F8FC21FF22D1ED006A84F8F1
:1038C000082277EEC77AFEF72AB8DFED6B6AFFF7BA
:1038D000CEB9B5EEC07AF1EE10FA00F1C484B7EEBD
:1038E000006A36EE477AC6EE076AFFF729BAD8EDC6
:1038F000015A65EEC65AB0EE674AA5EE874AF4EE65
:10390000C44A74EE665AF1EE10FAC8BFF0EE455A9A
:10391000012BCCED005A3EF4E0ADD8ED055A65EE32
:10392000C65AB0EE674AA5EE874AF4EEC44A74EE72
:10393000665AF1EE10FAC8BFF0EE455A022BCCEDF4
:10394000015A3EF4CAADD8ED095A65EEC65AB0EE3A
:10395000674AA5EE874AF4EEC44A74EE665AF1EE61
:1039600010FAC8BFF0EE455A032BCCED025A3EF4D4
:10397000B4ADD8ED0D5A65EEC65AB0EE674AA5EE65
:10398000874AF4EEC44A74EE665AF1EE10FAC8BFE4
:10399000F0EE455A042BCCED035A3EF49EADD8ED23
:1039A000115A65EEC65AB0EE674AA5EE874AF4EEA4
:1039B000C44A74EE665AF1EE10FAC8BFF0EE455AEA
:1039C000052BCCED045A3EF488ADD8ED155A65EEC2
:1039D000C65AB0EE674AA5EE874AF4EEC44A74EEC2
:1039E000666AF1EE10FAC8BFF0EE456A062BCCED20
:1039F000056A3EF472ADD8ED196A66EEC66AB0EE9D
:103A0000674AA6EE874AF3EE045AF4EEC44A74EE0F
:103A1000656AF1EE10FAC8BFF0EE456A072BCCEDEF
:103A2000066A3EF45AADD8ED1D6A26EEC66AE6EE89
:103A3000077AF4EEE47A77EEE57AF1EE10FAB8BFA1
:103A4000F0EE457ACCED077AFEF747BD99F82030C5
:103A5000C3EB431103EB8101C90089B2FEF7A3BC9C
:103A6000707100206C71002080AF0020384500206C
:103A7000787300204C4500200000C842DFF88485A0
:103A8000B9F1000F41F04280D8ED006ADDED0C4A3B
:103A9000DFF874C565EEA66ABDEEC77A17EE101A98
:103AA000B0EE667AA4EE867AF0EE676AE7EE056A13
:103AB000BDEEE67A17EE106A17EE100A9E42A8BF16
:103AC0001846B142C8BF084607EE100AB8EEC77ADA
:103AD000012A8CED007A3EF491AA98ED047ADDED8E
:103AE0000D6A25EE877AA6EE867AF0EE676AE7EE33
:103AF000056ABDEEE67A17EE106A17EE100A9E42CE
:103B0000A8BF18468E42B8BF084607EE100AB8EEA6
:103B1000C77A022A8CED017A3EF470AA98ED087AF1
:103B2000DDED0E6A25EE877AA6EE867AF0EE676AFC
:103B3000E7EE056ABDEEE67A17EE106A17EE100A98
:103B40009E42A8BF18468E42B8BF084607EE100A2C
:103B5000B8EEC77A032A8CED027A3EF44FAA98EDAC
:103B60000C7ADDED0F6A25EE877AA6EE867AF0EE06
:103B7000676AE7EE056ABDEEE67A17EE106A17EEA1
:103B8000100A9E42A8BF18468E42B8BF084607EEEC
:103B9000100AB8EEC77A042A8CED037A3EF42EAAF6
:103BA00098ED107ADDED106A25EE877AA6EE867A1A
:103BB000F0EE676AE7EE056ABDEEE67A17EE106A88
:103BC00017EE100A9E42A8BF18468E42B8BF08469C
:103BD00007EE100AB8EEC77A052A8CED047A3EF497
:103BE0000DAA98ED147ADDED116A25EE877AA6EE1E
:103BF000867AF0EE676AE7EE056ABDEEE67A17EEC2
:103C0000106A17EE100A9E42A8BF18468E42B8BF2F
:103C1000084607EE100AB8EEC77A062A8CED057A38
:103C20003EF4ECA998ED187ADDED126A25EE877A5C
:103C3000A6EE867AF0EE676AE7EE056ABDEEE67AF2
:103C400017EE106A17EE100A9E42A8BF18468E4261
:103C5000B8BF084607EE100AB8EEC77A072A8CEDFF
:103C6000067A3EF4CBA998ED1C7ADDED136A65EE79
:103C7000875AE6EE265AE5EE257AFDEEE77A17EE4C
:103C8000900A8342A8BF03468142D8BF194607EE77
:103C9000901AF8EEE77ACCED077ABEF1000F7EF4C9
:103CA0001CACFEF7AFB9DFF86493D4ED017A94ED64
:103CB000006AB9F80000D9F8143077EEA77AF0EE70
:103CC000006AB0EE677AA6EE267A013804EBC002ED
:103CD000D6EE267A083A1033F6EE003A27EE237A2B
:103CE00067EEA37A84ED207AC4ED217ABE4C264695
:103CF00004F1800192ED027A92ED036AD6ED036A37
:103D0000D6ED027A53ED014A13ED025A37EE674AB7
:103D100076EEC65A77EE277AE4EE845A0138A2F19D
:103D20000802E5EE047A06F1080603F1080336EE10
:103D3000267A01F10801E4EE877AE5EE475A67EE4C
:103D4000A37A25EEA37AC1ED007A81ED017AD1D173
:103D5000B8F1140F7EF408AAFCF71CFD059BA34ED6
:103D6000C01A7080D4F8B071FEF7FEB9DFF89C92EB
:103D70009D48D9F80820B9F80C1026F01BF99C4B87
:103D800093F80080B8F1140F01F06F86D4F8B07189
:103D90000137C4F8B07188E7DFF87092B9F80070A5
:103DA000D9F804E04FEA570C4FEA8C0204EB87087D
:103DB000FF0804EB020300F09F80103201378D48AA
:103DC00003EB0717424410330EF1100608F11001FF
:103DD00051ED032A51ED043A10ED043A10ED032A97
:103DE00051ED026A11ED016A10ED020A10ED018A2F
:103DF00012ED044A12ED035A53ED044A53ED035AEF
:103E000013ED027A53ED017A52ED020A12ED011A16
:103E100073EE238A72EE221A40ED048A40ED031AF3
:103E200070EE268A78EE061A40ED028A40ED011AFD
:103E300074EE848A75EE851A43ED048A43ED031A05
:103E400077EE208A77EE811A43ED028A43ED011A5C
:103E500073EE633A75EE655A16ED035A32EE623A26
:103E600074EE644A65EE631A16ED044A23EE052AE1
:103E700064EE652AE3EE041A10339F4224EE843A7E
:103E8000A3EE842A00F1100006F11006A5EE853A93
:103E900001F1100102F11002E4EE852A41ED071A4A
:103EA00001ED082A02ED073A42ED082A56ED055ABF
:103EB00016ED065A70EE666A38EE466A30EEC77A3C
:103EC00071EE677A26EE253A65EEE63A25EE674A08
:103ED00067EE054AE6EE053AA6EE853AA7EE254AD4
:103EE000E7EEA54A01ED063A41ED053A02ED064A34
:103EF00042ED054A7FF46CAF1FFA8CF672463146EC
:103F0000394822F0FFF93146D9F80420404622F022
:103F1000F9F9374B1B78142B7FF424AF1CE7D4F846
:103F2000B4C1B4F8ACA1344BCAF120095FFA89F9E5
:103F30000AEB4C165FEA990003EB860601F01A853E
:103F4000013000012D492B4A06EB000E06F110034B
:103F500013ED024A13ED035A13ED016A13ED047ACF
:103F600051ED024A51ED035A51ED016A51ED047AC7
:103F700064EE244A65EE255A66EE266A67EE277AD5
:103F800010339E4542ED024A42ED035A42ED016A6A
:103F900042ED047A01F1100102F11002D8D1184A61
:103FA000103806441118204419F0030309D0B6EC68
:103FB000017AF1EC017A67EE277A013BE0EC017AB5
:103FC000F5D1BAF1000F40F05587B8F1140F7EF427
:103FD000CBA8FCF7DFFB059B044ED4F8B071C01AE8
:103FE0007080FEF7C1B800BF9027002070710020DC
:103FF0006C710020A02700205C630020EC6400208E
:10400000DC640020B4440020A4620020446300204B
:10401000D4F8B491D24BD34ADFEDD37AD2ED008AF3
:10402000D24E4FEAC9010B44F8EE688A9B8809EE2C
:10403000103A643BC82BA8BFC82368EEA78AF8EEE5
:10404000497A782BB8BF782368EEA78A07EE903AB2
:104050004944B0EE680A06EB8106B8EEE78A27F01D
:104060009BF9B8EEC99AF0EE409AB0EE680A27F0D4
:10407000F5F838EE097A79EE487A28EE098A67EE83
:10408000877AB7EE006A88EE277AB8F1140FF8EE57
:10409000007A77EE076A60EE277A89EEA67A77EEE5
:1040A000065A36EE477AC6EE256A67EEA67A27EEFE
:1040B000267AC6ED006A86ED047AC6ED026AC6ED80
:1040C000017AC6ED037A01F0DB84A94BA94A09F114
:1040D000010983FB093CACEBE97C0CEB4C0C013790
:1040E000A9EB0C0C92F80080C4F8B071C4F8B4C10C
:1040F00017E7DFF8BC9299F80020900801F0A4853A
:10410000DFF8B0E200F1010C4FEA4C1C0EEB0C069C
:104110000EF12003AEF1700113ED076A53ED056A4D
:1041200013ED037A53ED017A53ED025A13ED084A69
:1041300053ED064A13ED045A26EE066A66EEA66AA9
:1041400027EE077A67EEA77AA4EE046A20339E4230
:10415000E4EEA46A01F11001A5EE057AE5EEA57A78
:10416000F1EEC65AB1EEE66AF1EEC76AB1EEE77A51
:1041700041ED085A01ED076A41ED066A01ED057A45
:10418000CAD1ACF1200CE64404EB001012F003039A
:1041900018BF0EF1080E0FD05EED017A1EED027A07
:1041A00067EEA77A013BE7EE077A0EF1080EB1EE53
:1041B000E77AA0EC017AEFD1B8F1140F01F0468450
:1041C0000137C4F8B071FDF73BBF6B4BD3F800E08B
:1041D000BEF832607608FFF76BB976EE665AFFF7E5
:1041E00060BB664A6649D2ED007A664A91ED007A74
:1041F0001278C4ED807A84ED817A002A01F08E83F2
:1042000077EE676A6049C4ED7E7AC4ED7D6AFF226D
:10421000D1ED006ADFED5D7A84F80822FDF77FBBFF
:104220005B494B69002B3DF40AAA5A485A4B008857
:1042300093FBF0F00B684FF0010E186081F811E06D
:10424000FDF7FDB952494A69002A3DF429AA0A68D6
:1042500013604B74FDF724BA504B9B7B002B3EF44C
:104260007CAAFEF786B8F7EE006AFEF769BDF7EEA6
:10427000006AFEF7E1BDB4F8488108F1FF380FFA93
:1042800088F8B8F1000FA4F848817EF786AC44495D
:10429000FEF7DEB8B4F81A1101F57A7189B2FEF7AB
:1042A00082B8DFF8148198F80020013A0D2A18D856
:1042B000DFE812F09C01AB01580136011D0100013D
:1042C000EA00E100BC00A5009000840092010E000D
:1042D0001F20049325F0F4FA049B10B9012288F8FA
:1042E0000020012B00F0F587F278002A3EF4E0ADC3
:1042F0002C4A1278D00706D4049309F003FB049BE0
:10430000002841F07E84284ED4F8981132689142FA
:1043100001F27E8498F80030012B3EF4C9AD94F888
:104320009421002A3EF4C4AD0B2B0DD801229A40F3
:1043300040F6030112EA01090CD112F4C06F03D058
:10434000093B012B41F28A86184B32685A600B23D5
:1043500088F80030002384F89431FEF7A9BD00BF2F
:104360005C6500209876002027D4D2366C8300202C
:10437000565555556C710020B868002080AF00205C
:1043800038450020787300204C45002000000000D4
:10439000048600201C86002020A10700A88F002092
:1043A00068720020DC710020248600203862002022
:1043B0003E63002010280020136F0020012B01D144
:1043C000F5F73CFF0D23132088F800301DF0E6F8C8
:1043D000B37886E7C74AC84952680968C8328A4232
:1043E00005D326F04BFDB37800283FF47AAF032BBA
:1043F00001F0F385012388F80030B37871E7BF4BF3
:104400001B78002B01F06F841A2025F059FA002840
:1044100041F0698494F89431002B41F064840923BD
:1044200088F8003011F0C4FEB3785AE71A2025F05E
:1044300047FA0028F6D0B24B1B88002BF2D1B14BC3
:104440004520D3F8009024F0E1FC0E2024F0DEFC9F
:10445000484624F0A5FDDDF82090484624F0A0FD54
:10446000A94AAA4B12681A6048460A2388F8003005
:1044700024F056FED6E724F019FC11F0D3FE0028F4
:1044800041F02785B3782CE724F010FCA04B0021E5
:1044900005208DE80300A3F108020291532012F0D9
:1044A0006FFB0028EED1934AB3781060082288F899
:1044B000002016E724F0FAFB964A0292A2F10C03C0
:1044C0004FF007090193CDF80090A2F108030021F5
:1044D000143A472012F054FB0028D3D1854B88F8BA
:1044E00000904FF0FF3283E80500B378F9E624F03E
:1044F000DDFB894B002102208DE80300A3F10802B7
:104500000291482012F03CFB0028BBD1794AB378D5
:1045100010604FF0FF315160062288F80020E0E67D
:1045200024F0C4FB7D4A0292A2F10C0325210193E1
:104530000091A2F10A035021163A492012F020FB03
:1045400000289FD1DBF8002012F0800201F0DB840C
:10455000684AB37810604FF0FF315160052288F847
:104560000020BEE6DFF88C9124F0A0FB624AD9F867
:10457000043012686433934284D2402024F06EFBEE
:1045800000287FF47FAFD9F80030DFF8B8A1644984
:104590004FF0400B0FE0049124F038FC0499D9F857
:1045A00000300A680133013ABBF1010B0A60C9F817
:1045B000003001F087851AF803301846002BEAD145
:1045C00000234FF0FF32C9F80030042388F8003090
:1045D000C9F80420B37884E6012B01F069840E2326
:1045E000132088F800301CF0D9FF4BE74D4B1B78A7
:1045F000DB0701F164841F2025F062F900283FF4F5
:1046000041AF0C2388F800303CE73B4A3949126837
:104610004A60434800220A600321026088F80010C3
:104620005FE6414BDFED417A93ED080AB4EEE70A0D
:10463000F1EE10FA40F2498626F0F8FED4ED457A04
:1046400020EE270A26F05CFEB0F5617F00F3EF87CD
:1046500007EE900AF8EEE76ADFED357A66EEA76AB4
:1046600007EE906AB8EEE77AFDEEE67A17EE903A3A
:104670002033402B41F2F3829FED2E0A26F040FEBC
:1046800000B207EE900AB8EEE77A2B49D1ED037A33
:1046900077EE877AC1ED037AFDF773BE099B93F835
:1046A00000E00EF0010EBEF1000F7DF416AFFDF735
:1046B000A9BC224BDFED227A1E68C4ED727A16F097
:1046C000805640F0A38410F4800600F01582002686
:1046D000B6EE007A67EE877AF4EEE75AF1EE10FA5A
:1046E00048BFF0EE675A40F19184C4ED835AFDF75C
:1046F00047BB00BF386200202486002024630020CE
:1047000058AF002054AF002068AF002060AF0020F9
:1047100040DE0308F8DD0308DCDD03082EDC0308B7
:10472000C4AE0020DC710020183E00208FC2753C12
:10473000D06D393A0000000068720020CC7900206A
:1047400000000080C8DB0308FCF724F8E14B05906B
:1047500093F80080B8F1140F05BFDF4ED4F8B071A4
:10476000D4F8B0713780FCF734BEFCF713F8074675
:10477000FDF7F0BD74EE677AB7EE007AF4EEC77A13
:10478000F1EE10FAC4ED727A41F3DD8084EEA77A7F
:104790008DED0C7AFDF7EABABAF1000F00F0A887A8
:1047A00098ED007ADDED0C6ADFF848C325EE877AD4
:1047B000A6EE867AF0EE676AE7EE056ABDEEE67A67
:1047C00017EE106A17EE100A9E42A8BF1846B142B3
:1047D000C8BF084607EE100AB8EEC77A012A8CED6A
:1047E000007A3DF47AAE98ED047ADDED0D6A25EE9F
:1047F000877AA6EE867AF0EE676AE7EE056ABDEE86
:10480000E67A17EE106A17EE100A9E42A8BF184605
:10481000B142C8BF084607EE100AB8EEC77A022AAE
:104820008CED017A3DF459AE98ED087ADDED0E6A13
:1048300025EE877AA6EE867AF0EE676AE7EE056ADD
:10484000BDEEE67A17EE106A17EE100A9E42A8BF78
:104850001846B142C8BF084607EE100AB8EEC77A3C
:10486000032A8CED027A3DF438AE98ED0C7ADDED3A
:104870000F6A25EE877AA6EE867AF0EE676AE7EE93
:10488000056ABDEEE67A17EE106A17EE100A9E4230
:10489000A8BF1846B142C8BF084607EE100AB8EED6
:1048A000C77A042A8CED037A3DF417AE98ED107A9E
:1048B000DDED106A25EE877AA6EE867AF0EE676A5D
:1048C000E7EE056ABDEEE67A17EE106A17EE100AFB
:1048D0009E42A8BF1846B142C8BF084607EE100A5C
:1048E000B8EEC77A052A8CED047A3DF4F6AD98ED62
:1048F000147ADDED116A25EE877AA6EE867AF0EE5F
:10490000676AE7EE056ABDEEE67A17EE106A17EE03
:10491000100A9E42A8BF1846B142C8BF084607EE1B
:10492000100AB8EEC77A062A8CED057A3DF4D5ADAB
:1049300098ED187ADDED126A25EE877AA6EE867A72
:10494000F0EE676AE7EE056ABDEEE67A17EE106AEA
:1049500017EE100A9E42A8BF1846B142C8BF0846CB
:1049600007EE100AB8EEC77A072A8CED067A3DF4F6
:10497000B4AD98ED1C7ADDED136A65EE875AE6EE6C
:10498000265AE5EE257AFDEEE77A17EE902A934255
:10499000A8BF13468A42A8BF194607EE901AF8EE40
:1049A000E77ACCED077AFDF798BDDE003EF578ADED
:1049B000FDF7ECBCDFED497AFDF78DBB8223FDF7F7
:1049C000BFBBB5F93C20696207EE902A0121F8EEE1
:1049D000E77AEA66C5F888100022012BC5ED1F7A38
:1049E000C5ED1E7AC5F8802001F0338143457DF482
:1049F00005AFB5F93E202A6707EE902A0021012273
:104A0000F8EEE77AA962C5F89C200022012BC5EDDB
:104A1000247AC5ED237AC5F8942001F01D81434521
:104A20007DF41DAFB5F940206A6707EE902A00219A
:104A30000122F8EEE77AE962C5F8B0200022012BE6
:104A4000C5ED297AC5ED287AC5F8A8207DF438AFE0
:104A50009FED238A032F36D0B9F1000F09D007EE5E
:104A6000909AF8EEE77AF4EEC87AF1EE10FA01F1D6
:104A70000E821C4A6B6F1268F08094F8B801002116
:104A800003EB580393FBF8F3EB6291621163D1627D
:104A900030B1154B1B8823F40063002B7DF411AF5C
:104AA000124B1B6813F4003341F0C68010481A46BD
:104AB000C15C012903F10C0300F002860132152AC2
:104AC000F6D1FDF7FEBEB0EE480A26F019FC00B2A2
:104AD000C2E700BF6C71002070710020000002432B
:104AE00000000000AC7B0020D47900208C3E002028
:104AF00038E40308A4620020B6EE007AF4EEC75A48
:104B0000F1EE10FA3FF7E4ADFDF73AB9D8ED004AFF
:104B10009DED0C4ADFF830C565EEA44AFDEEC73ABC
:104B2000E4EE064AB0EE674AA4EE854A13EE901A08
:104B3000F4EEC46AF1EE10FAF0EE444A88BFF0EEEB
:104B4000474AFDEEE44A14EE900A14EE906A984249
:104B5000A8BF1E468142C8BF0E4604EE906AF8EE1A
:104B6000E44A012ACCED004A3DF448AAD8ED044AB3
:104B70009DED0D4A65EEA44AE4EE064AB0EE674AA2
:104B8000A4EE854AF4EEC46AF1EE10FAF0EE444A5F
:104B900088BFF0EE474AFDEEE44A14EE900A14EEA8
:104BA000906A9842A8BF1E468842B8BF0E4604EEDF
:104BB000906AF8EEE44A022ACCED014A3DF41EAABE
:104BC000D8ED084A9DED0E4A65EEA44AE4EE064A89
:104BD000B0EE674AA4EE854AF4EEC46AF1EE10FA2C
:104BE000F0EE444A88BFF0EE474AFDEEE44A14EE88
:104BF000900A14EE906A9842A8BF1E468842B8BF39
:104C00000E4604EE906AF8EEE44A032ACCED024A1E
:104C10003DF4F4A9D8ED0C4A9DED0F4A65EEA44A87
:104C2000E4EE064AB0EE674AA4EE854AF4EEC46AA2
:104C3000F1EE10FAF0EE444A88BFF0EE474AFDEE7E
:104C4000E44A14EE900A14EE906A9842A8BF1E46F9
:104C50008842B8BF0E4604EE906AF8EEE44A042A91
:104C6000CCED034A3DF4CAA9D8ED104A9DED104A97
:104C700065EEA44AE4EE064AB0EE674AA4EE854A21
:104C8000F4EEC46AF1EE10FAF0EE444A88BFF0EE9A
:104C9000474AFDEEE44A14EE900A14EE906A9842F8
:104CA000A8BF1E468842B8BF0E4604EE906AF8EED2
:104CB000E44A052ACCED044A3DF4A0A9D8ED144AF3
:104CC0009DED114A65EEA44AE4EE064AB0EE674A4D
:104CD000A4EE854AF4EEC46AF1EE10FAF0EE444A0E
:104CE00088BFF0EE474AFDEEE44A14EE900A14EE57
:104CF000906A9842A8BF1E468842B8BF0E4604EE8E
:104D0000906AF8EEE44A062ACCED054A3DF476A90D
:104D1000D8ED184A9DED124A65EEA44AE4EE064A23
:104D2000B0EE674AA4EE854AF4EEC46AF1EE10FADA
:104D3000F0EE444A88BFF0EE474AFDEEE44A14EE36
:104D4000900A14EE906A9842A8BF1E468842B8BFE7
:104D50000E4604EE906AF8EEE44A072ACCED064AC5
:104D60003DF44CA9D8ED1C4A9DED134A65EEA45ABA
:104D7000E6EE045AE5EE257AF4EEE76AF1EE10FA73
:104D8000C8BFF0EE477AFEF778BFA74FDFF89C92D6
:104D900097ED004A97ED057AD7ED014A97ED066A3F
:104DA000D7ED046A97ED035AD7ED025A67EE897A78
:104DB00009EB8803A4EE277AA4EEA76A66EEC76A19
:104DC000A5EE476AE5EEA76A20EE070A87ED056AB9
:104DD000C7ED066A83ED007A29EE088A26F090FA7C
:104DE00069EE288AD7ED0E5AD7ED176A97ED091AA2
:104DF000D7ED121A97ED0F5A97ED187A97ED0A2A08
:104E0000D7ED132A97ED0D6AD7ED167A97ED0C3A88
:104E1000D7ED0B3A97ED154AD7ED144AE1EE085A53
:104E2000002209EB8803E8EEA16A00B2C4F89C21D5
:104E3000A2EE085AC4F8A021C4F8A421A8EEA27AD0
:104E400026EE656A67EEE67AA3EE655AA3EE886AF7
:104E5000A6EEC47AE8EEA47A87ED0E5AC3ED205A86
:104E600087ED0F6AC3ED406A87ED177AC7ED187AB0
:104E7000FEF7FFBB6D4B4FEA890603EBCC1C5FEAE4
:104E80009A0302EB060E264400F07B8701334FEABB
:104E900003190CEB09000CF110030EF1100106F1DF
:104EA000100213ED024A13ED035A13ED016A13EDDC
:104EB000047A51ED024A51ED035A51ED016A51ED68
:104EC000047A64EE244A65EE255A66EE266A67EE99
:104ED000277A1033984242ED024A42ED035A42EDDE
:104EE000016A42ED047A01F1100102F11002D8D1F9
:104EF000A9F110039C440EEB03021E441AF0030AAE
:104F00003FF463A8BCEC017AF2EC017A67EE277AF1
:104F1000BAF1010AE6EC017AF4D1FFF756B8444B36
:104F2000444AB3F90430DFED447A82FB0312DB1705
:104F3000C3EBA2031BB208EE103AB8EEC88A28EE03
:104F4000278AB0EE480AF4F7C7FEF0EE408AB0EECA
:104F5000480AF4F747FE394BD878002800F09483CC
:104F60003749B4F98E31B1F9022044F25066D21AB1
:104F7000B24240F30F85A2F50C42A03A4642964257
:104F800000F3FD848242A8BF0246B1F90010B4F9D3
:104F90008CE11344A1EB0E0244F250611BB28A4231
:104FA000A4F88E3140F3EE84A2F50C42A03A96426A
:104FB00003DC9042A8BF104606460EEB060212B272
:104FC00007EE902A07EE103AF8EEE77AF8EEC76A95
:104FD00027EEE87A60EE277AA0EE267AA4F88C21F4
:104FE000E8EEA67ADFED176A27EE267A67EEA67A54
:104FF000BDEEC77AFDEEE77A17EE102A17EE903A6B
:10500000A4F89021A4F89231FDF74ABFB7EE007AD8
:1050100077EE677AF4EEE75AF1EE10FA88BFF0EE19
:10502000675AFFF762BB00BFE06500205C630020A9
:10503000908800206766666635FA8E3C245B002007
:10504000805B0020CDCCCC3DA4620020D8ED004A8E
:105050009DED0C4ADFF828C665EEA44AFDEEC73A7E
:10506000E4EE064AB0EE674AA4EE854A13EE901AC3
:10507000F4EEC46AF1EE10FAF0EE444A88BFF0EEA6
:10508000474AFDEEE44A14EE900A14EE906A984204
:10509000A8BF1E468142C8BF0E4604EE906AF8EED5
:1050A000E44A012ACCED004A3DF412AAD8ED044AA4
:1050B0009DED0D4A65EEA44AE4EE064AB0EE674A5D
:1050C000A4EE854AF4EEC46AF1EE10FAF0EE444A1A
:1050D00088BFF0EE474AFDEEE44A14EE900A14EE63
:1050E000906A9842A8BF1E468842B8BF0E4604EE9A
:1050F000906AF8EEE44A022ACCED014A3DF4E8A9B0
:10510000D8ED084A9DED0E4A65EEA44AE4EE064A43
:10511000B0EE674AA4EE854AF4EEC46AF1EE10FAE6
:10512000F0EE444A88BFF0EE474AFDEEE44A14EE42
:10513000900A14EE906A9842A8BF1E468842B8BFF3
:105140000E4604EE906AF8EEE44A032ACCED024AD9
:105150003DF4BEA9D8ED0C4A9DED0F4A65EEA44A78
:10516000E4EE064AB0EE674AA4EE854AF4EEC46A5D
:10517000F1EE10FAF0EE444A88BFF0EE474AFDEE39
:10518000E44A14EE900A14EE906A9842A8BF1E46B4
:105190008842B8BF0E4604EE906AF8EEE44A042A4C
:1051A000CCED034A3DF494A9D8ED104A9DED104A88
:1051B00065EEA44AE4EE064AB0EE674AA4EE854ADC
:1051C000F4EEC46AF1EE10FAF0EE444A88BFF0EE55
:1051D000474AFDEEE44A14EE900A14EE906A9842B3
:1051E000A8BF1E468842B8BF0E4604EE906AF8EE8D
:1051F000E44A052ACCED044A3DF46AA9D8ED144AE4
:105200009DED114A65EEA44AE4EE064AB0EE674A07
:10521000A4EE854AF4EEC46AF1EE10FAF0EE444AC8
:1052200088BFF0EE474AFDEEE44A14EE900A14EE11
:10523000906A9842A8BF1E468842B8BF0E4604EE48
:10524000906AF8EEE44A062ACCED054A3DF440A9FE
:10525000D8ED184A9DED124A65EEA44AE4EE064ADE
:10526000B0EE674AA4EE854AF4EEC46AF1EE10FA95
:10527000F0EE444A88BFF0EE474AFDEEE44A14EEF1
:10528000900A14EE906A9842A8BF1E468842B8BFA2
:105290000E4604EE906AF8EEE44A072ACCED064A80
:1052A0003DF416A9D8ED1C4A9DED134A65EEA45AAB
:1052B000E6EE045AE5EE257AF4EEE76AF1EE10FA2E
:1052C000C8BFF0EE477AFEF7BAB89FEDE67AFFF76F
:1052D000DCB9E549E54A8968126891423FF604A8BD
:1052E00098F800200C3A022A7DF6E2AD94F8942159
:1052F00088F80030002A3DF4DBADFFF72BB8BAF197
:10530000000F00F03884DFF87C839DED0C4AD8ED67
:10531000004A65EEA44AE4EE064AB0EE674AA4EEFF
:10532000854AF0EE444AB9F1000F06D0F4EE446A23
:10533000F1EE10FAC8BFF0EE474ABDEEC77A17EE9D
:10534000101ABDEEE47A04EE901A17EE100A8142AC
:1053500000F38D859842A8BF184607EE100AB8EEF4
:10536000C77ADFF81CC3012A8CED007A3DF4B5A89A
:1053700098ED047A9DED0D4A25EE877AA4EE067A23
:10538000B0EE674AA7EE054AB0EE447AB9F1000FD5
:1053900000F0EC84F4EEC46AF1EE10FA40F3E68417
:1053A00008469842A8BF184607EE100AB8EEC77A1A
:1053B000022A8CED017A3DF490A898ED087A9DEDD3
:1053C0000E4A25EE877AA4EE067AB0EE674AA7EE7B
:1053D000054AB0EE447AB9F1000F00F0BC84F4EE57
:1053E000C46AF1EE10FA40F3B68408469842A8BFAA
:1053F000184607EE100AB8EEC77A032A8CED027A37
:105400003DF46BA898ED0C7A9DED0F4A25EE877A56
:10541000A4EE067AB0EE674AA7EE054AB0EE447AEB
:10542000B9F1000F00F08C84F4EEC46AF1EE10FACA
:1054300040F3868408469842A8BF184607EE100A33
:10544000B8EEC77A042A8CED037A3DF446A898EDAD
:10545000107A9DED104A25EE877AA4EE067AB0EE1A
:10546000674AA7EE054AB0EE447AB9F1000F00F0A2
:105470005C84F4EEC46AF1EE10FA40F356840846F8
:105480009842A8BF184607EE100AB8EEC77A052A58
:105490008CED047A3DF421A898ED147A9DED114A23
:1054A00025EE877AA4EE067AB0EE674AA7EE054AA3
:1054B000B0EE447AB9F1000F00F02C84F4EEC46A27
:1054C000F1EE10FA40F3268408469842A8BF184629
:1054D00007EE100AB8EEC77A062A8CED057A3CF47E
:1054E000FCAF98ED187A9DED124A25EE877AA4EE6E
:1054F000067AB0EE674AA7EE054AB0EE447AB9F1F3
:10550000000F00F0FD83F4EEC46AF1EE10FA40F3F0
:10551000F78308469842A8BF184607EE100AB8EE6F
:10552000C77A072A8CED067A3CF4D7AF98ED1C7A3F
:105530009DED134A65EE875AE4EE065AE5EE857A4C
:10554000B9F1000F00F0D483F4EEE67AF1EE10FA30
:1055500040F1CE830A469A42A8BF1A4604EE902A2A
:10556000F8EEE44ACCED074AFCF7B7BF01297FF714
:105570006FAA07EE10EAB8EEC77AC7EE876AB1EEF7
:10558000E68AFFF767BA012940F3638307EE10EA62
:10559000B8EEC77AC7EE876AB1EEE68A032F14D059
:1055A000B9F1000F09D007EE909AF8EEE77AF4EE21
:1055B000C87AF1EE10FA00F16A84EA6E02EB580242
:1055C00092FBF8F26A62FFF711BAB0EE480A05934F
:1055D00025F096FE059B00B2E2E7012940F33C83EB
:1055E00007EE10EAB8EEC77AC7EE876AB1EEE68A30
:1055F000032F14D0B9F1000F09D007EE909AF8EEFE
:10560000E77AF4EEC87AF1EE10FA00F140842A6FDE
:1056100002EB580292FBF8F2AA62FFF700BAB0EE72
:10562000480A059325F06CFE059B00B2E2E707EE01
:10563000906ADFED0F6AB8EEE77A66EEA65A9FED44
:105640000D5A9FED0D6ADFED0D7AA5EE856A26EE07
:10565000A55AE5EE867AE5EE276A26EE870AFFF779
:105660000DB800BF00000000D4220020CC62002052
:1056700084F9223F92E741B99730083C15A82ABE29
:10568000A4620020B4440020E24B9FEDE36AB3F92A
:105690000020B3F9023007EE902A06EE903AF8EEB9
:1056A000E77AF8EEE66A27EEE87A60EE277AA0EE6F
:1056B000267AE8EEA67A27EE067A67EE867A97E4EF
:1056C000D4F8BC6153003EB1991800EB81017678A3
:1056D0004978B142BDF4F5A8134400EB83030022DE
:1056E000C4F8BC31A4F81022C4F81422FDF7E9B8BC
:1056F000D8ED006ADDED0C4A65EEA66AE4EE866A36
:10570000F0EE674AE6EE854AFDEEE46A16EE90EAB0
:10571000714500F34A819E45A8BF9E4606EE90EA79
:10572000F8EEE66A002E00F0EA84DFF814C3012ADE
:10573000CCED006A3CF4D1AED8ED046ADDED0D4A43
:1057400065EEA66AE4EE866AF0EE674AE6EE854A02
:10575000FDEEE46A16EE90EA714500F323819E4562
:10576000A8BF9E4606EE90EAF8EEE66A002E00F02C
:105770009E84022ACCED016A3CF4AFAED8ED086AF3
:10578000DDED0E4A65EEA66AE4EE866AF0EE674A43
:10579000E6EE854AFDEEE46A16EE90EA714500F306
:1057A00010819E45A8BF9E4606EE90EAF8EEE66A96
:1057B000002E00F06184032ACCED026A3CF48DAE29
:1057C000D8ED0C6ADDED0F4A65EEA66AE4EE866A56
:1057D000F0EE674AE6EE854AFDEEE46A16EE90EAE0
:1057E000714500F3EB809E45A8BF9E4606EE90EA09
:1057F000F8EEE66A002E00F07784042ACCED036A06
:105800003CF46BAED8ED106ADDED104A65EEA66A89
:10581000E4EE866AF0EE674AE6EE854AFDEEE46A5B
:1058200016EE90EA714500F3C6809E45A8BF9E46DD
:1058300006EE90EAF8EEE66A002E00F04A84052AA9
:10584000CCED046A3CF449AED8ED146ADDED114AA2
:1058500065EEA66AE4EE866AF0EE674AE6EE854AF1
:10586000FDEEE46A16EE90EA714500F3A1809E45D4
:10587000A8BF9E4606EE90EAF8EEE66A002E00F01B
:105880004984062ACCED056A3CF427AED8ED186AA7
:10589000DDED124A65EEA66AE4EE866AF0EE674A2E
:1058A000E6EE854AFDEEE46A16EE90EA714500F3F5
:1058B0008B809E45A8BF9E4606EE90EAF8EEE66A0B
:1058C000002E00F0E483072ACCED066A3CF405AE16
:1058D000D8ED1C6ADDED134A65EEA65AE4EE865A51
:1058E000E5EE857AFDEEE77A17EE902A914203DC29
:1058F0009A42A8BF1A46114607EE901AF8EEE77AC8
:10590000002E7FF44EA8059B002B7FF44AA8049B31
:105910005B45B8BFF0EE477AFFF743B877EEC76A4A
:10592000F0EE477AFEF76EBCBEF834309FED3B7A5E
:1059300007EE903AF8EEE77A394B67EE877AC3EDD7
:10594000007AFCF723BD374B1E6816F080567EF4B4
:10595000BFAEFEF7B8BE9FED340A344E25EE800A86
:1059600025F0CEFCD4F8B071F080FCF7FDBB3049D7
:10597000FCF765BD2F4A30481146FEF715BB32468D
:10598000FFF703BB2D498A42BCBF02F50C42A0328F
:10599000FFF70DBB294EB242BCBF02F50C42A0324C
:1059A000FFF7ECBA06EE901ADEE606EE901AB7E6BE
:1059B00006EE901A60E706EE901A3BE706EE901AA4
:1059C00016E706EE901AF1E606EE901A76E791EDEC
:1059D000000A06930592049125F092FCDFF864E03A
:1059E000DFF864C0DEF8ECE0104E8CFB0E3C4FEAB2
:1059F000EE7ECEEBAC1E07EE90EAF8EEE77A308052
:105A0000FDEEE77A04A917EE900A0EC97080FCF744
:105A10001BBD00BF805B0020CDCCCC3D6F12833A14
:105A200098000020CC7900200000C842707100204E
:105A300068720020DC64002090270020B0B9FFFFCE
:105A4000A4620020681C0020D34D6210FAF7A2FE69
:105A5000DF4BE04E93F80080059B99F80020D4F8C6
:105A6000B071C01AB080FEF7ABBBFAF793FED84B0B
:105A7000D84E93F80080059BC01A7080FEF786B957
:105A8000FAF788FE059BD34ED4F8B491D4F8B071E0
:105A9000C01A7080FEF719BB07EE906A9FEDCE7AB0
:105AA000DFEDD86A84F88461F8EEE77A67EE877AEA
:105AB00037EEA67ABDEEC76A16EE103A2033402BB9
:105AC00040F26581DFEDC56AC54BBDEEE77AC3EDF7
:105AD000016A17EE103A2033402B00F255819FEDFA
:105AE000CA7AF4EEC77AF1EE10FA40F31782DFEDCE
:105AF000BD5A9FEDBD6A01E0F0EE477AF4EEC67A3A
:105B0000F1EE10FA37EEE57AF6DCDFEDC47AB4EEAA
:105B1000E77AF1EE10FA40F15D82DFEDB25A9FEDC7
:105B2000B36A01E0B0EE677AB4EEC67AF1EE10FA2D
:105B300077EE257AF6D49FEDB37AF4EEC77AF1EEDC
:105B400010FA40F398819FEDB07A77EE677A67EEAE
:105B5000A75A9FEDAE5A9FEDAE6A9FEDAE7AA5EEC5
:105B6000856A27EEA55AA5EE867AE5EE077AC4ED9A
:105B7000627AFDF79DBDFDEEC74A0DF1300E9A46E3
:105B8000DFF878C2DFF8788214EE901A0EEB82020A
:105B90004B4606E07245E8EC014A0CF1100C3CF46F
:105BA0009CACDCED004ABEEC014A65EEA44AE6EE90
:105BB000044AB0EE674AA5EE244AF0EE444A33B1F7
:105BC000F4EE446AF1EE10FAC8BFF0EE474AFDEE7B
:105BD000E44A14EE909A494504EE901A04DCD1454B
:105BE000A8BFD14604EE909AF8EEE44A002ED1D137
:105BF00005980028CED104985845B8BFF0EE474A22
:105C0000C8E77B4A126802F59C520832C4F8982112
:105C100098F80020012A7DF44BA994F89421002AD9
:105C20007DF446A9032B00F0ED8124F09DFF0123B4
:105C300084F89431FDF73CB96E4B1B78032B00F0D0
:105C400057810023FEF732BF6B4800F1800EFEF74C
:105C50009DBA9FED628AA1E49FED608AC8E4DFED02
:105C60006A7AF4EEE76AF1EE10FA40F31D82DFED96
:105C70005D5A9FED5D6A01E0F0EE676AF4EEC66A78
:105C8000F1EE10FA76EEE57AF6DCDFED646AF4EE1A
:105C9000E67AF1EE10FA40F10482DFED525A9FED00
:105CA000536A01E0F0EE667AF4EEC67AF1EE10FA8D
:105CB00077EEA56AF6D4DFED537AF4EEE76AF1EEFB
:105CC00010FA04DDDFED507A77EEE66AB5E4DFED39
:105CD000527AF4EEE76AF1EE10FA44BFDFED4F7A44
:105CE00077EEE66AA9E4089823F01AFAFEF79ABB61
:105CF000FDEEE77A17EE902A8A42FFF631AC2AE4ED
:105D0000BDEEC77A17EE100A8842BFF603AC07EE65
:105D1000101A04E4BDEEC77A17EE100A8842BFF6E7
:105D2000D4AB07EE101AFFF7D5BBBDEEC77A17EE5E
:105D3000100A8842BFF6A4AB07EE101AFFF7A5BB06
:105D4000BDEEC77A17EE100A8842BFF674AB07EEB5
:105D5000101AFFF775BBBDEEC77A17EE100A88421E
:105D6000BFF644AB07EE101AFFF745BBBDEEC77A8E
:105D700017EE100A8842BFF614AB07EE101AFFF7B1
:105D800015BB7246FFF7BAB8DFED147AEFE6F4EE12
:105D9000E67AF1EE10FA40F3C780DFED125A9FED7C
:105DA000126A01E0B0EE667AB4EEC67AF1EE10FA4D
:105DB00077EE656AF6DC9FED197AF4EEC76AF1EECC
:105DC00010FA40F1AE80DFED075A9FED086A29E036
:105DD0006C7100207071002035FA8E3C00000000CC
:105DE00098000020DB0FC940E4CB1641E4CB16C17C
:105DF00024860020C879002090270020B444002089
:105E0000A4620020DB0FC93FDB0F494092E741B994
:105E10009730083C15A82ABEDB0FC9BFDB0F49C06D
:105E2000F0EE476AF4EEC66AF1EE10FA36EEA57AA5
:105E3000F6D45FED0C6AB4EEE67AF1EE10FA2BDDE3
:105E40005FED0F6A36EEC77A67EE075A1FED115AFB
:105E50001FED116A5FED116AA5EE856A27EE255ADE
:105E6000E5EE866AA5EE267AF0EE476A2CE607EEA6
:105E7000101AFFF774BA1FED187AF4EEC77AF1EE34
:105E800010FA44BF1FED1B7A77EE677A5FE6F08069
:105E9000A5F8B480FCF71CBD5FED216AB4EEE67A8C
:105EA000F1EE10FA44BF5FED236A36EEC77ACBE716
:105EB000F4F754F800283EF4E5AAFEF790BB8020E2
:105EC00022F0E4F908B104F07FFF24F04DFEFEF764
:105ED00092BB24F0D3FF00283EF4D4AA934A944BFB
:105EE00012681A600A2388F80030B378FEF7F9B90F
:105EF0001BF038FBFCF7E5BC94F8E831002B7BF491
:105F0000D5ACFBF7C0BC8B49B3780A604FF0FF32C9
:105F10004A60072288F80020FEF7E3B9B0EE677AFE
:105F2000F3E5B0EE667A84E7F0EE476A43E7824B2A
:105F3000D3ED007AB1EE677AB4EEC7CAF1EE10FA8B
:105F40005DD4B4EEE7CAF1EE10FA88BFB0EE67CACE
:105F50007A4BC7ED00AA1B689342BBF699ABFCF7DE
:105F6000CEBD774A774B10681B689847079BDBEDDF
:105F7000007A93ED007A744BD7ED006A93ED006AD6
:105F8000724B83ED020A724B67EE277A2B4427EEA1
:105F90008B7AD3ED007A67EE277AF0EE665AECEE54
:105FA000275AB1EE467AB4EEE57AF1EE10FA4BDDFF
:105FB000684B1B78012B02D0192B7BF4A8ABDFEDCB
:105FC000667AB4EEE7CAF1EE10FACCBF01230023E3
:105FD000FBF7A8BBF0EE477AADE5DFF89091D9F872
:105FE00000001AF0B7FB5D4B1B780022022BC9F8AA
:105FF00000207EF4FFA904F0FFFEFEF7FBB9B0EE2F
:1060000047CAA5E7802022F041F900287CF450AF70
:106010000BE6132B05D1B0EE480A25F071F9AAF86A
:106020000000B0EE480AD5F878374D4898474D4BF8
:106030001B78132BB0EE408A7BF413AA25F060F98D
:10604000AAF80200FBF70DBAB4EEE56AF1EE10FA19
:106050008CBFB0EE657AB0EE467AA9E7452022F013
:10606000D5FEFF2022F0D2FE3F4822F043FE4846F4
:1060700022F0CCFEFEF768B9059800287FF49BABB0
:1060800004985845B8BFF0EE476AFFF794BB0598EF
:1060900000287FF418AC04985845B8BFF0EE476A62
:1060A00011E4F0EE676A06E6F0EE667AEDE5059833
:1060B00000287FF45EAB04985845B8BFF0EE476AFD
:1060C000FFF757BB1AF80330002B7EF4DBA9FEF76D
:1060D00077BA059800287FF4B2AB04985845B8BF4A
:1060E000F0EE476AFFF7ABBB059800287FF485AB5D
:1060F00004985845B8BFF0EE476AFFF77EBB059895
:1061000000287FF412AB04985845B8BFF0EE476AF8
:10611000FFF70BBB059800287FF4B3AB04985845F4
:10612000B8BFF0EE476AFFF7ACBB00BF68AF002016
:1061300060AF0020386200208044002064440020CA
:10614000F84300200C4400208444002070620020AA
:106150001C4400201C6B002000009642C4620020FA
:106160006C8300206C710020F8090408C8AE002080
:1061700038B50B4C23688BB15A68821A002A054641
:1061800004DA0CE05A68AA1A002A07DB9A6822602F
:1061900018461A6890472368002BF3D138BD38BDE4
:1061A000744800200D4B04210022890710B40272AC
:1061B00003F1780402D51979815401329C4203F12C
:1061C000180308D0072A06DC99798907F3D49C4282
:1061D00003F11803F6D15DF8044B7047380004084A
:1061E00010B4104C0423214613F001034FF00002B9
:1061F00001F1180108D10132062A0ED08B7913F073
:10620000010301F11801F6D002EB420204EBC202D5
:106210005DF8044B13790370704703705DF8044B0D
:10622000704700BF38000408012332213122417039
:10623000427103700371704723220323027043707D
:10624000704700BF08B506F04FFFF4F7DBFA00BF58
:10625000024A034B127819780DF02EBCC524002099
:10626000C62400202DE9F04F2DED028BA0F10A038A
:1062700089B00C46E72B00F21187DFE813F01C0110
:106280000F070F070F070F070F070F070F070F075E
:106290000F070F070F070F070F070F070F070F074E
:1062A0000F070F070F070F070F070F070F079005BF
:1062B0000F070F070F0780050F070F070F07790557
:1062C0000F0719050F0700050F07F4040F07EC046B
:1062D0000F07C7040F07B3040F070F070F07AD041D
:1062E000A6040F0799040F070F07E6010F07BE0169
:1062F0000F070F070F07A2010F070F070F070F0761
:1063000083010F07FC000F07E60593060F070F0731
:106310000F070F070F070F070F0781030F0753031F
:106320000F071F030F0767020F071E020F070F0754
:106330000F070F07FC02BB02F502ED01E800C203E4
:106340007E0666068F040F0758043C040F070F07EC
:106350000F070F0731040F070F0710040F070F0770
:106360000F070104F70651060E060F070F070F0768
:10637000FE05B7060F0764010F070F070F070F078A
:106380000F070F070F070F070F070F070F070F075D
:106390000F070F070F07FC020F070F070F070F0765
:1063A0000F070F070F070F070F070F070F070F073D
:1063B0000F072D010F070F070F070F070F070F0715
:1063C0000F070F070F070F070F070F070F070F071D
:1063D0000F070F070F070F070F070F070F070F070D
:1063E0000F070F070F070F070F070F070F070F07FD
:1063F0000F070F070F070F070F070F070F070F07ED
:106400000F070F070F070F070F070F070F070F07DC
:106410000F070F070F070F070F070F070F070F07CC
:106420000F070F070F070F070F070F070F070F07BC
:106430000F070F070F070F070F070F070F070F07AC
:106440000F070F070F070F070F07DA05AF05A54E58
:10645000337853B1A44F002537F8021F2046F3F7D5
:10646000CBF933780135AB42F6DC012009B0BDEC45
:10647000028BBDE8F08F9B4E3378002BF5D09B4FFD
:106480000025B846236817F81520591C21601A709A
:1064900098F8011001EB810101EB810101F2EE217D
:1064A00089B22046F3F7A8F933780135AB4208F1F9
:1064B0000208E7DCD9E78E4D284623F0DBFD0028F3
:1064C000D3DD2B460544226813F8011B501C9D4266
:1064D00020601170F7D1C8E70B68DFF868C2591C5B
:1064E0009CF8002021601A709CF80030002BBCD072
:1064F000804E814D814882490023226816F8017F31
:1065000002F1010EC4F800E01770226815F8017F4F
:1065100002F1010EC4F800E01770226810F8017F44
:1065200002F1010EC4F800E01770226811F8017F33
:1065300002F1010EC4F800E017709CF8002001334E
:106540009A42DADC91E70B686E4F591C3A78216069
:106550001A703B78002B88D00025EEB2304618F038
:1065600039FA23684278591C216030461A7018F0B5
:1065700031FA01892046F3F73FF93B780135AB4208
:10658000EBDC72E70B68604D591C2A7921601A70A8
:1065900023686A79591C21601A7029882046F3F70C
:1065A0002BF92368AA79591C21601A706988204642
:1065B000F3F722F92368EA79591C216001201A7047
:1065C00054E7F3F7CBFC2368504D002803F1010199
:1065D0000CBF0222032221601A7029882046F3F79B
:1065E000F4F8A9682046F3F7F0F8F3F78FFC0146BA
:1065F0002046F3F7EAF8012038E70B68444A454D96
:106600001178454A581C2060197011682046F3F72C
:10661000DCF82368414A591C127A21601A702988D3
:106620002046F3F7E9F8A9882046F3F7E5F8298929
:106630002046F3F7E1F800212046F3F7DDF8204685
:106640000021F3F7D9F8012010E708460822334962
:10665000F3F78DF8012009E7314D324E9FED328A74
:10666000DFF8E480DFED318A05F120070EE0FCEE73
:10667000E77ACDED017ABDF8041020460435F3F732
:10668000BBF8AF4206F118063FF4EFAE717C00296B
:10669000F3D0274BD5ED007A1B78012BE7D1254BA2
:1066A0001B68DB0440F1B885F5EE407AF1EE10FA94
:1066B00040F0E58540F2DC51DFE70B681E4A1F49D8
:1066C000D0781F4A5D1C2560187023684979581CD2
:1066D000206019702368D278591C216001201A703B
:1066E000C4E600BFA047002096790020F4490020AE
:1066F000A0680020BB5B0020CB5B0020EB5B002090
:10670000DB5B00204D71002054450020D422002086
:10671000D0620020C03D0020286F002014780020A7
:10672000A4620020947200200000404200E08244F5
:1067300078730020A876002050620020987B00200B
:1067400060620020B95B0020DB9B91410021204664
:10675000F3F752F800212046F3F74EF800212046C7
:10676000F3F74AF82368B94D00265A1C22601E70C0
:1067700023682A68591C92F82C2021601A7023681B
:106780002A68591C92F8362021601A7023682A68FA
:10679000591C92F8372021601A7023685A1C226015
:1067A0001E7023685A1C22601E7023685A1C2260C7
:1067B0001E702B682046598FF3F71EF82B68204671
:1067C000198FF3F719F823682A68591C92F82E20BC
:1067D00021601A7023685A1C22601E702B682046A4
:1067E000598EF3F709F82B682046998EF3F704F8D1
:1067F00001203BE6964B9B8AB3F5006F00F21585AE
:10680000B3F5806F00F23885B3F5007F34BF012700
:106810000227904D05F10C0655F8041B91FBF7F18A
:10682000204689B2F2F7E8FFB542F5D18A4D8B4F89
:1068300005F10C06B5EC010AD7ED087A80EE270ABF
:1068400024F05EFD81B22046F2F7D6FFAE42F1D1D0
:10685000834D05F10C0655F8041B204689B2F2F76A
:10686000CBFFAE42F7D100E6084610227D49F2F791
:106870007EFF0120FAE500258146DFF8FC81DFF884
:10688000FCB1059504950695079501214FF6FF7A11
:1068900005E001350B2D00F0218418F9011F4F1C74
:1068A0004AFA05F3F5D0DE07F3D5BBF800302B41EB
:1068B000D807EED506A8F3F7D5FAEAE76A4E0B68D3
:1068C0007279624D591C21601A702B682046198C10
:1068D000F2F792FF2B682046D98BF2F78DFF718972
:1068E0002046F2F789FFB1892046F2F785FF2B6831
:1068F0002046598CF2F780FF2B682046998CF2F7DE
:106900007BFFF1892046F2F777FF318A2046F2F7C4
:1069100073FF2A68236892F82620591C2160012001
:106920001A70A3E5504EF378002B00F081840B68B9
:106930000822591C21601A702368012299182160CD
:106940001A702368494D591C2A7921601A702368EE
:10695000AA78591C21601A7029882046F2F74CFF4A
:10696000E9892046F2F748FF2368F279591C216033
:106970001A702368EA78591C216001201A7075E5A5
:106980000DF08EF8FF28064600F05F8408A9002568
:1069900001F8125D0DF10D008DF80D500DF060F84D
:1069A00008A800F8115D0DF04FF808A800F8105D78
:1069B0000DF03EF808A820F8085D0DF02DF82368CA
:1069C0005A1C22601E7023689DF80D20591C2160FE
:1069D0001A7023689DF80E20591C21601A702368D4
:1069E0009DF80F20591C21601A7023689DF8102013
:1069F000591C21601A702046BDF81810F2F7FCFEF1
:106A000033E51B4B0A681B781A4D511C03F0020337
:106A10002160137023682A7D591C21601A7029682F
:106A20002046F2F7D2FE69682046F2F7CEFE2989A9
:106A30002046F2F7E1FEE9892046F2F7DDFE204626
:106A4000298AF2F7D9FE012010E500BFB8680020BE
:106A500040880020788800209C760020F07B002071
:106A6000B0450020946200208476002054730020FA
:106A7000B0880020B488002090DE030898680020C9
:106A8000AE4D08462988F2F7B7FE69882046F2F72E
:106A9000B3FE2046A988F2F7AFFE0120E6E4A84D38
:106AA00005F16006A9882046F2F7A6FEE98820468F
:106AB000F2F7A2FE29892046F2F79EFE2368AA7A01
:106AC000591C21601A702368EA7A591C21601A70D7
:106AD00055F80C1B2046F2F778FEAE42E2D1C4E432
:106AE000984952232268501C2060137011F8013F0E
:106AF000002BF7D1B9E4944800232268056803EB22
:106B00004301561C6D5C26601570026825680A44B6
:106B10006E1C527826602A70026825680A44013388
:106B20009278691C0A2B21602A70E6D19DE4874D7A
:106B30000B682A68591C127821601A702B68226829
:106B40009978531C2360002311702A6821681A4425
:106B500001335279481C032B20600A70F5D1236859
:106B60002A68591C127A21601A7023682A68591CF5
:106B7000D27821601A7023682A68591C1279216022
:106B80001A702B6820465989F2F736FE2A68236866
:106B9000527A591C21601A702A680FE000212046A1
:106BA000F2F713FE20460021F2F726FE01205DE4F5
:106BB0000B68674A581C91782060197023685278D6
:106BC000591C216001201A7050E40B6801229918A9
:106BD000216010461A7049E408460021F2F7F5FDDD
:106BE000012043E45B4D5C4E05F1280795F9021046
:106BF0005A4B93F906208A4203F1080300F05182B0
:106C00009E42F6D10835BD42F0D12EE4544B03F13B
:106C10005A0522685979501C206011702268197831
:106C2000501C2060117022685978501C206011702F
:106C300022689978501C206011702268D978501C05
:106C400020601170226819790633501C9D42206023
:106C50001170DED109E40B68424A591C527D216053
:106C600001201A7002E4404D05F1800655F8041F1A
:106C70002046F2F7AAFDAE42F8D1FFF7F6BB3B4D36
:106C800005F14006B5F880102046F2F7B5FD2368FF
:106C900095F88220591C21601A70236895F883208A
:106CA0000435591CB54221601A70EBD1FFF7DDBBEA
:106CB0002C4D0B682A7A591C21601A70A98B20462A
:106CC000F2F79AFD298B2046F2F796FD698B204654
:106CD000F2F792FD2368EA7C591C21601A70A98C96
:106CE0002046F2F789FDE98C2046F2F785FD2368FE
:106CF000AA7F591C21601A70236895F82020591C1E
:106D000021601A70698C2046F2F776FD2368EA7AD2
:106D1000591C21601A70E9682046F2F756FD236875
:106D20002A7C591C21601A70236895F82120591C6F
:106D3000216001201A70FFF799BB00BF3C4500207D
:106D4000206B002060DE0308B8680020ECB0002053
:106D50006C6200207C8F002010780020E8770020F3
:106D6000983E002014780020686700206C6700209F
:106D70000B68AA4A581C1178206019701EE7A84DAC
:106D800008462988F2F738FDA9882046F2F734FD35
:106D900020462989F2F730FD0120FFF767BBA14D9E
:106DA00005F15006287821F02DF82368027A591C45
:106DB00021601A7023686A78591C21601A70236850
:106DC000AA78591C21601A702368EA780435591C86
:106DD000AE4221601A70E5D1FFF747BB924B03F139
:106DE000700522681978501C20601170226859784B
:106DF000501C2060117022689978501C206011701E
:106E00002268D978501C2060117022681979501CB2
:106E10002060117022685979501C2060117022681E
:106E200099790733501C9D4220601170D9D1FFF72A
:106E30001CBB7E4D0846E989F2F7DEFC2046A98995
:106E4000F2F7DAFC0120FFF711BB0B6800255A1C92
:106E50000A601D700B685A1C0A601D700B685A1C72
:106E60000A60204629461D70F2F7AFFC20462946ED
:106E7000F2F7ABFC0120FFF7F9BA6D4D0846298AFD
:106E8000F2F7BAFC698A2046F2F7B6FC2046A98AD6
:106E9000F2F7B2FC0120FFF7E9BADFF8CCE10027F6
:106EA000FEB2714600232268501C206016702268D2
:106EB000501C20601370226811F8010F0133551C1B
:106EC000062B25601070EED10137062F0EF1060E4D
:106ED000E6D1584900232268501C206017702268B0
:106EE000501C20601370226811F8010F0133551CEB
:106EF0000B2B25601070EED123684F4A581C0721D8
:106F00002060197023680021581C206019702368C4
:106F100092F8F020591C216001201A70FFF7A6BAE0
:106F20000B68464A41491078454A5D1C2560187037
:106F300023688978581C2060197023689278591C3E
:106F4000216001201A70FFF791BA3E4D084629884A
:106F5000F2F752FC69882046F2F74EFCB5F904308E
:106F6000394AD91782FB0323C1EBA301204689B21A
:106F7000F2F742FC0120FFF779BA344B0846198832
:106F8000F2F73AFC324B20461988F2F735FC314BC8
:106F900022681B78511C03F001032160012013704B
:106FA000FFF764BA0B682C4E01255A1C0A601D704D
:106FB0000B68B278591921601A7022F09BF8236887
:106FC000264A27495F1927601870B1F90010B2F9F5
:106FD0000000F2F78BFD23685A192260187031887F
:106FE0002046F2F709FC2846FFF740BA0A681D4B15
:106FF000501C19782060117022685978501C20604C
:10700000117022689978501C206011702268DB781A
:10701000511C216001201370FFF728BAD0620020B4
:10702000C03D0020D4620020146C0020506200207B
